:1010000000000420250A0200690A02006B0A02009F
:101010006D0A02006F0A0200710A0200000000005F
:10102000000000000000000000000000730A020041
:10103000750A020000000000770A0200790A020027
:101040003D9F01001D7B01007B0A02007B0A02001C
:101050007B0A02007B0A02007B0A02007B0A020074
:101060007B0A02007B0A02007B0A02007B0A020064
:101070007B0A0200B18200007B0A02007B0A0200A8
:101080007B0A02007B0A02007B0A02007B0A020044
:101090007B0A02007B0A02007B0A02007B0A020034
:1010A0007B0A02007B0A02007B0A02007B0A020024
:1010B0007B0A02007B0A0200000000000000000022
:1010C0007B0A02007B0A02007B0A02007B0A020004
:1010D000216500007B0A02007B0A0200FDBA0100C4
:1010E0007B0A02007B0A02007B0A0200000000006B
:1010F000000000007B0A0200000000007B0A0200E2
:1011000000000000000000000000000000000000DF
:1011100000000000000000000000000000000000CF
:1011200000000000000000000000000000000000BF
:1011300000000000000000000000000000000000AF
:10114000000000000000000000000000000000009F
:10115000000000000000000000000000000000008F
:10116000000000000000000000000000000000007F
:10117000000000000000000000000000000000006F
:10118000000000000000000000000000000000005F
:10119000000000000000000000000000000000004F
:1011A000000000000000000000000000000000003F
:1011B000000000000000000000000000000000002F
:1011C000000000000000000000000000000000001F
:1011D000000000000000000000000000000000000F
:1011E00000000000000000000000000000000000FF
:1011F00000000000000000000000000000000000EF
:1012000010B5054C237833B9044B13B10448AFF340
:1012100000800123237010BDE800002000000000C2
:101220001C55020008B5034B1BB103490348AFF33B
:10123000008008BD00000000EC0000201C550200EA
:10124000154B002B08BF134B9D46A3F5803A002198
:101250008B460F461348144A121A20F0F1FE0F4B2A
:10126000002B00D098470E4B002B00D09847002051
:10127000002104000D000D48002802D00C48AFF3F7
:10128000008020F083FE2000290000F01DF820F0EF
:1012900057FE00BF0000080000000420000000000E
:1012A00000000000E800002068540020000000005A
:1012B0000000000080B483B000AF786000BF0C373E
:1012C000BD465DF8047B704780B584B000AF7860A0
:1012D00039603968786806F02BFC07F0DDFBF860B0
:1012E000FB68002B05D10E4B0E4A5D210E4820F005
:1012F00009FEF86800F04EF805E0F86808F001F91A
:10130000F86806F07BFC06F06DFC034683F00103F1
:10131000DBB2002BF1D1F86807F0D0FBD9E700BFB2
:10132000A8340200DC340200B434020080B483B07C
:1013300000AF0346FB7100BF0C37BD465DF8047B70
:10134000704780B582B000AF78600B467B807B88A9
:101350001946786800F04CFA00BF0837BD4680BDDA
:1013600080B500AF00F01FFA00BF80BD80B582B02D
:1013700000AF78600B467B807B881946786807F061
:1013800005FB03461846FFF7D1FF7B881846083750
:10139000BD4680BD80B582B000AF786007F0E8FA46
:1013A00003461846FFF7C2FF0349786800F050F87B
:1013B00000BF0837BD4680BD6D13000080B483B008
:1013C00000AF0346FB7100BF0C37BD465DF8047BE0
:1013D000704780B483B000AF78607B6800221A60E9
:1013E0007B6800229A807B6818460C37BD465DF802
:1013F000047B704780B483B000AF786039607B684D
:1014000018460C37BD465DF8047B704780B584B044
:1014100000AFF860B9607A60B968F868FFF7EAFF72
:10142000FB687A681A60FB6800225A60FB681846FD
:101430001037BD4680BD80B483B000AF786039609E
:101440003B6818460C37BD465DF8047B70470000CA
:1014500090B585B000AF786039600023FB607B6891
:10146000BB60104B194641F27830FFF7E4FF0446A9
:101470003A68B968204600F017F8FC60FB68002B5A
:1014800005D000F003FF0246FB68934201D0012320
:1014900000E00023002B00D0FEE700BF1437BD465C
:1014A00090BD00BF0801002080B584B000AFF86097
:1014B000B9607A60FB68B968184600F00FFEFB68F7
:1014C0007A68C3F83829FB6803F63C12FB6803F618
:1014D0005813194610460DF06EF8FB6803F64410D9
:1014E000FB6803F58B510431FB681B4A0DF041F991
:1014F000FB6803F65813184600F066FAFB6803F51C
:101500008B5300221A70FB6803F58B5301330022C2
:101510001A70FB6803F58B530433184600F064FA25
:10152000FB6803F59B530C3300221A70FB6803F52C
:101530009B531033094AB9681846FFF767FFFB68E9
:101540000433FA68064918460DF07EFAFB6818461F
:101550001037BD4680BD00BF43180000B315000022
:101560006515000080B584B000AFF860B9603B60DD
:101570001346FB71F86800F004F800BF1037BD4651
:1015800080BD80B582B000AF78607B6803F65813E9
:10159000184600F039FA0346002B06D07B6803F5A5
:1015A0009B531033184608F001FA00BF0837BD46B8
:1015B00080BD80B582B000AF786000F067FE034662
:1015C000184600F004F800BF0837BD4680BD90B54E
:1015D00087B000AF78607B6804337B6178690DF079
:1015E00006FE034683F00103DBB2002B05D17B68C6
:1015F00003F58B531B78022B01D1012300E000235C
:10160000002B00F0A6807B6803F58B531B78022B20
:101610007CD0022BE2DC002B02D0012B40D097E0E3
:101620007B68184600F06BFF0346002B01D005F0E5
:101630007DF87B68184600F07CFF0346002B40F0E5
:101640008A807B6803F63C1318460CF0C6FF0346FD
:10165000002B14BF01230023DBB2002B7DD178695E
:101660000DF068FE03461846FFF7A8FE7B6803F5F9
:101670008B5301221A7000E000BF78690DF084FEE0
:10168000034683F00103DBB2002B1ED078690DF016
:1016900093FE03461A467B6803F58B5301331A7099
:1016A0007B6803F63C127B6803F58B5301331B7890
:1016B000194610460CF0A4FF0346002B14BF01236B
:1016C0000023DBB2002BD7D04AE07B6893F8983038
:1016D000FB7478690DF0B2FE03461846FFF76EFE04
:1016E000FB7C002B0DD07B6893F8983083F00103CE
:1016F000DBB2002B05D07B6803F59B530C33012232
:101700001A707B6803F58B5302221A707B6803F60C
:101710003C1318460CF0CEFF0346002B14BF0123E8
:101720000023DBB2002B1AD17B6803F58B53002218
:101730001A707B6803F59B530C331B78002B3FF426
:101740004DAF7B6803F59B530C3300221A7000BF2A
:1017500044E700BF04E000BF02E000BF00E000BFBC
:101760007B6803F65813184600F061F903463B8284
:101770003B8A002B13D07B68D3F838497B6803F68B
:101780005813184600F063F902463B8A1946104682
:10179000A047F8603B8AFA689A4200D0FEE700BF93
:1017A0001C37BD4690BD80B582B000AF00F06EFD25
:1017B00078607B68002B02D0786800F004F800BFE6
:1017C0000837BD4680BD80B582B000AF78607B68C9
:1017D00003F65813184600F046F97B6803F59B534F
:1017E0001033184608F0E2F800BF0837BD4680BD48
:1017F00080B584B000AF78600B467B8000F046FD7A
:10180000F860FB68002B05D07B881A467968F86879
:1018100000F004F800BF1037BD4680BD80B584B02D
:1018200000AFF860B9601346FB80FB6803F6441311
:10183000FA88B96818460CF0BCFF00BF1037BD46E7
:1018400080BD80B582B000AF78600B46FB70FB783E
:101850001946786800F004F800BF0837BD4680BD1F
:1018600080B584B000AF78600B46FB707B6803F5F1
:101870008B530433184600F008F9F8607B6803F5D1
:101880008B530433184600F00CF903467B81FB7838
:10189000002B06D17B687A89F968184600F02AFD8A
:1018A00005E07B89F978FA68786800F00BF87B68C6
:1018B00003F58B530433184600F003F900BF1037CB
:1018C000BD4680BD90B5A7B000AFF8607A601A46FB
:1018D0000B46FB7213463B810023A7F89630FB684A
:1018E000184600F040FEFB7A07F11400334A8021CD
:1018F00020F0C0FE07F11403184620F0EFFE034667
:101900001A4607F114031946002002F04EFC034664
:101910001846FFF753FD0023A7F89630B7F8962036
:101920003B899A4220D2B7F89630282B1CD8B7F8BA
:10193000962013465B00134407F11402D018B7F841
:10194000962013465B001344C3F18001B7F896302C
:101950007A6813441B781A4A20F08CFEB7F8963048
:101960000133A7F89630D9E7B7F8962013465B0005
:10197000134407F11402D018B7F8962013465B0001
:101980001344C3F180030F4A194620F073FE07F198
:101990001404013407F11403184620F09FFE034697
:1019A000013B1A462146002002F0FFFB0346184681
:1019B000FFF704FD00BF9C37BD4690BDE434020034
:1019C000F83402000035020080B582B000AF7860C4
:1019D0007B681846FFF7FDFC786800F044F87B68E8
:1019E00018460837BD4680BD80B582B000AF78602C
:1019F0007B681846FFF7EDFC786800F062F87B68BA
:101A000018460837BD4680BD80B483B000AF78600B
:101A10007B681A687B6806339A420CBF0123002357
:101A2000DBB218460C37BD465DF8047B704780B4C6
:101A300083B000AF78607B681A687B680633D31A7E
:101A40009BB218460C37BD465DF8047B704780B4E6
:101A500083B000AF78607B68063318460C37BD460C
:101A60005DF8047B704780B483B000AF78607B681A
:101A70009A1D7B681A607B684FF400629A8000BFF1
:101A80000C37BD465DF8047B704780B483B000AF6F
:101A900078607B68063318460C37BD465DF8047BDA
:101AA000704780B483B000AF78607B681A687B6849
:101AB0000633D31A9BB218460C37BD465DF8047B3B
:101AC000704780B483B000AF78607B689A1D7B68F4
:101AD0001A607B684FF400729A8000BF0C37BD46D5
:101AE0005DF8047B704780B483B000AF786079689C
:101AF0004FF000024FF00003C1E9002379684FF076
:101B000000024FF00003C1E902237B6818460C373E
:101B1000BD465DF8047B704780B483B000AF786049
:101B20007B68D3E900231343002B0CBF0123002360
:101B3000DBB218460C37BD465DF8047B704780B5B4
:101B400082B000AF786039603A680021786803F0AD
:101B500034FC00BF0837BD4680BD000080B582B0B0
:101B600000AF78603960786803F01CFC03461A46C1
:101B70003B681A70024B18460837BD4680BD00BF4F
:101B80004038020080B582B000AF78600B46FB7031
:101B90007B68D3E90001FB781A4600F053F803464E
:101BA00018460837BD4680BD80B582B000AF78606A
:101BB0000B46FB707B68FA781146184600F016F861
:101BC00000BF0837BD4680BD80B582B000AF7860E9
:101BD0000B46FB707B68D3E90201FB781A4600F0E4
:101BE00031F8034618460837BD4680BD2DE9F04F51
:101BF00083B000AF7860F9707968D1E900ABFE7806
:101C00004FF001004FF00001A6F1200EC6F1200CAC
:101C100001FA06F300FA0EFE43EA0E0320FA0CFC6A
:101C200043EA0C0300FA06F2D443DD430AEA04084F
:101C30000BEA05097B68C3E9008900BF0C37BD4684
:101C4000BDE8F08F2DE9F00384B000AFC7E90201D1
:101C50001346FB71F979D7E90223C1F12006A1F1FE
:101C6000200022FA01F403FA06F6344323FA00F0C6
:101C7000044323FA01F54FF001024FF0000304EA98
:101C8000020805EA030948EA0903002B14BF0123EF
:101C90000023DBB218461037BD46BDE8F00370479D
:101CA00080B483B000AF0346FB7100BF0C37BD4664
:101CB0005DF8047B704780B483B000AF78607B68C8
:101CC00000221A607B6800225A607B6818460C3735
:101CD000BD465DF8047B704780B582B000AF786088
:101CE00039600822396878680DF0F2FE034618461C
:101CF0000837BD4680BD80B483B000AF78607B6894
:101D00001A897B68DB88D31A9BB218460C37BD460C
:101D10005DF8047B704780B483B000AF78607B6867
:101D2000DA887B681B899A420CBF01230023DBB24F
:101D300018460C37BD465DF8047B7047B0B582B0DD
:101D400000AF786039607B683A681A607B6804335A
:101D500003241D46002C05DB2846FFF7ACFF0835A1
:101D6000013CF7E77B68002283F824207B6800228F
:101D700083F825207B6828331846FFF79CFF7B6893
:101D800018460837BD46B0BD80B582B000AF786058
:101D90000B46FB707B681A68FB78002B01D001238F
:101DA00000E00023194610460DF054F8034618468B
:101DB0000837BD4680BD80B582B000AF78600B4665
:101DC000FB707B681B68FA78114618460DF042F8E4
:101DD000034618460837BD4680BD80B582B000AFC7
:101DE00078600B46FB70FB7819467868FFF7E3FFD5
:101DF000034618460837BD4680BD80B582B000AFA7
:101E0000786039603B681946786800F005F8034649
:101E100018460837BD4680BD80B582B000AF7860F7
:101E2000396008223968786800F005F803461846DA
:101E30000837BD4680BD80B584B000AFF860B9609A
:101E40001346FB80FB681B68FA88B96818460DF0DA
:101E50002BF8034618461037BD4680BD80B483B0CA
:101E600000AF78607B6893F8D2287B6893F8D3380A
:101E70009A420CBF01230023DBB218460C37BD4643
:101E80005DF8047B704780B584B000AFF8600B4606
:101E90007A60FB72F97A7B680022F86800F035FC02
:101EA000034618461037BD4680BD80B584B000AFEC
:101EB000F8600B467A60FB72F97A7B680122F86859
:101EC00000F023FC034618461037BD4680BD80B5A0
:101ED00084B000AFF8600B467A60FB72F97A7B68D9
:101EE0000222F86800F011FC034618461037BD4680
:101EF00080BD80B483B000AF78607B68002B07D0D2
:101F00007B685A1E7B681340002B01D1012300E03F
:101F1000002318460C37BD465DF8047B704780B43B
:101F200085B000AF78600023FB737B685B087B6043
:101F30007B68002B14BF01230023DBB2002B03D0EE
:101F4000FB7B0133FB73F0E7FB7B18461437BD4680
:101F50005DF8047B7047000080B485B000AF034695
:101F6000FB71FB791C2B6DD801A252F823F000BF46
:101F7000E51F0000EB1F0000F11F0000F71F00002D
:101F800045200000FD1F0000032000000920000084
:101F900045200000452000004520000045200000AD
:101FA0000F200000152000001B2000002120000051
:101FB000452000004520000045200000332000009F
:101FC0004520000045200000452000002D20000095
:101FD0002720000045200000452000003920000097
:101FE0003F2000000023FB6031E00123FB602EE076
:101FF0000E23FB602BE00B23FB6028E00C23FB602F
:1020000025E00923FB6022E00323FB601FE002239D
:10201000FB601CE00423FB6019E01123FB6016E069
:102020001223FB6013E01323FB6010E01423FB601A
:102030000DE01623FB600AE01723FB6007E018237E
:10204000FB6004E0FB7903F58043FB6000BFFB68A5
:1020500018461437BD465DF8047B704780B485B0E0
:1020600000AF0346FB71FB79082B2DD801A252F873
:1020700023F000BF992000009F200000A520000051
:10208000AB200000B1200000B7200000C3200000FA
:10209000C9200000BD2000007023FB6017E0712301
:1020A000FB6014E07223FB6011E07323FB600EE021
:1020B0007423FB600BE07523FB6008E07823FB6072
:1020C00005E07623FB6002E07723FB6000BFFB683E
:1020D00018461437BD465DF8047B704780B582B062
:1020E00000AF786039607B683A681A607B68181DB9
:1020F0007B68D1334FF4006219460CF037FC7B68E3
:1021000003F150027B68043319461046FFF716FEB0
:102110007B68803318460DF094FA7B68002283F8C0
:1021200098207B680022C3F89C207B68524AC3F841
:10213000A0207B68C822A3F8A4207B68002283F833
:10214000A6207B68002283F8A7207B684FF6FF72E9
:10215000A3F8A8207B68AC33484A39681846FFF7D3
:1021600055F97B680022C3F8B4207B68B833184661
:10217000FFF7B9FC7B68042283F8C820404B1A683B
:102180007B68C3F8CC207B68002283F8D0207B6872
:10219000002283F8D1287B68002283F8D2287B684C
:1021A000002283F8D3287B68002283F810297B68FB
:1021B000002283F811297B68002283F812297B68AA
:1021C000002283F813297B68002283F814297B6896
:1021D000002283F815297B68002283F816297B6882
:1021E000FF2283F817297B68002283F818297B686F
:1021F0000022C3F81C297B680022C3F820297B68D1
:102200000022C3F824297B680022C3F828297B68B0
:10221000002283F82C297B6803F513614FF000023C
:102220004FF00003C1E900237B681B68002B00D13D
:10223000FEE7144A7B6813607B6804337A681249AE
:1022400018460CF013FC7B6803F6D4033C220021F3
:1022500018461FF0F5FE7B68B83377211846FFF764
:102260006EFC7B68AC33184607F0A0FB7B68184611
:102270000837BD4680BD00BF00F8FF076F2900008A
:10228000343F0200801400203924000080B400AFE5
:10229000034B1B681846BD465DF8047B704700BFC2
:1022A0008014002080B483B000AF78607B68002287
:1022B000C3F81C297B680022C3F820297B68002210
:1022C000C3F824297B680022C3F8282900BF0C37F3
:1022D000BD465DF8047B704780B582B000AF786082
:1022E0007B68043318460CF05BFF0346184608373A
:1022F000BD4680BD90B587B000AFF860B9601346A9
:10230000FB800023FB7500237B750023BB75FB68F6
:10231000012283F81429FB688033FA88B9681846CB
:102320000DF0B2F9FB68042283F8C820FB68002294
:1023300083F89820FB68803307F115021146184690
:102340000DF002FA0346002B14BF01230023DBB279
:10235000002B66D17B7D5BB2002B64DAFB68D3F87F
:1023600020395A1CFB68C3F820297B7D1B1103F020
:102370000303002B0AD07B7D06221946F86800F083
:1023800035FD03461846FFF78BFC4DE07B7D194673
:10239000F86800F080FB0346FB75FB7D002B0ED038
:1023A0007C7DFB7D1846FFF7D7FD03461A46214684
:1023B000F868FFF78CFD03461846FFF771FCF868D4
:1023C000FFF74CFD034683F00103DBB2002B06D080
:1023D000F86800F03CFA03461846FFF761FC7B7D85
:1023E00003F00F03BB75FB6893F8D138002B0CD0BA
:1023F000FB6893F8D138BA7D9A4206D0FB68D3F8CF
:1024000024395A1CFB68C3F82429BB7D0E2B03D842
:10241000BB7D0133DAB200E00122FB6883F8D128EA
:1024200002E000BF00E000BFFB68002283F814292F
:1024300000BF1C37BD4690BD80B584B000AFF860CA
:10244000B9603B601346FB71B968F86800F004F8A6
:1024500000BF1037BD4680BD80B582B000AF786048
:1024600039607B6893F89830002B09D07B68D3F8EB
:10247000CC303A689A4203D17B68002283F89820D6
:10248000786800F0E4F90346002B14BF0123002311
:10249000DBB2002B2CD17B6893F8D030002B23D0FB
:1024A0007B6893F8D01001230C22786800F0EAFCD6
:1024B0000346002B14BF01230023DBB2002B19D1EC
:1024C0007B68002283F8D0207B6893F8C830042B07
:1024D0000AD07868FFF700FF02467B68C3F8CC207B
:1024E0007B68012283F89820786800F04EFA02E0B9
:1024F00000BF00E000BF00BF0837BD4680BD80B40C
:1025000083B000AF78607B6893F8C830042B09D0A3
:102510007B6893F8983083F00103DBB2002B01D085
:10252000012300E0002318460C37BD465DF8047B0C
:10253000704780B483B000AF78607B6893F8C83090
:10254000012B09D17B6893F8983083F00103DBB24B
:10255000002B01D0012300E0002318460C37BD46B4
:102560005DF8047B704780B483B000AF78607B680F
:10257000D3F81C395A1C7B68C3F81C2900BF0C37E0
:10258000BD465DF8047B704780B588B000AFF86049
:10259000B9607A603B600023FB778023FB75BB68E2
:1025A000002B02D17023BB6101E0BB68BB61FB68FB
:1025B00093F81439002B02D00D23FB774DE0FB6814
:1025C000B833B969184602F081FF0346002B02D0E8
:1025D0000D23FB7741E0F868FFF740FC034683F0EA
:1025E0000103DBB2002B02D00323FB7735E0FB684D
:1025F00003F15000F97DBB6906220DF080FB034614
:10260000FB77FB7F002B14BF01230023DBB2002BE1
:1026100020D1FB6850333A6892B279681846FFF7C8
:102620000AFC0346FB77FB7F002B14BF012300232A
:10263000DBB2002B10D1FB68503318460DF0D4FBF1
:102640000346FB77FB7F002B14BF01230023DBB283
:10265000002B02E000BF00E000BFFB7F032B0AD18C
:10266000FB68B8330B211846FFF769FAFB68AC33F7
:10267000184607F09BF9FB7F18462037BD4680BD02
:1026800080B485B000AF78600023FB737B68052BB6
:1026900020D801A252F823F0B1260000B72600008E
:1026A000BD260000C3260000C9260000CF2600007A
:1026B0000023FB730EE00223FB730BE00423FB7388
:1026C00008E00523FB7305E00623FB7302E0072304
:1026D000FB7300BFFB7B18461437BD465DF8047BD7
:1026E000704700BF80B483B000AF0346FB71FB7935
:1026F0000E2B03D9FB790F3BFB71F8E7FB791846EA
:102700000C37BD465DF8047B704780B586B000AFDE
:10271000F8607B600B46FB721346BB720023FB75AF
:10272000FB7A03F00F037B757B7D002B0AD1BB7A0C
:10273000022B40F08680FB68B83379681846FFF7B3
:10274000FEF97EE0FB6893F8D3381A46FB6893F8ED
:10275000D238D31A0E2B08DDFB68B8330E21184689
:10276000FFF7EDF90323FB756CE0FB6893F8D138B4
:102770007A7D9A422FD0FB6893F8D238BB75FB68FC
:1027800093F8D338BA7D9A4225D2BB7D1846FFF71D
:10279000A9FF034603F50D739B00FA681344043345
:1027A0003B613B691B78C3F30013DBB2002B0ED0F7
:1027B0003B691B78C3F30303DBB21A467B7D9A4265
:1027C00005D13A6913786FF30413137003E0BB7DEE
:1027D0000133BB75D3E7FB6893F8D3381846FFF78E
:1027E00081FF034603F50D739B00FA68134404331D
:1027F0003B617B7D03F00F03D9B23A69137861F333
:10280000030313703A69137843F010031370BB7A13
:1028100003F00303D9B23A69137861F346131370D6
:102820007B6823F07F413A69136861F3DE1313601C
:10283000FB6893F8D3380133DAB2FB6883F8D32806
:1028400000E000BFFB7D18461837BD4680BD80B54F
:1028500088B000AF78600023FB777B6893F8D228BC
:102860007B6893F8D3389A4279D07B6893F8D23852
:1028700003F50D739B007A6813440433BB61BB6995
:102880001B78C3F30013DBB2002B46D08023FB750B
:10289000BB691B78C3F30303DBB21A46FB7D13430A
:1028A000FB75BB691B7803F06003DBB2402B15D1CD
:1028B000BB691B68C3F3D713BB60FB7DBA681946BD
:1028C000786800F093FA0346FB77FB7F002B14BF78
:1028D00001230023DBB2002B1FD043E0BB691B6840
:1028E000C3F3D7133B61BB691B7803F06003DBB212
:1028F000002B0CBF01230023FB73FB7BF97D3A699E
:10290000786800F0BFFA0346FB77FB7F002B14BF0B
:1029100001230023DBB2002B23D1BA6913786FF3B4
:10292000041313707B6893F8D2380133DAB27B68F2
:1029300083F8D2287B6893F8D2380F2B8DD17B682F
:10294000002283F8D2287B6893F8D3381846FFF723
:10295000C9FE03461A467B6883F8D3287DE700BF8B
:1029600000E000BFFB7F18462037BD4680BD80B524
:1029700082B000AF7860FFF789FC0346184600F08C
:1029800004F800BF0837BD4680BD80B588B000AFF1
:1029900078607B68B8331846FFF7BEF80346002B13
:1029A0006AD17B68B83307F10F0211461846FFF76A
:1029B000D5F8F8610023FB76FB7BFA7E9A425DD264
:1029C0007B68B833FA7E11461846FFF7DBF80346FA
:1029D00083F00103DBB2002B46D1FB691B683B612E
:1029E0003B69002B1DD1FB695B687B617B69772BA1
:1029F00009D17B681B68184603F040FE0346184661
:102A0000FFF72CFB78617A698021786800F0EEF995
:102A10000346002B14BF01230023DBB2002B13D08D
:102A200031E07B6893F82C39002B0DD001233A69F3
:102A30008021786800F026FA0346002B14BF01239A
:102A40000023DBB2002B1BD17B68B833FA7E114622
:102A50001846FFF7A9F87B68B8331846FFF75CF80B
:102A60000346002B0ED100E000BFFB7E0133FB7656
:102A7000FB690C33FB619FE700BF04E000BF02E08D
:102A800000BF00E000BF7B68012283F82C2900BF53
:102A90002037BD4680BD80B584B000AF78600B465E
:102AA000FB700023FB737B68803307F1080211463B
:102AB00018460CF0DEFF0346FB73FB7B002B14BFB4
:102AC00001230023DBB2002B2BD1BB68052B1FD8C1
:102AD000022B14D2002B02D0012B08D018E0FB7877
:102AE0001946786800F097FA0346FB731AE0FB7802
:102AF0001946786800F0A0FA0346FB7312E0BA6842
:102B0000FB781946786800F0FBFA0346FB7309E08E
:102B1000FB78052219467868FFF7D9F90346FB735D
:102B200000E000BFFB7B18461037BD4680BD80B576
:102B300086B000AFF8607A603B600B46FB72012301
:102B4000FB757B680C2B03D07B68712B0AD013E0DC
:102B5000FB7A1946F86801F007F803461A463B6805
:102B60001A700CE0FB7A1946F86802F0D9FA0346AD
:102B70001A463B681A7002E00023FB7500BFFB7D1C
:102B800018461837BD4680BD80B588B000AFF860E4
:102B90000B467A60FB720023BB7707F11403796858
:102BA000184601F02FFB7B69002B06D1BB6903F0AF
:102BB0000103002B01D1012300E00023012B21D0D0
:102BC000FB68002283F81429BB695B101A46FB6876
:102BD0001A44BB6903F00103002B09D0BB695B10E9
:102BE0001946FB680B441B6879690B441B6800E0BD
:102BF0007B69104698470346BB77FB68012283F840
:102C000014291AE007F11E03F97A7A68F868FFF7C9
:102C10008EFF0346FB77FB7F002B27D1FB7F83F0E2
:102C20000103DBB2002B08D0FB7A0D221946F868AD
:102C3000FFF74DF90346BB7719E0BB7F002B08D1A6
:102C4000FB7A7A681946F868FFF72FF90346BB77D5
:102C50000DE0BB7F1846FFF77FF90246FB7A194665
:102C6000F868FFF734F90346BB7700E000BFBB7F8D
:102C700018462037BD4680BD80B58EB002AF786162
:102C8000FA60BB600B46FB74002387F82F300023EB
:102C90003B6200237B620023BB62BB68042B03D032
:102CA000BB68052B09D017E007F12003F968184627
:102CB00001F0BAFA0723BB620FE03B46F9681846F9
:102CC00001F0C4FA07F120033A4692E8030083E8D2
:102CD00003000823BB6200E0FEE73B6A002B06D13D
:102CE0007B6A03F00103002B01D1012300E00023E4
:102CF000002B09D0FB7C0D2219467869FFF7E7F815
:102D0000034687F82F306BE07B69803318460CF060
:102D100057FF7B69803307F11A0207F11C0118463F
:102D20000CF000FF03461846FEF7BAFF7B698033BC
:102D300018460CF05BFF03461846FEF7B1FF7B69AF
:102D4000002283F814297B6A5B101A467B691A44B7
:102D50007B6A03F00103002B09D07B6A5B101946E4
:102D60007B690B441B68396A0B441B6800E03B6AB3
:102D700010469847034687F82F307B69012283F875
:102D8000142997F82F30002B0ED097F82F301846C3
:102D9000FFF7E2F80246FB7C19467869FFF797F8DF
:102DA000034687F82F301BE0FB697A8BF97C019290
:102DB0000093FB68BA6A786900F0E9F8034687F87F
:102DC0002F3097F82F30002B09D0FB7C00221946BA
:102DD0007869FFF77CF8034687F82F3000E000BFE2
:102DE00097F82F3018463037BD4680BD80B586B085
:102DF00000AFF8600B467A60FB720023FB75FB7A2C
:102E00001B1103F00303002B03D1FB687A68C3F89E
:102E10009C20FB6803F15000F97A002306220CF095
:102E20006EFF0346FB75FB7D002B14BF01230023BF
:102E3000DBB2002B1ED1FB685033796818460DF0C9
:102E40006DF90346FB75FB7D002B14BF01230023A6
:102E5000DBB2002B10D1FB68503318460CF0C4FFD6
:102E60000346FB75FB7D002B14BF01230023DBB25F
:102E7000002B02E000BF00E000BFFB7D18461837C2
:102E8000BD4680BD80B588B000AFF8607A601A4654
:102E90000B46FB721346BB720023FB7707F114034A
:102EA0007968184601F09CF97B69002B06D1BB6953
:102EB00003F00103002B01D1012300E00023012BCB
:102EC0003AD0FB6803F15000F97A7B6806220CF0D7
:102ED00016FF0346FB77FB7F002B14BF0123002363
:102EE000DBB2002B4BD1BB695B101A46FB681A445E
:102EF000BB6903F00103002B09D0BB695B101946C5
:102F0000FB680B441B6879690B441B6800E07B6914
:102F1000104698470346FB77FB7F002B14BF012325
:102F20000023DBB2002B2CD1FB68503318460CF089
:102F30005BFF0346FB7725E0BB7A002B0FD0FB7AC3
:102F40000D221946F868FFF751FF0346FB77FB7F18
:102F5000002B14BF01230023DBB2002B12E0FB7A0D
:102F600000221946F868FFF741FF0346FB77FB7F15
:102F7000002B14BF01230023DBB2002B02E000BFB3
:102F800000E000BFFB7F18462037BD4680BD80B5FE
:102F900086B000AFF8607A603B600B46FB7200239E
:102FA000FB75FB6803F15000F97A3B687A680CF016
:102FB000A6FE0346FB75FB7D002B14BF01230023F7
:102FC000DBB2002B1FD1FB685033BA8C396A18462C
:102FD000FEF731FF0346FB75FB7D002B14BF012379
:102FE0000023DBB2002B10D1FB68503318460CF0E5
:102FF000FBFE0346FB75FB7D002B14BF0123002362
:10300000DBB2002B02E000BF00E000BFFB7D1846F2
:103010001837BD4680BD80B582B000AF78600B46E2
:10302000FB70FB78002219467868FEF750FF0346D4
:1030300018460837BD4680BD80B584B000AF7860C3
:103040000B46FB700023FB730223BB737B6880334A
:103050001846FEF750FE0346002B14BF0123002341
:10306000DBB2002B12D07B68803307F10E021146D1
:1030700018460CF069FB0346FB73FB7B002B14BF67
:1030800001230023DBB2002B00D0FEE7BB7B022B29
:1030900027D17B681B68184605F02EFD7B6800224F
:1030A00083F812297B68002283F816297B68FF22A7
:1030B00083F817297B68002283F818297868FFF7BE
:1030C000F1F8702280217868FFF790FE0346FB73C9
:1030D000FB7B002B14BF01230023DBB2002B08D0A5
:1030E000FEE77B681B68184605F0F7FC034B0022DF
:1030F0001A60FB7B18461037BD4680BD8014002047
:1031000080B586B000AFF8600B467A60FB72002392
:10311000FB7500233B61FB68803307F11002114609
:1031200018460CF0A6FC0346FB75FB7D002B0CD06B
:10313000FB7D1846FEF710FF0246FB7A1946F86839
:10314000FEF7C5FE0346FB7528E07B68052B24D8F7
:103150007B68042B18D27B68022B03D07B68032B7F
:1031600009D01AE03A69FB7A1946F868FEF78BFE37
:103170000346FB7512E03A69FB7A1946F868FFF7D7
:1031800003FD0346FB7509E03A69F97A7B68F86844
:10319000FFF772FD0346FB7500E000BFFB7D18469C
:1031A0001837BD4680BD90B583B000AF78607B68AE
:1031B00003F150047B681B68184605F03CFE03468B
:1031C00019462046FEF7E0FD034618460C37BD467B
:1031D00090BD90B583B000AF78607B6803F1500478
:1031E0007B681B68184606F0A5F80346194620467A
:1031F000FEF7E1FD034618460C37BD4690BD80B58D
:1032000084B000AF78600023BB600023FB737B6851
:10321000803307F10802114618460CF02AFC0346D9
:10322000FB73FB7B002B14BF01230023DBB2002BBD
:1032300026D17B681B68BA68D2B21146184606F0E0
:103240008DF80346FB73FB7B002B1BD17B681B684F
:10325000184605F0F0FD0346002B06D07B6893F876
:103260001239002B01D0012300E00023002B0BD0EA
:103270007B681B68184605F070FE0346FB7304E08C
:1032800000BF02E000BF00E000BFFB7B1846103724
:10329000BD4680BD80B584B000AF78607B681B6898
:1032A000184605F0F4FD0346FB737B6803F15002FA
:1032B000FB7B002B01D0022300E0002319461046BF
:1032C000FEF779FD034618461037BD4680BD80B530
:1032D00084B000AF78600023BB730023FB737B686E
:1032E000803307F10E02114618460CF02DFA034602
:1032F000FB73FB7B002B14BF01230023DBB2002BED
:103300001DD1BB7B002B05D0002B15DB013B012B16
:1033100012D808E07B681B680021184605F0CBFD39
:103320000346FB730CE07B681B680121184605F01F
:10333000C2FD0346FB7303E00723FB7300E000BFFD
:10334000FB7B18461037BD4680BD90B583B000AFFB
:1033500078607B6803F150047B681B68184606F0B0
:1033600015F80346194620460CF065FD034618463D
:103370000C37BD4690BD80B584B000AF78600023A7
:10338000FB737B68803307F10C02114618460CF082
:1033900023FA0346FB73FB7B002B14BF012300239E
:1033A000DBB2002B09D17B681B68BA89114618462D
:1033B00006F000F80346FB7300E000BFFB7B1846F5
:1033C0001037BD4680BD90B583B000AF78607B6894
:1033D00003F150047B681B68184606F003F80346A7
:1033E00019462046FEF709FD034618460C37BD4630
:1033F00090BD80B584B000AF78600023FB737B681C
:10340000803307F1080211461846FEF765FC0346B3
:10341000FB73FB7B002B14BF01230023DBB2002BCB
:1034200009D17B681B68BA681146184605F0EEFFA3
:103430000346FB7300E000BFFB7B18461037BD4618
:1034400080BD90B583B000AF78607B6803F1500415
:103450007B681B68184605F0F3FF034619462046B3
:103460000CF0E9FC034618460C37BD4690BD80B50C
:1034700082B000AF78607B6803F150027B6893F8FC
:10348000123919461046FEF77FFC034618460837E6
:10349000BD4680BD80B584B000AF78600023BB73AB
:1034A0000023FB737B68803307F10E021146184638
:1034B0000CF01CF90346FB73FB7B002B14BF0123AC
:1034C0000023DBB2002B1ED17B681B68184605F079
:1034D000B2FC0346002B11D0BB7B002B07D07B68CE
:1034E0001B68184605F039FD0346FB7306E07B6850
:1034F0001B68184605F009FD0346FB73BA7B7B6821
:1035000083F8122900E000BFFB7B18461037BD4648
:1035100080BD90B583B000AF78607B6803F1500444
:103520007B681B68184609F043FC03461946204691
:10353000FEF741FC034618460C37BD4690BD90B5DA
:1035400083B000AF78607B6803F150047B681B6830
:10355000184609F038FC034619462046FEF72BFCB6
:10356000034618460C37BD4690BD80B584B000AF09
:10357000786039600023FB730023BB73BB7B1F2B78
:103580001DD8BB7B012202FA03F31A463B681340A5
:10359000002B10D07B685033BA7B11461846FEF7DB
:1035A0000AFC0346FB73FB7B002B14BF01230023A3
:1035B000DBB2002B05D1BB7B0133BB73DEE700BF61
:1035C00000E000BFFB7B18461037BD4680BD80B5CC
:1035D00084B000AF786039600023FB733B68002241
:1035E0001A607B6880331846FEF795FB034683F02C
:1035F0000103DBB2002B21D07B68803307F10E0280
:10360000114618460CF0A0F80346FB73FB7B002B19
:1036100014BF01230023DBB2002B11D1BB7B1F2B76
:1036200002D90723FB730CE03B681A68BB7B194681
:1036300001238B401A433B681A60D2E700BF00E0C9
:1036400000BFFB7B18461037BD4680BD80B582B0F9
:1036500000AF78607B68D3F8A03019467868FFF730
:1036600084FF034618460837BD4680BD80B584B048
:1036700000AF78600023BB600023FB7307F10803F1
:1036800019467868FFF7A3FF0346FB73FB7B002B0B
:1036900014BF01230023DBB2002B04D1BA687B687E
:1036A000C3F8A02000E000BFFB7B18461037BD46E2
:1036B00080BD80B582B000AF78607B6803F15002B6
:1036C0007B68B3F8A430194610460CF0B4FB0346EF
:1036D00018460837BD4680BD80B582B000AF78601F
:1036E0007B6803F180027B68A433194610460CF016
:1036F00073F8034618460837BD4680BD80B584B0D0
:1037000000AF78600023FB737B681B68184605F0E8
:1037100092FB0346002B09D07B6893F91739B3F16C
:10372000FF3F01D1002300E00223FB737B6850338D
:10373000FA7B11461846FEF73EFB03461846103743
:10374000BD4680BD80B584B000AF786000237B7338
:103750000023FB737B68803307F10D021146184686
:103760000BF0F2FF0346FB73FB7B002B14BF01231E
:103770000023DBB2002B46D17B7B002B02D0022B37
:1037800003D03DE00023FB733EE07B681B681846D6
:1037900005F051FB0346002B2FD07B6893F91739B6
:1037A000B3F1FF3F02D00D23FB732DE07B68D3F80C
:1037B000A0301846FEF79DFB034683F00103DBB201
:1037C000002B02D00723FB731EE07B68D3F8A030E8
:1037D0001846FEF7A4FB0346BB7397F90E207B68DF
:1037E00083F817297B6818687B68B3F8A420B97B35
:1037F000084B05F004FC0346FB73FB7B002B03E046
:103800000C23FB7300E000BFFB7B18461037BD465E
:1038100080BD00BF7149000080B584B000AF786002
:103820000023FB737B68803307F1080211461846BA
:103830000CF01FF90346FB73FB7B002B14BF012325
:103840000023DBB2002B09D17B68B833B9680122B1
:10385000184601F0EDFD0346FB7300E000BFFB7B63
:1038600018461037BD4680BD80B584B000AF786083
:103870000023FB737B68803307F10802114618466A
:103880000CF0F7F80346FB73FB7B002B14BF0123FE
:103890000023DBB2002B09D17B68B833B968002262
:1038A000184601F0C5FD0346FB7300E000BFFB7B3B
:1038B00018461037BD4680BD80B582B000AF786035
:1038C0007B6803F150027B68D3F89C3019461046A0
:1038D0000CF024FC034618460837BD4680BD80B571
:1038E00084B000AF78600023FB737B685033042101
:1038F00018460CF013FC0346FB73FB7B002B14BF34
:1039000001230023DBB2002B0FD17B68503303214E
:1039100018460CF003FC0346FB73FB7B002B14BF23
:1039200001230023DBB2002B00E000BFFB7B184625
:103930001037BD4680BD80B582B000AF78607B682F
:103940005033032118460CF0E9FB034618460837AC
:10395000BD4680BD80B582B000AF78607B685033D3
:10396000002118460CF0DAFB034618460837BD461E
:1039700080BD80B584B000AF78600023FB737B68A6
:103980005033052118460CF0C9FB0346FB73FB7B43
:10399000002B14BF01230023DBB2002B50D17B6826
:1039A00050330C2118460CF0B9FB0346FB73FB7B2C
:1039B000002B14BF01230023DBB2002B42D17B6814
:1039C0005033182118460CF0A9FB0346FB73FB7B10
:1039D000002B14BF01230023DBB2002B34D17B6802
:1039E0005033222118460CF099FB0346FB73FB7BF6
:1039F000002B14BF01230023DBB2002B26D17B68F0
:103A0000503340F2012118460CF088FB0346FB734B
:103A1000FB7B002B14BF01230023DBB2002B17D14B
:103A20007B685033402118460CF078FB0346FB734B
:103A3000FB7B002B14BF01230023DBB2002B08E02B
:103A400000BF06E000BF04E000BF02E000BF00E0EE
:103A500000BFFB7B18461037BD4680BD90B583B0D4
:103A600000AF78607B6803F1500405F055F8034619
:103A7000194620460CF09AFB034618460C37BD4603
:103A800090BD80B582B000AF78607B685033012173
:103A90001846FEF790F9034618460837BD4680BD24
:103AA00080B582B000AF78607B6850330021184643
:103AB000FEF781F9034618460837BD4680BD80B53C
:103AC00082B000AF78607B68503304211846FEF75F
:103AD00072F9034618460837BD4680BD80B483B0EE
:103AE00000AF78600C2318460C37BD465DF8047BA8
:103AF000704780B584B000AF78607B681B6807F1C1
:103B000008021146184605F0AFFC7B68503307F1F8
:103B1000080211461846FEF770F90346184610379A
:103B2000BD4680BD80B582B000AF78607B68503301
:103B3000022118460CF020F9034618460837BD4606
:103B400080BD80B582B000AF78607B6803F1500221
:103B50007B6893F8C83019461046FEF72CF90346E7
:103B600018460837BD4680BD80B584B000AF786088
:103B70000B46FB700023FB737B68803307F10E025A
:103B8000114618460BF0E0FD0346FB73FB7B002B50
:103B90004AD1BB7B042B13DC032B07DA012B02DC9D
:103BA000002B03DA0CE0022B05D009E0BA7B7B681E
:103BB00083F8C82009E07B68012283F8C82004E06C
:103BC0007B68032283F8C82000BF7B68002283F84B
:103BD000D020F97801230C227868FFF753F90346C7
:103BE000FB737B6893F8C830042B13D0FB7B002B4E
:103BF00007D17868FEF770FB02467B68C3F8CC20DB
:103C000004E0124B1A687B68C3F8CC207B68012261
:103C100083F89820FB7B002B12D07B68FA7883F81E
:103C2000D0200023FB730BE0FB7B1846FEF794F9D2
:103C30000246FB7819467868FFF7D8F80346FB730D
:103C4000FB7B18461037BD4680BD00BF343F0200E5
:103C500090B583B000AF78607B6803F150047B6857
:103C60001B68184603F064F9034619462046FEF720
:103C7000B4F8034618460C37BD4690BD90B583B0E6
:103C800000AF78607B6803F150047B681B681846BE
:103C900003F0E0FD034619462046FEF79EF8034672
:103CA00018460C37BD4690BD80B584B000AF786033
:103CB0000023FB607B681B68184605F03BFB03464E
:103CC000FB72FB7A002B02D1134BFB6018E0FB7AEE
:103CD0000A2B0AD8FB7A4FF4FA6202FB03F303F5CE
:103CE0005C2303F53463FB600AE0FB7A192B07D8E9
:103CF000FB7A41F2883202FB03F2084B1344FB606B
:103D00007B685033F96818460CF0C9F8034618462A
:103D10001037BD4680BD00BFCC3F0D00B0DB230097
:103D200090B585B000AF78600023FB737B681B689B
:103D300007F10E021146184603F02EFA0346FB73F4
:103D4000FB7B002B0AD17B68503397F90E2011467C
:103D50001846FEF742F80346FB730DE07B6803F15B
:103D60005004FB7B1846FEF7F7F803461946204639
:103D70000CF002F80346FB73FB7B18461437BD4674
:103D800090BD80B584B000AF78600023BB73002382
:103D9000FB737B68803307F10E02114618460BF067
:103DA000F9FC0346FB73FB7B002B14BF01230023AC
:103DB000DBB2002B0AD17B681B6897F90E201146F5
:103DC000184603F00FFA0346FB7300E000BFFB7BCD
:103DD00018461037BD4680BD90B585B000AF7860FD
:103DE0007B681B6807F10E021146184603F096F92E
:103DF0000346FB73FB7B002B0AD17B68503397F99A
:103E00000E2011461846FDF7E8FF0346FB730DE050
:103E10007B6803F15004FB7B1846FEF79DF80346D0
:103E2000194620460BF0A8FF0346FB73FB7B1846A0
:103E30001437BD4690BD80B584B000AF78600023D4
:103E4000BB730023FB737B68803307F10E021146BE
:103E500018460BF09FFC0346FB73FB7B002B14BF43
:103E600001230023DBB2002B0AD17B681B6897F982
:103E70000E201146184603F069F90346FB7300E073
:103E800000BFFB7B18461037BD4680BD90B585B09E
:103E900000AF78600023FB737B681B6807F10E029C
:103EA0001146184603F0D2F90346FB73FB7B002B47
:103EB0000AD17B68503397F90E2011461846FDF75A
:103EC0008CFF0346FB730DE07B6803F15004FB7B22
:103ED0001846FEF741F80346194620460BF04CFF02
:103EE0000346FB73FB7B18461437BD4690BD80B577
:103EF00084B000AF78600023BB730023FB737B6842
:103F0000803307F10E02114618460BF043FC0346BE
:103F1000FB73FB7B002B14BF01230023DBB2002BC0
:103F20000AD17B681B6897F90E201146184603F0EA
:103F3000A9F90346FB7300E000BFFB7B184610376E
:103F4000BD4680BD80B584B000AF78600023FB73B0
:103F50007B68803307F10E02114618460BF0F4FB24
:103F60000346FB73FB7B002B14BF01230023DBB252
:103F7000002B1CD17B68803307F10D0211461846D7
:103F80000BF008FC0346FB73FB7B002B14BF0123E3
:103F90000023DBB2002B0CD17B681B68B97B97F93F
:103FA0000D20184603F03CFD0346FB7302E000BF02
:103FB00000E000BFFB7B18461037BD4680BD90B5C2
:103FC00085B000AF78600023FB737B681B6807F146
:103FD0000C021146184603F085FD0346FB73FB7B7C
:103FE000002B09D17B685033BA89114618460BF073
:103FF00022FF0346FB730DE07B6803F15004FB7B5B
:104000001846FDF7A9FF0346194620460BF0B4FEFB
:104010000346FB73FB7B18461437BD4690BD80B545
:1040200084B000AF78600023FB737B68803307F1B6
:104030000C02114618460BF0CFFB0346FB73FB7BCB
:10404000002B14BF01230023DBB2002B09D17B68B6
:104050001B68BA891146184603F030FD0346FB730E
:1040600000E000BFFB7B18461037BD4680BD80B422
:1040700083B000AF7860FEE780B483B000AF7860B3
:10408000FEE790B583B000AF78607B6803F1500421
:1040900005F016FA03461846FEF7F2FA03461946EB
:1040A0002046FDF788FE034618460C37BD4690BDF6
:1040B000B0B586B000AF78604FF000024FF000035B
:1040C000C7E902230023FB7502F02AF938617B68F7
:1040D000803307F10802114618460BF0F3FB034644
:1040E000FB75FB7D002B14BF01230023DBB2002BEB
:1040F0001BD13B691A464FF00003D7E902019942F0
:1041000008BF904202D20723FB750FE0D7E90201F6
:104110003B691A464FF00003841A61EB03057B6884
:1041200003F51363C3E9004500E000BFFB7D1846BB
:104130001837BD46B0BD80B582B000AF78607B68EF
:1041400003F150017B6803F51363D3E900230846AC
:104150000BF001FF034618460837BD4680BD80B509
:1041600082B000AF78607B681B68184608F006FED6
:10417000034619467868FFF7F8F9034618460837EA
:10418000BD4680BD80B582B000AF78607B681B689B
:10419000184608F001FE034619467868FFF7E5F96E
:1041A000034618460837BD4680BD80B586B000AFCF
:1041B000F860B9607A600D23FB75FEF767F8386127
:1041C0003B69002B07D07B68BA68F9683869FEF74D
:1041D000DBF90346FB75FB7D18461837BD4680BDED
:1041E00080B582B000AF7860396078683B6829227A
:1041F000034900F03DF800BF78680837BD4680BD30
:104200000435020080B582B000AF7860396078680C
:104210003B681622034900F02BF800BF7868083786
:10422000BD4680BDF036020080B582B000AF786038
:10423000396078683B680322034900F019F800BF31
:1042400078680837BD4680BDF837020080B582B077
:1042500000AF7860396078683B680322034900F05A
:1042600007F800BF78680837BD4680BD1C380200DB
:1042700080B489B000AFF860B9607A603B60002319
:10428000FB617B68002B00D1FEE77B68013BBB61D3
:10429000FA69BB699A4217D2FA69BB6913445B0891
:1042A0007B617A6913465B0013449B001A46BB6826
:1042B00013441B683A689A4203D97B690133FB6156
:1042C000E6E77B69BB61E3E7FA6913465B001344E9
:1042D0009B001A46BB6813441B683A689A420ED189
:1042E000FA6913465B0013449B001A46BB681344EB
:1042F000FA68043393E8030082E8030005E0FB68F2
:1043000000221A60FB6800225A60F8682437BD4614
:104310005DF8047B704780B483B000AF0346FB7147
:1043200000BF0C37BD465DF8047B704780B582B096
:1043300000AF7860786800F021F803461B7803F03E
:104340000803002B14BF01230023DBB218460837F3
:10435000BD4680BD80B582B000AF7860786800F05F
:104360000DF803461B7803F01003002B14BF012344
:104370000023DBB218460837BD4680BD80B483B049
:1043800000AF78607B681B6818460C37BD465DF847
:10439000047B704780B483B000AF78607B689B7EFD
:1043A000C3F30003DBB218460C37BD465DF8047B4F
:1043B000704780B582B000AF78607B6850330621CB
:1043C00018460BF0ABFE034618460837BD4680BDC5
:1043D00080B586B000AFF860B9601346FB71012369
:1043E000FB750023BB82BB68002B15D0FB79002B2B
:1043F00012D1FB6803F15000BB681968BB689B8849
:104400001A460BF0A5FE0346002B14BF0123002320
:10441000DBB2002B0FD054E1FB685033002118466B
:104420000BF009FD0346002B14BF01230023DBB270
:10443000002B40F02781FB6803F15002BB68002B82
:1044400003D0BB6893F9153000E0002319461046ED
:10445000FDF7C3FC0346002B14BF01230023DBB28E
:10446000002B40F01181FB6850336FF07F0118463C
:10447000FDF7B3FC0346002B14BF01230023DBB27E
:10448000002B40F00381BB68002B15D0BB68DB7D9F
:10449000C3F30003DBB2002B03D0BB8A43F010034D
:1044A000BB82BB68DB7DC3F34003DBB2002B03D0D0
:1044B000BB8A43F02003BB82FB685033BA8A1146A3
:1044C00018460BF0B8FC0346002B14BF0123002351
:1044D000DBB2002B40F0DC80FB68503318460BF059
:1044E0009DFE0346002B14BF01230023DBB2002BEB
:1044F00040F0D080FB6803F15002BB68002B02D073
:10450000BB689B7900E0002319461046FDF753FC79
:104510000346002B14BF01230023DBB2002B40F025
:10452000BB80FB6803F15002BB68002B02D0BB6864
:104530009B7D00E0002319461046FDF73CFC034636
:10454000002B14BF01230023DBB2002B40F0A68018
:10455000FB6803F15001BB68002B03D0BB68D3E9B3
:10456000022303E04FF000024FF0000308460BF077
:10457000F2FC0346002B14BF01230023DBB2002B07
:1045800040F08E80FB68503318460BF09EFE0346C9
:10459000002B14BF01230023DBB2002B40F08280EC
:1045A000FB68503318460BF039FE0346002B14BF4E
:1045B00001230023DBB2002B76D1FB685033FA795C
:1045C000114618460BF0AAFD0346002B14BF012329
:1045D0000023DBB2002B69D1FB68503318460BF087
:1045E00074FE0346002B14BF01230023DBB2002B13
:1045F0005ED1FB68503318460BF010FE0346002BCB
:1046000014BF01230023DBB2002B53D1FB6803F15D
:104610005002BB68002B02D0BB681B7D00E000236A
:1046200019461046FDF7C7FB0346002B14BF0123B4
:104630000023DBB2002B3FD1FB6803F15002BB68C3
:10464000002B02D0BB681B6900E00023194610460E
:104650000BF025FC0346002B14BF01230023DBB223
:10466000002B2BD1FB68503318460BF02EFE03466F
:10467000002B14BF01230023DBB2002B20D1002329
:10468000FB751EE000BF1CE000BF1AE000BF18E091
:1046900000BF16E000BF14E000BF12E000BF10E052
:1046A00000BF0EE000BF0CE000BF0AE000BF08E062
:1046B00000BF06E000BF04E000BF02E000BF00E072
:1046C00000BFFB7D18461837BD4680BD80B584B05D
:1046D00000AFF860B9601346FB71054B1B68FA79AF
:1046E000B968184600F006F800BF1037BD4680BD17
:1046F0008014002080B586B000AFF860B960134622
:10470000FB718023FB75FB6803F15000F97D712379
:1047100006220BF0F4FA0346002B14BF01230023FA
:10472000DBB2002B1AD1FB791A46B968F868FFF79B
:104730004FFE0346002B14BF01230023DBB2002BE6
:104740000ED1FB68503318460BF04EFB0346002B8E
:1047500014BF01230023DBB2002B02E000BF00E006
:1047600000BF00BF1837BD4680BD000080B584B0D3
:1047700000AFF860B9607A60FB70054B1868FB7891
:104780007A68B96800F006F800BF1037BD4680BDF2
:104790008014002090B587B000AFF860B9607A60EF
:1047A000FB70FB6893F81639002B00F0D080FB6893
:1047B00093F8163963F07F03FB757B68002B08D0F4
:1047C0007B681846FFF7C6FD0346002B01D0012386
:1047D00000E00023BB75B868FFF7DCFD03467B757E
:1047E000FB68002283F81629FB6803F15000F97D6D
:1047F000002306220BF083FA0346002B14BF01238B
:104800000023DBB2002B40F0A480FB6803F15004CE
:10481000FB781846FDF7A0FB0346194620460BF02F
:104820007DFC0346002B14BF01230023DBB2002BC9
:1048300040F09180FB685033BA7D11461846FDF771
:10484000A3FA0346002B14BF01230023DBB2002B85
:1048500040F08380FB6850337A7D11461846FDF79F
:1048600093FA0346002B14BF01230023DBB2002B75
:1048700075D1FB78002B0DD1FB781A467968F86862
:10488000FFF7A6FD0346002B14BF01230023DBB274
:10489000002B66D1BB681846FFF748FD0346002B86
:1048A00004D07B7D002B01D0012300E00023002BEE
:1048B00040D0BB6807F114021146184606F0C6FA4C
:1048C0000346002B14BF01230023DBB2002B4AD187
:1048D000BB6807F110021146184606F01EFA03469F
:1048E000002B14BF01230023DBB2002B1ED1FB6879
:1048F00050333A7D11461846FDF75DFA0346002B0A
:1049000014BF01230023DBB2002B11D1FB6850330D
:104910003A69114618460BF0C2FA0346002B14BF41
:1049200001230023DBB2002B04D002E000BF1CE017
:1049300000BF1AE0FB68503318460BF055FA0346E7
:10494000002B14BF01230023DBB2002B0DE000BFBE
:104950000AE000BF08E000BF06E000BF04E000BFBF
:1049600002E000BF00E000BF00BF1C37BD4690BDA5
:1049700080B582B000AF78600B46FB70054B1B68BA
:1049800097F903201146184600F006F800BF0837D3
:10499000BD4680BD8014002080B584B000AF786033
:1049A0000B46FB707B6893F81739FB737B68FF221B
:1049B00083F817297B681B68184604F0CEFA034673
:1049C0001846FFF7A8FC7B6803F150003923062244
:1049D00080210BF094F90346002B14BF0123002320
:1049E000DBB2002B56D17B685033FA7B1146184658
:1049F000FDF7E1F90346002B14BF01230023DBB2CE
:104A0000002B49D17B68503397F903201146184693
:104A1000FDF7E3F90346002B14BF01230023DBB2AB
:104A2000002B3BD17B68503318460BF0DDF9034671
:104A3000002B14BF01230023DBB2002B30D17B6895
:104A400003F150003023062280210BF058F9034671
:104A5000002B14BF01230023DBB2002B22D17B6883
:104A6000503300211846FDF7A6F90346002B14BF6A
:104A700001230023DBB2002B16D17B68503318468C
:104A80000BF0B2F90346002B14BF01230023DBB265
:104A9000002B0AE000BF08E000BF06E000BF04E012
:104AA00000BF02E000BF00E000BF00BF1037BD46FE
:104AB00080BD90B583B000AF78607B6803F150048F
:104AC0007B681B68184604F086FA034619462046A0
:104AD0000BF024FB034618460C37BD4690BD80B54D
:104AE00082B000AF78607B6803F150027B6893F876
:104AF000183919461046FDF747F903461846083796
:104B0000BD4680BD90B585B000AF78600023FB73D3
:104B10007B6803F150047B681B68184604F0FDFBBA
:104B200002460B4620460BF016FA0346FB73FB7B4E
:104B3000002B14BF01230023DBB2002B00BFFB7B43
:104B400018461437BD4690BD80B584B000AF78607C
:104B50000023FB737B6803F180027B6803F6181364
:104B6000194610460AF0C2FD0346FB73FB7B002B7F
:104B700014BF01230023DBB2002B0BD17B681A6822
:104B80007B6893F818391946104604F052FA034628
:104B9000FB7300E000BFFB7B18461037BD4680BDAD
:104BA00080B584B000AF78600023FB737B681B681E
:104BB000184604F026FB0346FB73FB7B002B14BF57
:104BC00001230023DBB2002B30D17B6880331846F1
:104BD000FDF791F80346012B8CBF01230023DBB2C4
:104BE000002B25D07B68803307F10C021146184654
:104BF0000AF0F2FD0346FB73FB7B002B14BF01237D
:104C00000023DBB2002B15D17B681B68BA891146E3
:104C1000184604F038FA0346FB73FB7B002B14BFE5
:104C200001230023DBB2002B06D1CEE700BF04E056
:104C300000BF02E000BF00E000BFFB7B184610375A
:104C4000BD4680BD80B584B000AF78600023FB73A3
:104C50007B681B68184604F0FAFA0346FB73FB7B7B
:104C6000002B14BF01230023DBB2002B30D17B6863
:104C700080331846FDF73FF80346072B8CBF01230E
:104C80000023DBB2002B25D07B68803307F10802BC
:104C900011461846FDF720F80346FB73FB7B002BFB
:104CA00014BF01230023DBB2002B15D17B681B68E6
:104CB000BA681146184604F012FA0346FB73FB7BF0
:104CC000002B14BF01230023DBB2002B06D1CEE75B
:104CD00000BF04E000BF02E000BF00E000BFFB7BBC
:104CE00018461037BD4680BD80B584B000AF7860EF
:104CF0000023FB737B68803307F10C0211461846D2
:104D00000AF06AFD0346FB73FB7B002B14BF0123F3
:104D10000023DBB2002B09D17B681B68BA891146DE
:104D2000184604F00FFA0346FB7300E000BFFB7B5C
:104D300018461037BD4680BD80B584B000AF78609E
:104D40000023FB737B68803307F108021146184685
:104D5000FCF7C2FF0346FB73FB7B002B14BF012350
:104D60000023DBB2002B09D17B681B68BA681146AF
:104D7000184604F013FA0346FB7300E000BFFB7B08
:104D800018461037BD4680BD80B584B000AF78604E
:104D90000023FB737B68803307F10C021146184631
:104DA0000AF01AFD0346FB73FB7B002B14BF0123A3
:104DB0000023DBB2002B09D17B681B68BA8911463E
:104DC000184604F060F90346FB7300E000BFFB7B6C
:104DD00018461037BD4680BD80B584B000AF7860FE
:104DE0000023FB730023BB607B68803307F108025C
:104DF00011461846FCF770FF0346FB73FB7B002B44
:104E000014BF01230023DBB2002B09D17B681B6890
:104E1000BA681146184604F062F90346FB7300E0D5
:104E200000BFFB7B18461037BD4680BD80B584B0FF
:104E300000AF78600023BB730023FB737B68803373
:104E400007F10E02114618460AF050FC0346FB73A8
:104E5000FB7B002B14BF01230023DBB2002B17D1F7
:104E6000BB7B83F00103DBB2002B08D07B681B689F
:104E70000021184603F0C9FF0346FB7309E07B6875
:104E80001B680649184603F0C0FF0346FB7300E0A9
:104E900000BFFB7B18461037BD4680BDCD460000E5
:104EA00080B584B000AF78600023FB737B688033EB
:104EB00007F10C02114618460AF08EFC0346FB73FC
:104EC000FB7B002B14BF01230023DBB2002B09D195
:104ED0007B681B68BA891146184603F0C0FF034679
:104EE000FB7300E000BFFB7B18461037BD4680BD5A
:104EF00080B586B000AF786039607B68803307F199
:104F00000E0207F1100118460AF026FE0346FB7553
:104F1000FB7D002B14BF01230023DBB2002B40F0EC
:104F2000E680FB897F2B02D90623FB75F2E0FB8923
:104F3000DBB29AB23B689A803B68186839693B6873
:104F40009B881A461DF054F87B6803F180023B6889
:104F50000633194610460AF0F7FB0346FB75FB7D46
:104F6000002B14BF01230023DBB2002B40F0C180D3
:104F70003B6804221A763B680F225A763A68937E81
:104F800043F0040393763A68937E6FF300039376BD
:104F90003A68937E6FF3410393763A68937E6FF39A
:104FA000041393763B6800221A613B6800225A6121
:104FB0007B6803F180023B681833194610460AF0FB
:104FC000C3FB0346002B14BF01230023DBB2002BDD
:104FD00040F091807B6803F180023B6819331946E9
:104FE00010460AF0B1FB0346002B14BF0123002337
:104FF000DBB2002B40F081807B68803307F10D022B
:10500000114618460AF072FB0346002B14BF012319
:105010000023DBB2002B72D17B68803307F10B02D7
:10502000114618460AF062FB0346002B14BF012309
:105030000023DBB2002B64D17B68803307F10C02C4
:10504000114618460AF052FB0346002B14BF0123F9
:105050000023DBB2002B56D17B68803307F10A02B4
:10506000114618460AF042FB0346002B14BF0123E9
:105070000023DBB2002B48D17B6803F180023B6840
:105080001033194610460AF0DAFB0346002B14BF12
:1050900001230023DBB2002B39D17B6803F18002AE
:1050A0003B681433194610460AF0C9FB0346002B2F
:1050B00014BF01230023DBB2002B2AD1797B3A688D
:1050C000937E61F382039376F97A3A68937E61F373
:1050D00000039376397B3A68937E61F341039376BC
:1050E000B97A3A68937E61F30413937612E000BFB5
:1050F00010E000BF0EE000BF0CE000BF0AE000BF00
:1051000008E000BF06E000BF04E000BF02E000BF0F
:1051100000E000BFFB7D18461837BD4680BD00008B
:1051200080B584B000AF78600B46FB700023FB7342
:105130007B681B68184603F07EFE034683F001037C
:10514000DBB2002B02D00D23FB732AE07B681B68C7
:10515000184603F016FFB860BB68002B02D103238A
:10516000FB731EE0B9687868FFF7C2FE0346FB7365
:10517000FB7B002B14BF01230023DBB2002B0FD1DC
:10518000FB7803F00F03DAB27B6883F816297B689B
:105190001B680E49184603F008FF0346FB7300E046
:1051A00000BFFB7B002B0BD0FB7B1846FCF7D4FE2B
:1051B0000246FB7819467868FDF718FE0346FB7334
:1051C000FB7B18461037BD4680BD00BF6D47000011
:1051D000B0B58AB002AF78600023FB777B6880337C
:1051E00007F11E02114618460AF0AEFA0346FB7795
:1051F000FB7F002B14BF01230023DBB2002B72D1F5
:10520000BB7F082B02D00723FB7775E07B688033D8
:1052100007F11D02114618460AF096FA0346FB777D
:10522000FB7F002B14BF01230023DBB2002B5CD1DA
:105230007B68803307F11A0207F1140118460AF05F
:105240008BFC0346FB77FB7F002B14BF012300235D
:10525000DBB2002B4BD17B8B102B02D00723FB77CB
:105260004AE07B68803307F11A0207F11001184603
:105270000AF072FC0346FB77FB7F002B14BF01236F
:105280000023DBB2002B34D17B8B102B02D0072301
:10529000FB7731E07B68803307F11A0207F10C01DC
:1052A00018460AF059FC0346FB77FB7F002B14BF1E
:1052B00001230023DBB2002B1DD17B8B102B02D0EE
:1052C0000723FB7718E07B681868B97F7C7F7D69CE
:1052D0003B69FA68019200932B46224603F0DDFFFA
:1052E0000346FB7708E000BF06E000BF04E000BF14
:1052F00002E000BF00E000BFFB7F18462037BD463C
:10530000B0BD80B584B000AF78600023FB737B68CC
:10531000803307F10802114618460AF090FA034656
:10532000FB73FB7B002B14BF01230023DBB2002B9C
:1053300009D17B681B68BA681146184603F0D7FF8D
:105340000346FB7300E000BFFB7B18461037BD46E9
:1053500080BD2DE9F00F82B000AF7860F9707968F8
:10536000D1E900ABFC784FF001004FF00001A4F14F
:105370002006C4F1200501FA04F300FA06F63343CF
:1053800020FA05F52B4300FA04F24AEA02084BEA38
:1053900003097B68C3E9008900BF0837BD46BDE843
:1053A000F00F704780B483B000AF78601B231846BD
:1053B0000C37BD465DF8047B704780B586B000AF02
:1053C000F860B9607A6007F112031946F868FCF7D3
:1053D000C5FB78610023FB74BB7CFA7C9A4223D224
:1053E0007B691B68BA689A4216D17B695B687A68E8
:1053F0009A4211D1FB7C1946F868FCF7E5FB03469D
:1054000083F00103DBB2002B0DD0FB68FA7C114660
:105410001846FFF79EFF06E0FB7C0133FB747B69B7
:105420000C337B61D8E700BF00BF1837BD4680BD95
:1054300080B586B000AFF860B9601346FB710023F9
:10544000FB7407F111031946F868FCF787FB7861D4
:105450000023BB747B7CBA7C9A422DD27B691B7A79
:10546000002B21D07B691B68BA689A421CD1FB795A
:10547000002B0DD0FB680833BA7C11461846FFF7A5
:1054800068FFFB68BA7C11461846FCF7AFFB06E0E4
:10549000FB680833BA7C11461846FCF7A7FB0123CA
:1054A000FB74BB68002B06D1BB7C0133BB747B69EA
:1054B0000C337B61CEE700BFFB7C002B01D00023C7
:1054C00000E0072318461837BD4680BD80B586B07A
:1054D00000AF786039600023FB7507F10E031946B1
:1054E0007868FCF73BFB38610023FB73BB7BFA7BDE
:1054F0009A4217D23B691B7A002B0CD03B691B6880
:105500003A689A4207D1FB7B19467868FCF75CFB46
:105510000346FB7506E0FB7B0133FB733B690C33F1
:105520003B61E3E7FB7D18461837BD4680BD0000B0
:1055300080B483B000AF0346FB71FB7903F01F0218
:10554000074997F907305B09012000FA02F241F898
:10555000232000BF0C37BD465DF8047B704700BFB9
:1055600000E100E080B483B000AF0346FB71FB793B
:1055700003F01F02074997F907305B09012000FA81
:1055800002F2203341F8232000BF0C37BD465DF8FE
:10559000047B704700E100E080B483B000AF0346B5
:1055A000FB71FB7903F01F02074997F907305B098C
:1055B000012000FA02F2603341F8232000BF0C37CB
:1055C000BD465DF8047B704700E100E080B483B025
:1055D00000AF03463960FB7197F90730002B0BDAF7
:1055E0003B68DAB20C49FB7903F00F03043B52012C
:1055F000D2B20B441A7609E03B68DAB2074997F950
:1056000007305201D2B20B4483F8002300BF0C379D
:10561000BD465DF8047B704700ED00E000E100E06E
:105620002DE9B04F8EB000AFC7E90601D7E90601FA
:105630004FF000024FF00003420B42EAC1424B0B15
:10564000544901FB03F0002101FB02F144185149C8
:10565000A2FB0101631819464FF000024FF000034E
:10566000020F42EA01120B0FC7E90C23D7E90C0124
:105670004FF000024FF000034B0243EAD0534202C6
:10568000C7E90A23D7E90C8944464D464FF000028A
:105690004FF000036B0143EAD463620114461D46D8
:1056A000B4EB080465EB09054FF000004FF0000172
:1056B000A90141EA9461A001001B61EB05014FF0D3
:1056C00000024FF00003CB0043EA5073C2001046C3
:1056D000194610EB080A41EB090BD7E90623B2EB98
:1056E0000A01396163EB0B037B61D7E90434C7E935
:1056F0000C34D7E90C2328484FF00001994208BF29
:10570000904205D2254B264A902126481CF0FAFBF0
:105710007B6B254A02FB03F23B6B40F2314101FBFC
:1057200003F3D1183B6B204AA3FB022319440B4619
:10573000C7E90823C7E90823D7E908234FF0FF305A
:1057400047F6FF711418BC604B41FB60D7E9023487
:10575000C7E90834D7E908014FF000024FF0000311
:10576000CA0B0023C7E90823D7E90A01D7E90823B0
:1057700084183C6041EB03037B60D7E90034C7E940
:105780000A34D7E90A23104619463837BD46BDE822
:10579000B08F00BFD07B6308452C1600843902000F
:1057A000743A0200943902007B2DE8BD80B485B0C4
:1057B00000AFF860B9607A60FB68BA6802F5A87259
:1057C000796843F8221000BF1437BD465DF8047BAA
:1057D000704780B483B000AF786039607B683A6806
:1057E000C3F8042300BF0C37BD465DF8047B704747
:1057F00080B483B000AF786039607B683A68C3F8E2
:10580000082300BF0C37BD465DF8047B704780B4A9
:1058100083B000AF786039607B68D3F804233B68BD
:10582000134018460C37BD465DF8047B704780B4C2
:1058300083B000AF78600B467B807B887A68134426
:105840001B6818460C37BD465DF8047B704780B472
:1058500085B000AF78600B467B807B887A68134404
:1058600000221A607B887A6813441B68FB60FB681F
:1058700000BF1437BD465DF8047B704780B483B029
:1058800000AF78607B68D3F8043518460C37BD4606
:105890005DF8047B704780B483B000AF78603960F6
:1058A0007B683A68C3F8082500BF0C37BD465DF831
:1058B000047B704780B483B000AF78600B467B8078
:1058C0007A887B68134418460C37BD465DF8047B24
:1058D000704780B483B000AF78600B46FB70FA78F5
:1058E0007B6813441A460123136000BF0C37BD4682
:1058F0005DF8047B704780B483B000AF7860396096
:105900007B683A68C3F8442300BF0C37BD465DF896
:10591000047B704780B483B000AF786039607B68E7
:105920003A68C3F8482300BF0C37BD465DF8047BD6
:105930007047000080B586B000AF154B7B617B6976
:10594000D3E84F3F3B613B69DBB2FB70FB78DBB2D6
:10595000002B04D0BFF32F8F00BF002313E00123DF
:10596000FB730B4BBB60FA7BB968C1E8432F7B60CC
:105970007B68002BE1D102210648FFF739FFBFF316
:105980005F8F00BF012318461837BD4680BD00BF9A
:10599000881400200040024080B500AF0221054875
:1059A000FFF717FFBFF35F8F00BF034B00221A7092
:1059B00000BF80BD0040024088140020B0B584B014
:1059C00000AFC7E902011346FB71FB79002B29D117
:1059D000D7E9020102460B464FF000044FF00005E4
:1059E0005D0145EAD265540122462B46121A63EB4B
:1059F00001034FF000044FF000059D0045EA927549
:105A0000940022462B46121841EB03034FF000008E
:105A10004FF00001D90041EA5271D00002460B4616
:105A2000C7E90223D7E90201FFF7FAFD02460B4658
:105A3000104619461037BD46B0BD2DE9B04F86B0AF
:105A400000AFC7E902011346FB71D7E902452046C2
:105A500029464FF000024FF000034B0143EAD063A8
:105A6000420110461946001B61EB05014FF0000290
:105A70004FF000038B0143EA90638201121A63EB3B
:105A800001034FF000004FF00001D90041EA5271CC
:105A9000D00002460B4612EB040A43EB050B40F222
:105AA000FF124FF000031AEB02084BEB03094FF013
:105AB00000024FF000034FEA582242EAC9524FEA6F
:105AC0005923C7E90423FB79002B0BD1D7E9040143
:105AD0004FF47A724FF000031CF098F802460B4620
:105AE000C7E90423D7E90423104619461837BD46F1
:105AF000BDE8B08F80B485B000AFC7E9020113469E
:105B0000FB71FB790A4A1B0113440833D3E90023D4
:105B1000D7E90201994208BF90422CBF012300231C
:105B2000DBB218461437BD465DF8047B704700BFF2
:105B3000A014002080B582B000AFFFF7FBFE034643
:105B4000002B34D00023FB704FF482712648FFF7FE
:105B50006EFE0346002B0ED0244B1B680133234AF4
:105B600013600123FB70BFF35F8F00BF4FF482719E
:105B70001D48FFF76CFE1D4B1B6801335B087B6003
:105B8000FFF70AFFFB78002B29D0184B1B6803F0A6
:105B90000103002B05D1164B164AEA2116481CF0CA
:105BA000B1F9124B1B680133104A136017E04FF430
:105BB00082710D48FFF73BFE0346002B05D10B4BCE
:105BC0001B6803F00103002B05D0084B1B68023350
:105BD0005B087B6003E0054B1B685B087B607B68B0
:105BE00018460837BD4680BD00400240841400209E
:105BF000D83902004C3A0200F039020080B500AFFB
:105C00000248FFF73BFE0346184680BD00400240B5
:105C100080B586B000AF78603960FFF78BFF7861A0
:105C2000BFF35F8F00BFFFF7E9FF3861BFF35F8FFE
:105C300000BFFFF77FFFF8607B68FA681A607A6937
:105C4000FB689A4203D0FFF7D9FF034600E03B69A7
:105C50003A68136000BF1837BD4680BD2DE9B043D8
:105C600086B000AFF860B9601346FB71FB681C4654
:105C70004FF00005204629464FF000024FF0000388
:105C80004B0143EAD063420110461946001B61EB09
:105C900005014FF000024FF000038B0143EA9063CF
:105CA0008201121A63EB01034FF000004FF0000174
:105CB000D90041EA5271D00002460B46121945EB59
:105CC00003034FF000004FF00001D90341EA5241B5
:105CD000D00302460B4614461D46BB6818464FF0DB
:105CE00000010122FFF7A9FE02460B4614EB020851
:105CF00045EB0309C7E90489FB79002B0BD1D7E9F0
:105D000004014FF47A724FF000031BF07FFF02464C
:105D10000B46C7E90423D7E9042310461946183770
:105D2000BD46BDE8B08380B584B000AF0346FB71CB
:105D300007F1080207F10C0311461846FFF768FF48
:105D4000FB68B968FA791846FFF788FF02460B46E8
:105D5000104619461037BD4680BD000080B584B09E
:105D600000AF03460A46FB711346BB71FB792C4A10
:105D70001B01134408331B8819462A48FFF767FDA7
:105D8000FB791846FFF7CFFFC7E90201BB79002B6B
:105D900008D1FB791A46D7E90201FFF7ABFE0346AB
:105DA000002B38D0FB791E4A1B01134404331B68B7
:105DB00019461C48FFF7AEFDFB79194A1B01134435
:105DC0000C331B6819461748FFF712FDFB79032BAC
:105DD0000BD0032B18DC012B02DC002B08DA13E0BC
:105DE000022B11D10CF0ECFD16E00BF021FA13E0C0
:105DF000FB790D4A1B01134401221A700B4B01223F
:105E00001A7001F00DFF07E0094B0A4A4FF4A77121
:105E100009481CF077F800BF00BF1037BD4680BDB1
:105E20000C3A020000400240A01400209814002008
:105E3000043A0200603A0200F03902002DE9B00F86
:105E40008BB000AFF861B9617A617B69D3E9002357
:105E5000C7E908233B6AFA699A4210D93B6AFA6992
:105E6000D31A002B0BDAD7E90823111C396043F150
:105E7000FF337B60D7E90023C7E9082310E03B6AC2
:105E8000FA699A420CD23A6AFB69D31A002B07DAF4
:105E9000D7E9082312F1000A43F1010BC7E908AB67
:105EA000D7E908234FF000004FF0FF3102EA000865
:105EB00003EA0109FB691A464FF0000318EB0204DC
:105EC00049EB0305BB691A464FF00003A118B960FE
:105ED00045EB0303FB60D7E90223104619462C3734
:105EE000BD46BDE8B00F704780B588B000AFC7E9C8
:105EF00002011346FB71FB791A46D7E90201FFF74D
:105F00005DFDC7E90601FB791A46D7E90601FFF7EF
:105F100094FDC7E90401D7E9042310461946203748
:105F2000BD4680BDB0B588B000AFF860B9603B60D9
:105F30001346FB71FB79244A1B0113440C331B6885
:105F400019462248FFF754FCFB791F4A1B011344F2
:105F500004331B6819461D48FFF7CDFC3A68B96841
:105F6000F868FFF76BFFC7E90601FB791A46D7E926
:105F70000601FFF723FD02460B466FF07F404FF00E
:105F8000000102EA000403EA0105C7E90445FC79BF
:105F9000FB791A46D7E90601FFF7A6FF02460B4632
:105FA0000B48210101440831C1E90023FB79064A6D
:105FB0001B0113441B683A6919460448FFF7F6FBB6
:105FC00000BF2037BD46B0BD0C3A02000040024081
:105FD000A014002080B58AB000AFF860B960134605
:105FE000FB7107F1180207F11C0311461846FFF771
:105FF0000FFEFB69B969FA791846FFF72FFE0246D2
:106000000B46C7E9042307F11003FA79B968F86869
:10601000FFF788FFFFF7F2FD0246BB699A4207D0FF
:1060200007F1180207F11C0311461846FFF7F0FDAF
:10603000F869BB690233FA791946FFF70FFEC7E921
:106040000801FB791A46D7E90801FFF753FD03461B
:10605000002B06D0FB7901211846FFF77FFE40BFD9
:106060000AE0FB79064A1B0113440C331B681946EE
:106070000448FFF7AEFB00BF00BF2837BD4680BD18
:106080000C3A02000040024080B584B000AFF860D6
:10609000B9607A607B680322B968F868FFF742FF4D
:1060A0004FF4002319460348FFF793FB00BF103756
:1060B000BD4680BD0040024080B582B000AF0346BF
:1060C000FB71FB79134A1B01134404331B68194607
:1060D0001148FFF71FFCFB790E4A1B0113440C33D8
:1060E0001B6819460C48FFF783FBFB79094A1B0123
:1060F000134408331B8819460748FFF7A8FBFB79B0
:10610000064A1B01134400221A7000BF0837BD461F
:1061100080BD00BF0C3A020000400240A0140020E5
:1061200080B582B000AF4022002133481BF088FFC9
:10613000324B00221A60324B00221A7031494FF064
:1061400000024FF00003C1E90023002013F0EAF938
:1061500000BF13F03BFA034683F00103DBB2002BD0
:10616000F7D106212420FFF731FA2420FFF714FA93
:106170002420FFF7DDF900212348FFF78CFB4FF4C3
:1061800082712148FFF763FB02211F48FFF7B3FB31
:1061900002211D48FFF71DFB00237B6020E01B4A06
:1061A0007B681B01134408331B8819461648FFF708
:1061B0004EFB164A7B681B01134404331B681946C7
:1061C0001148FFF7A7FB114A7B681B0113440C33EE
:1061D0001B6819460C48FFF70BFB7B6801337B609B
:1061E0007B68032BDBD900210748FFF772FB00BF58
:1061F0000837BD4680BD00BFA014002084140020D5
:106200008814002090140020004002400C3A020044
:1062100080B582B000AF04212448FFF75AFB002369
:106220007B6020E0224A7B681B01134408331B88F3
:1062300019461E48FFF70BFB1D4A7B681B011344E0
:1062400004331B6819461948FFF764FB184A7B683A
:106250001B0113440C331B6819461448FFF7C8FA96
:106260007B6801337B607B68032BDBD902210F48FD
:10627000FFF7BEFA02210D48FFF74CFB4FF4827185
:106280000A48FFF7E4FA00F028F92420FFF76AF93A
:106290002420FFF781F900212420FFF797F913F05C
:1062A0007DF900BF0837BD4680BD00BF00400240F9
:1062B0000C3A020080B582B000AF7860114B00222A
:1062C0001A70114B1B78DBB2002B05D00E4B00224D
:1062D0001A70786803F065FE0B4B1B7CDBB2002B59
:1062E00005D0094B00221A74786803F0C6FE054BEE
:1062F0001B78DBB2002BE1D100BF00BF0837BD46E1
:1063000080BD00BF98140020A014002080B500AF0D
:106310000120FFF708FD02460B461046194680BDD6
:1063200080B500AFFFF7F2FF4FF47A724FF0000331
:106330001BF06CFC02460B461346184680BD80B528
:1063400084B000AFF860B9607A6000227968B868FC
:10635000FFF740FE00BF1037BD4680BD80B582B05C
:1063600000AF78600020FFF7A7FE00BF0837BD46EA
:1063700080BD80B500AFFFF7C9FF02460B4613464C
:10638000184680BD80B584B000AFF860B9607A600F
:1063900001227968B868FFF71DFE00BF1037BD46BF
:1063A00080BD80B582B000AF78600120FFF784FE29
:1063B00000BF0837BD4680BD80B400AF00BFBD46FA
:1063C0005DF8047B704780B400AF00BFBD465DF848
:1063D000047B704780B500AF4FF480231946054811
:1063E000FFF706FABFF34F8F00BFBFF36F8F00BFF9
:1063F00000BF80BD0040024080B500AF4FF4802355
:1064000019460248FFF7E5F900BF80BD0040024091
:1064100080B500AFFFF77AFF02460B4613461846D9
:1064200080BD80B400AF1F231846BD465DF8047BD5
:10643000704780B582B000AF786039600222396859
:106440007868FFF7C7FD00BF0837BD4680BD80B53F
:1064500000AF0220FFF730FE00BF80BD80B584B0E2
:1064600000AF07F10C0207F1080311461846FFF7C9
:10647000CFFBBB68F96803221846FFF7EFFB024623
:106480000B46C7E90023D7E9002310463B461A46CE
:106490003E21FFF7F9FDFFF7B1FB0246FB689A4288
:1064A000DFD100BF00BF1037BD4680BD80B584B0CE
:1064B00000AF786039600320FFF735FC02460B46D9
:1064C000C7E9022307F108031A4639687868FFF71D
:1064D000DBFD00BF1037BD4680BD80B500AF032097
:1064E000FFF7EAFD00BF80BD80B500AF4FF4A67393
:1064F00019460348FFF7DEF90346184680BD00BF82
:106500000040024080B400AF044BD3E90E23134691
:106510001846BD465DF8047B704700BFA0140020FC
:1065200080B582B000AF4FF482711D48FFF77FF94C
:106530000346002B05D002211948FFF759F9FFF750
:10654000F9FA00237B6022E0164A7B681B011344A2
:106550000C331B6819461248FFF759F90346002B04
:1065600012D0104A7B681B01134408331B8819465C
:106570000B48FFF75CF90346002B05D07B68DBB2C4
:1065800000211846FFF7EAFB7B6801337B607B68DC
:10659000032BD9D900BF00BF0837BD4680BD00BF5F
:1065A000004002400C3A020080B500AFFFF7AEFE9B
:1065B00002460B461046194680BD000080B400AF6D
:1065C000BFF34F8F00BF074BDB6803F4E062054960
:1065D000054B1343CB60BFF34F8F00BF00BF00BF1D
:1065E000FCE700BF00ED00E00400FA0580B400AF56
:1065F00000BFBD465DF8047B704780B400AF00BFAC
:10660000BD465DF8047B704780B400AF4FF0804317
:10661000D3F80034064A13604FF080434FF0FF3246
:10662000C3F8002400BFBD465DF8047B704700BF7F
:10663000E014002080B400AF00BFBD465DF8047BCD
:106640007047000080B582B000AF786001F077FF3E
:1066500003461A46074B1A70064B1B78002B03D0D3
:10666000054B04221A6001E0FFF7A8FF00BF0837BE
:10667000BD4680BDE44A0020E014002080B485B00F
:1066800000AF7860284B1B6803F00103002B02D099
:106690000123FB7340E0244B1B6803F00203002B33
:1066A00002D00823FB7337E01F4B1B6803F0040381
:1066B000002B02D00223FB732EE01B4B1B6803F060
:1066C0000803002B02D00323FB7325E0164B1B6845
:1066D00003F48033002B05D1134B1B6803F4802394
:1066E000002B02D00623FB7316E00F4B1B6803F44C
:1066F0000033002B0BD10C4B1B6803F40023002B41
:1067000005D1094B1B6803F48013002B02D006232C
:10671000FB7301E00023FB73FB7B18461437BD4677
:106720005DF8047B704700BFE014002080B400AF28
:1067300000BFBD465DF8047B7047000080B584B0A3
:1067400000AF78607B68002B0AD0074B43F0010351
:10675000FB607B689B01BB60FB68B868984700E002
:1067600000BF1037BD4680BD503B020080B584B0ED
:1067700000AF0346FB71FB79184601F081F903462F
:10678000BB730023FB730D4B93F900307F2B09D0B3
:106790000A4B93F9003097F90E209342A8BF134695
:1067A000FB7305E097F90E307F2B01D0BB7BFB73A9
:1067B00097F90F3018461037BD4680BDDC17002012
:1067C00080B582B000AF1A4B01221A70194B7F229C
:1067D0001A70194A194B1A60184B194ADA60194B8A
:1067E00000221A7000237B6008E0174A7B685B0177
:1067F000134400221A607B6801337B607B680F2B97
:10680000F3D900233B6007E0104A3B6813447F2222
:106810001A703B6801333B603B680F2BF4D9202290
:1068200000210B481BF00CFC00BF0837BD4680BDA3
:10683000E4140020DC17002009170020E8160020CF
:1068400090170020E5140020E8140020CC17002049
:10685000A817002080B483B000AF78600B467B801F
:106860007B88DAB27B681A707B881B0A9AB27B68D5
:106870000133D2B21A7000BF0C37BD465DF8047BFD
:106880007047000080B483B000AF0346FB71FB7912
:1068900001229A40064B1B681340002B14BF0123B2
:1068A0000023DBB218460C37BD465DF8047B704709
:1068B000E817002080B58AB000AF0346FB71FB7972
:1068C000012202FA03F37B620E4B7B617B6953E882
:1068D000003F3B613B69FB60FA687B6A1343FB60E6
:1068E000FB683B62074BFB61F9693A6A41E80023A8
:1068F000BB61BB69002BE7D101F092F900BF2837DB
:10690000BD4680BDE817002080B48BB000AF0346C1
:10691000FB71FB79012202FA03F3DB437B620F4B2D
:106920007B617B6953E8003F3B613B69FB60FA6830
:106930007B6A1340FB60FB683B62084BFB61F969B3
:106940003A6A41E80023BB61BB69002BE7D100BF75
:1069500000BF2C37BD465DF8047B7047E817002068
:1069600080B489B000AF4FF0FF33FB61FB6923F0C7
:106970000103FB610F4BFB60FB6853E8003FBB600A
:10698000BB687B607A68FB6913407B607B68BB6196
:10699000084B7B617969BA6941E800233B613B6937
:1069A000002BE7D100BF00BF2437BD465DF8047B54
:1069B000704700BFE817002080B58CB000AF78604A
:1069C0000023FB623D4B00221A707B6801331B7869
:1069D00003F00803002B67D007F1080320220021F1
:1069E00018461BF02DFB7B680133BB607B681B786E
:1069F0009BB2BB8107F10803184601F04EFA03462B
:106A000087F82B3007F10803184601F02DFA0346EA
:106A100083F00103DBB2002B48D197F82B30002B19
:106A200044D0274B1B7897F82B209A4202D1254B54
:106A3000FB6212E097F82B20214B1B78013B9A4216
:106A400002D1214BFB6208E097F82B201C4B1B78EE
:106A500001339A422CD11D4BFB621D4B1B681D4A12
:106A600013601D4A97F82B301370144B01221A70D3
:106A7000FB6A3B6197F82B2007F108031146184683
:106A800001F020FA124B1B685A1C11490A6007F1E9
:106A900008021946104601F024FA07F108030F49CD
:106AA000184601F0BCF904E000BF02E000BF00E0BE
:106AB00000BF00BF3037BD4680BD00BF2418002096
:106AC000F017002004180020F417002014180020EC
:106AD000EC170020281800202C1800208817002010
:106AE000B0B586B000AF7860396000237B617B6908
:106AF0005A1C7A613A681344F4221A707B695A1C52
:106B00007A613A681344CE221A707B695A1C7A6102
:106B10003A68134436221A704FF080531B6E1846A1
:106B20004FF000014FF000024FF00003030000227D
:106B3000C7E902234FF080535B6E18464FF0000107
:106B4000D7E9022340EA020441EA0305C7E9024506
:106B50003A687B69D0187B69C3F1080207F1080322
:106B600019461BF045FA00BF1837BD46B0BD80B5C9
:106B700084B000AF78600B467B807A8807F10C0305
:106B800011461846FFF766FE07F10C0318460AF097
:106B90005FFC00BF1037BD4680BD000080B584B0EB
:106BA00000AF786039600023FB600CE0FB68C3F144
:106BB00007033A68D15C094AFB6813440A461A7015
:106BC000FB680133FB60FB68072BEFD93B68184675
:106BD0000AF049FC00BF1037BD4680BD8817002071
:106BE00080B584B000AF78600B467B807A8807F16F
:106BF0000C0311461846FFF72DFE07F10C0318464B
:106C00000AF03CFC00BF1037BD4680BD80B500AF28
:106C1000FFF7D6FD0AF075FC00BF80BD80B500AF60
:106C20000AF0D8FC0AF093FC024B00221A6000BF65
:106C300080BD00BFE817002080B582B000AF78604B
:106C4000164B1B78002B01D0002322E00AF094FCA5
:106C50000346023B052B15D801A252F823F000BFD2
:106C6000796C00007D6C0000816C00007D6C000080
:106C7000816C0000816C000001230AE0022308E01F
:106C8000032306E0064B074A40F29B1106481BF01F
:106C900039F918460837BD4680BD00BFE41400200E
:106CA000903A02003C3B0200983A020080B483B064
:106CB00000AF7860094B1B78002B14BF0123002321
:106CC000DBB283F00103DBB203F00103DBB2184651
:106CD0000C37BD465DF8047B704700BFE41400200C
:106CE00080B485B000AF78600A4A7B6813600A4BB5
:106CF0001B78002B05D0084B00221A700023FB7371
:106D000001E00D23FB73FB7B18461437BD465DF88D
:106D1000047B7047A0170020E414002080B584B0E5
:106D200000AF78600023FB737868FFF7BFFF03466E
:106D300083F00103DBB2002B15D17868FFF77CFFED
:106D40000346012B0BD00020FFF79CFD034683F088
:106D50000103DBB2002B02D00D23FB7304E0054BD3
:106D600001221A7000E000BFFB7B18461037BD46B9
:106D700080BD00BFE414002080B582B000AF786011
:106D80000AF035FC0346002B04D101F078FBFFF735
:106D9000E7FD04E0FFF7E4FD0020FFF78BFD002393
:106DA00018460837BD4680BD80B584B000AF786016
:106DB0000B46FB70FB7818460AF00BFB0AF0DCFB75
:106DC0000346022B01D101F053FBFB781846FFF775
:106DD000CDFC034618460AF01FFB0AF018FC0346D8
:106DE000FB73FFF7BDFDFB7B002B01D0002300E010
:106DF0000D2318461037BD4680BD000080B586B013
:106E000002AF786039600123FB730023BB733B68DA
:106E10009A883B681B68013BD2B21A700AF0ACFB3F
:106E20000346022B01D101F023FB386801F010F872
:106E30000346002B1ED0386801F016F80346002BDD
:106E400018D03B689B7EC3F34003DBB283F00103A1
:106E5000DBB2002B0ED02D4B1B781946386801F0A1
:106E600031F82B4B1B685A1C29490A6019463868AF
:106E700001F037F83B681B69002B16D03B681B6894
:106E8000581E3B685A693B6819693B689B790093B7
:106E90000B4601210AF0E2FB034683F00103DBB25B
:106EA000002B1ED00D23BB731BE03B689B7918465B
:106EB0000AF08FFA3B689B7E03F00403DBB2002BE1
:106EC00006D03B681B68013B18460AF0A8FC08E0A6
:106ED0003B681B68013B002118460AF0A8FB0346EB
:106EE000FB73FFF73DFD3968786805F0DCFEFB7B3E
:106EF00083F00103DBB2002B02D00220FFF7DAFCA3
:106F0000BB7B18461037BD4680BD00BFF017002080
:106F1000EC17002080B483B000AF7860034B1846B4
:106F20000C37BD465DF8047B704700BFE8160020B3
:106F300080B582B000AF78602820FFF7FFFB0AF031
:106F4000E5FB0AF0EAFB034618460837BD4680BD5C
:106F500080B483B000AF7860FB2318460C37BD4681
:106F60005DF8047B704780B582B000AF78600AF0AE
:106F7000EBFB034618460837BD4680BD80B582B09E
:106F800000AF78600B46FB70FB7818460AF0E3FB15
:106F900000BF0837BD4680BD80B582B000AF7860C5
:106FA0000B46FB70FB7818460AF0E2FB00BF08377F
:106FB000BD4680BD80B584B000AF78600B467B8055
:106FC0007A8807F10C0311461846FFF743FC07F1D6
:106FD0000C03002118460AF0D8FB0346002B02D010
:106FE0000023FB7301E00323FB73FB7B1846103780
:106FF000BD4680BD80B584B000AF786039603B6825
:10700000012118460AF0C1FB0346002B02D00023E1
:10701000FB7301E00323FB73FB7B18461037BD466F
:1070200080BD80B584B000AF78600B467B807A88E5
:1070300007F10C0311461846FFF70CFC07F10C038F
:10704000002118460AF0B4FB0346002B02D00023AF
:10705000FB7301E00A23FB73FB7B18461037BD4628
:1070600080BD80B584B000AF786039603B68012195
:1070700018460AF09DFB0346002B02D00023FB7349
:1070800001E00A23FB73FB7B18461037BD4680BD29
:1070900080B582B000AF786000200AF09AFB00BF94
:1070A0000837BD4680BD80B582B000AF7860012052
:1070B0000AF08FFB00BF0837BD4680BD80B582B0A7
:1070C00000AF78600B46FB7013463B803B884FF463
:1070D0007A7202FB03F30F4A13600F4AFB781370B6
:1070E000FFF73EFCFB7818460AF073F9094B1B6862
:1070F00018460AF0CBFA0346002B03D00520FFF711
:1071000003FC02E00520FFF7D5FB002318460837F3
:10711000BD4680BDE0170020E417002080B584B094
:1071200000AF786039600023FB733B68002B02D10D
:107130000723FB7305E00AF07DF903461A463B6816
:107140001A70FB7B18461037BD4680BD80B584B0F1
:1071500000AF78600B46FB700AF057F90346BB732B
:107160000023FB7397F903307F2B02D10723FB73B6
:107170000AE0084AFB781370BB7B1846FFF7F6FA63
:10718000034618460AF048F9FB7B18461037BD46FF
:1071900080BD00BFDC17002080B584B000AF7860F0
:1071A00039600023FB733B68002B02D10723FB737C
:1071B00010E007F1080318460AF026FB7A7A084B1C
:1071C00093F90030DBB2D31ADBB25E3BDBB25AB2CA
:1071D0003B681A70FB7B18461037BD4680BD00BF68
:1071E000DD17002080B584B000AF78600B46FB70DF
:1071F0000023FB73FA78144B93F90030DBB213448D
:10720000DBB2FB7097F9033013F15E0F02DA07234C
:10721000FB7314E007F108030422002118461AF05A
:107220000FFF00233B7297F9033018460AF042F92A
:1072300003467B7207F1080318460AF0D8FAFB7B75
:1072400018461037BD4680BDDD17002080B485B0DC
:1072500000AF786039600023FB733B68002B02D1DC
:107260000723FB7304E0064B93F900203B681A7078
:10727000FB7B18461437BD465DF8047B704700BFA2
:10728000DD17002080B584B000AF78600B46FB703E
:10729000144B1B78BB730023FB7307F10D031946D6
:1072A0007868FFF779FF0346FB73FB7B002B11D156
:1072B0000C4AFB78137097F90D3019467868FFF780
:1072C00091FF0346FB73FB7B002B05D0054ABB7B7C
:1072D000137002E000BF00E000BFFB7B18461037D0
:1072E000BD4680BDDD17002080B586B000AF786058
:1072F0000023FB7500233B6122E05E4A3B695B0192
:1073000013441B68002B18D03B695B01594A134496
:1073100000221946786805F0A2FC564A3B695B01D9
:1073200013441B68013BBB60524A3B695B01134439
:1073300000221A60B8680AF0B9F93B6901333B6171
:107340003B690F2BD9D90120FFF79CFA0346002B8C
:107350001DD00120FFF7D8FA474B1B68002B01D046
:10736000454B00E00023FB600023FA68434978683E
:1073700005F0BBFC404B1B68002B08D03E4B1B6844
:10738000013B18460AF092F93B4B00221A6002209A
:10739000FFF778FA0346002B08D00220FFF7B4FA73
:1073A0000F2300223549786805F09FFC0320FFF782
:1073B00069FA0346002B08D00320FFF7A5FA0E2335
:1073C00000222E49786805F090FC0420FFF75AFA55
:1073D0000346002B09D00420FFF796FA284B1B78B0
:1073E0001A460021786805F03AFC0620FFF74AFAB1
:1073F0000346002B09D00620FFF786FA214B93F9AC
:1074000000301946786805F096FC0020FFF73AFA3C
:107410000346002B0CD00AF0EAF80346002B05D1F6
:1074200001F02DF80020FFF76FFA01E00123FB7552
:107430000520FFF727FA0346002B12D0124B1B78CA
:10744000184609F0C6FF114B1B6818460AF01EF9D2
:107450000346002B03D00520FFF756FA01E0012375
:10746000FB75FB7D002B01D000F0DAFB00BF183765
:10747000BD4680BDE8140020A8170020E8160020B3
:10748000E5140020E5170020E4170020E017002095
:10749000F0B589B000AFF8607B600B46FB72134615
:1074A000BB720023FB610023BB6114E0454ABB694A
:1074B0005B0113441B68002B0AD1BB695B01414A85
:1074C0001344FB6120220021F8691AF0B9FD05E0A0
:1074D000BB690133BB61BB690F2BE7D9FB69002B8B
:1074E00006D1394B394A40F2EF3139481AF00AFDDA
:1074F000FB685A1CFB691A60FB681B789AB2FB692F
:107500009A80FB69FA7A5A75FB69BA7A9A7509F01A
:107510007CFF03461A46FB699A71FB6801331B78AE
:1075200003F02003002B07D02A4B1978FA69D37D8A
:1075300061F30003D37504E0FA69D37D6FF30003B0
:10754000D375FEF716FF03461E46FB681B781946E7
:10755000786809F0BDFF0346F31A7B61FEF7D6FE9B
:107560007B691A464FF00003841A61EB0305FB693F
:10757000C3E90245174B00221A70FB6801331B78E0
:1075800003F02003002B14D0F86900F055FC0346EB
:10759000002B0ED0104B1978FA69D37D61F34103AB
:1075A000D3750E4B1A68FB691A610D4B1A78FB698B
:1075B0001A75094B00221A7000F032FB00BF243705
:1075C000BD46F0BDE8140020AC3A0200583B020072
:1075D000983A0200C817002024180020281800201C
:1075E0002C18002080B582B000AF0346FB71FB79F8
:1075F000013B092B26D801A252F823F02576000082
:107600002D760000357600003D7600003D760000C6
:107610003D7600003D760000257600003D760000B6
:107620003D760000184B12221A7012E0164B112200
:107630001A700EE0144B16221A700AE0124B012247
:107640001A7006E0114B124A40F2354111481AF007
:1076500059FC114B00221A70104B00221A70FB7952
:10766000082B02D0FB79052B06D1074B00221A709C
:107670000020FFF71FF903E00420FFF71BF900BF0C
:1076800000BF0837BD4680BDE5140020903A0200D7
:107690007C3B0200983A0200C81700202418002002
:1076A00080B58AB000AF78600B46FB701346BB70A4
:1076B0007B680133BB607B681B789BB2BB817B68B6
:1076C00001331B7803F01003002B14BF01230023A8
:1076D000DAB2044B1A707868FFF76EF900BF2837EA
:1076E000BD4680BDC8170020F0B587B000AFF86078
:1076F000B96011461A460B46FB711346BB71FB6815
:10770000224A934206D0224B224A40F28441224828
:107710001AF0F8FBBB68002B03D1204B00221A6043
:107720002DE0FEF726FE03461E46BB681B78194671
:10773000386B09F0CDFE0346F31A7B61FEF7E6FDD8
:107740007B691A464FF00003841A61EB0305134B63
:10775000C3E90245BB680133104A1360BB681B785C
:107760009AB20E4B9A800D4AFB7953750B4ABB793E
:10777000937509F04AFE03461A46084B9A71012098
:10778000FFF798F800BF1C37BD46F0BD0817002072
:10779000C43A0200983B0200983A0200A817002061
:1077A00080B582B000AF78600B46FB707B68194AE9
:1077B000934206D0184B194A40F29D4118481AF0DE
:1077C000A1FBFB78013B062B18D801A252F823F04D
:1077D000ED770000F5770000F5770000ED77000009
:1077E000F5770000ED770000ED7700000220FFF74D
:1077F00061F80AE00320FFF75DF806E0094B074A4D
:1078000040F2AF4106481AF07DFB00BF0837BD4685
:1078100080BD00BF08170020C43A0200C03B020030
:10782000983A0200903A020080B582B000AF034659
:10783000FB71FB79184609F02CFE03461A46044BEF
:107840001A700620FFF736F800BF0837BD4680BD26
:10785000E517002080B483B000AF78606FF0630359
:1078600018460C37BD465DF8047B704780B584B080
:1078700000AF78600023FB737B681D4A934206D0FB
:107880001C4B1D4A40F2C6411C481AF03BFB1C48E9
:1078900000F0DEFA034683F00103DBB2002B1FD1B8
:1078A000174800F0E1FA034683F00103DBB2002B36
:1078B00016D1134B9B7E03F01003DBB2002B0FD1CC
:1078C0000F4B104A9A600123FB73FB7B83F001038B
:1078D000DBB2002B06D10C49094800F0A0FA02E007
:1078E00000BF00E000BF00BF1037BD4680BD00BF35
:1078F00008170020C43A0200DC3B0200983A02005C
:10790000E8160020041800208817002080B400AF7B
:1079100000BFBD465DF8047B704780B400AF00BF78
:10792000BD465DF8047B704780B500AF01F0D6FD21
:107930000346184680BD80B582B000AF7860FEF780
:1079400033FE02460B46104619460837BD4680BD39
:1079500090B585B000AFF8607B600B46FB721346B4
:10796000BB7297F82830002B06D01B4B1B4A40F205
:1079700017511B481AF0C6FA7B68002B05D03B6AEA
:10798000002B02D07B6A002B06D1164B134A4FF412
:10799000A36113481AF0B6FA002011F015FD124A3F
:1079A000BB7A1370114A7B6814460FCB84E80F0032
:1079B0000F4A3B6A14460FCB84E80F000D4A7B6ADE
:1079C00014460FCB84E80F00002011F007FD00BF24
:1079D0001437BD4690BD00BFDC3A0200F43B020004
:1079E000983A0200003B0200F0170020F417002034
:1079F000041800201418002080B582B000AF786011
:107A00003960002011F0E0FC044A3B68136000205C
:107A100011F0E4FC00BF0837BD4680BDEC17002024
:107A200080B584B000AF78600B46FB701346BB7026
:107A30000023FB73FB780A2B02D9FB781A2B02D99F
:107A40000723FB7315E0FB780B3B0C49BA78CA544B
:107A500009F0DBFC03461A46FB78934208D1FB7819
:107A60001846FEF783FE0346184609F0D5FC00E0F1
:107A700000BFFB7B18461037BD4680BDCC170020E9
:107A800080B485B000AF0346FB71FB790A2B02D9A5
:107A9000FB791A2B02D97F23FB7304E0FB790B3BA4
:107AA000054AD35CFB7397F90F3018461437BD466F
:107AB0005DF8047B704700BFCC17002080B582B012
:107AC00000AF78600B467B80054A7B8813807B88FB
:107AD000184600F021F8002318460837BD4680BD3F
:107AE000DE17002080B485B000AF786039600023D5
:107AF000FB733B68002B02D10723FB7303E0054BAC
:107B00001A883B681A80FB7B18461437BD465DF81F
:107B1000047B7047DE17002080B483B000AF0346BB
:107B2000FB8000BF0C37BD465DF8047B704700004A
:107B300080B582B000AF78603960174B1B78002B9E
:107B400001D000F02DF8154B0122C3F8402511F0AB
:107B500089FC00F09BFCFEF7E3FA00F0CBFB0E4B38
:107B60001B7883F00103DBB2002B01D0FEF73EFD52
:107B7000094B1B78184600F0B7FCFEF745FDFFF7F0
:107B800045F800F091F800F065FC034B00221A70F4
:107B900000BF0837BD4680BDE44A002000E0014038
:107BA00080B500AF00F05DFC00F08AF8FFF736F812
:107BB000FEF740FD0A4B1B7883F00103DBB2002B7C
:107BC00001D0FEF71AFD064B1B78184600F0A0FC0A
:107BD00000F0CAFBFEF71CFB00F05EFC00BF80BD9E
:107BE000E44A002080B400AF034B1B781846BD4622
:107BF0005DF8047B704700BFE44A002080B582B086
:107C000000AF78607868FFF76FFB00F092FC00F03F
:107C100063F87868FEF74EFB00BF0837BD4680BDAD
:107C200080B400AF00BFBD465DF8047B7047000024
:107C300080B400AF034B00221A6000BFBD465DF860
:107C4000047B704704C5004080B400AF0B4BD3F8F1
:107C5000083503F40073002B07D0084BD3F8083520
:107C60006FEA83536FEA935302E0044BD3F808356D
:107C70001846BD465DF8047B704700BF00C0004059
:107C800080B483B000AF074B0022C3F80021054B3E
:107C9000D3F800317B607B6800BF0C37BD465DF8D0
:107CA000047B704700C0004080B500AFFFF7C0FF05
:107CB000024B01221A6000BF80BD00BF00C000401F
:107CC00080B400AF034B01225A6000BFBD465DF88F
:107CD000047B704700C00040B0B584B000AF1C4BBF
:107CE0001B68FB601B4BD3F80031002B06D0FFF75D
:107CF000C7FFFFF7A9FF0346154A1360FEF706FB0F
:107D0000C7E90001144BD3E90023D7E90001841A25
:107D100061EB03050CA3D3E90023AB4208BFA242E9
:107D200007D20C4B01221A600B49D7E90023C1E9A5
:107D30000023074B1B68FA689A4201D009F082FBC6
:107D400000BF1037BD46B0BD80C3C90100000000B0
:107D50003818002000C000403018002080B400AF68
:107D600000BFBD465DF8047B704780B400AF00BF24
:107D7000BD465DF8047B704780B400AF054B1B68BF
:107D8000002B00DA03339B105BB21846BD465DF84A
:107D9000047B70473818002080B483B000AF0346DE
:107DA000FB7100BF0C37BD465DF8047B704780B5A2
:107DB00082B000AF7860786802F0BAFE03461846D9
:107DC00000F019F8034618460837BD4680BD80B557
:107DD00082B000AF78607868FCF7D0FA03461B7871
:107DE00003F02003002B14BF01230023DBB218464D
:107DF0000837BD4680BD80B483B000AF0346FB802A
:107E0000FB8803F44053B3F5005F0CBF012300234C
:107E1000DBB218460C37BD465DF8047B704780B571
:107E200082B000AF786039603968786803F0B3FADF
:107E300000BF0837BD4680BD80B582B000AF786016
:107E40007868FFF7B4FF034618460837BD4680BD83
:107E500080B582B000AF78607868FCF767FA0346B7
:107E600018460837BD4680BD80B584B000AF786045
:107E700007F10E031946786802F02EFF0346FB73E4
:107E8000FB7B002B04D1BB7B082B01D1012300E03D
:107E9000002318461037BD4680BD80B584B000AFC2
:107EA00078600023FB7307F10F031946786802F02E
:107EB000CDFF03461846FFF76FFFFB7B18461037D0
:107EC000BD4680BD80B582B000AF78600B46FB70C8
:107ED000FB781946786802F0E7FF00BF0837BD4617
:107EE00080BD80B582B000AF78603960396878684D
:107EF00002F037FF00BF0837BD4680BD80B483B0B5
:107F000000AF0346FB71FB7903F01F02074997F9A5
:107F100007305B09012000FA02F241F8232000BF7C
:107F20000C37BD465DF8047B704700BF00E100E000
:107F300080B483B000AF0346FB71FB7903F01F02EE
:107F4000074997F907305B09012000FA02F2203354
:107F500041F8232000BF0C37BD465DF8047B704715
:107F600000E100E080B483B000AF0346FB71FB7911
:107F700003F01F02074997F907305B09012000FA57
:107F800002F2603341F8232000BF0C37BD465DF894
:107F9000047B704700E100E080B483B000AF03468B
:107FA0003960FB7197F90730002B0BDA3B68DAB2C6
:107FB0000C49FB7903F00F03043B5201D2B20B448E
:107FC0001A7609E03B68DAB2074997F9073052019F
:107FD000D2B20B4483F8002300BF0C37BD465DF8D6
:107FE000047B704700ED00E000E100E080B483B066
:107FF00000AF7860044A7B68C2F8043300BF0C37D6
:10800000BD465DF8047B704700D0004080B483B06B
:1080100000AF7860044A7B68C2F8083300BF0C37B1
:10802000BD465DF8047B704700D0004080B483B04B
:1080300000AF0346FB71084BD3F80823FB791340CC
:10804000002B14BF01230023DBB218460C37BD46BA
:108050005DF8047B704700BF00D0004080B483B05F
:1080600000AF0346FB71FB7903F1804303F55043F6
:1080700001221A6000BF0C37BD465DF8047B7047D3
:1080800080B485B000AF0346FB80FB8803F18043DA
:1080900003F5504300221A60FB8803F1804303F587
:1080A00050431B68FB60FB6800BF1437BD465DF89A
:1080B000047B704780B483B000AF0346FB80FB882D
:1080C00003F1804303F550431B68002B14BF0123C9
:1080D0000023DBB218460C37BD465DF8047B7047C1
:1080E00080B483B000AF7860074BD3F800227B6880
:1080F000DB4305491340C1F8003200BF0C37BD46D1
:108100005DF8047B704700BF00D0004080B400AF32
:10811000044BD3F80835DBB21846BD465DF8047B46
:10812000704700BF00D0004080B400AF064BD3F8CA
:108130000435054A43F00103C2F8043500BFBD46CB
:108140005DF8047B704700BF00D0004080B483B06E
:1081500000AF064B1B687B60054B1B687A68D31A1F
:1081600018460C37BD465DF8047B7047C4180020E4
:10817000C018002080B500AFFFF7E8FF0346002BD2
:108180000CBF01230023DBB2184680BD80B500AFD1
:10819000FFF7DCFF0346032B8CBF01230023DBB278
:1081A000184680BD80B500AFFFF7D0FF03467F2B98
:1081B0008CBF01230023DBB2184680BD80B582B09E
:1081C00000AF0346FB71FFF7EDFF034683F00103A9
:1081D000DBB2002B09D0074B1B685A1C05490A600B
:1081E00003F07F030449FA79CA5400BF0837BD463B
:1081F00080BD00BFC41800204018002080B582B0A8
:1082000000AF0023FB71FFF7B5FF034683F00103C6
:10821000DBB2002B09D0074B1B685A1C05490A60CA
:1082200003F07F03044AD35CFB71FB7918460837DF
:10823000BD4680BDC01800204018002080B582B027
:1082400000AF00237B60FFF7A1FF0346002B12D095
:1082500000233B600CE07B681B027B60FFF7CEFFD6
:1082600003461A467B6813437B603B6801333B60DF
:108270003B68032BEFD97B6818460837BD4680BDA5
:1082800080B500AF4FF48070FFF7FAFE0120FFF7D2
:10829000ADFE0020FFF7E2FE00BF80BD80B500AF5D
:1082A0000120FFF7B3FE0420FFF7D8FE00BF80BD1A
:1082B00080B500AF4FF48070FFF7FCFE0346002B43
:1082C00016D00120FFF7B2FE0346002B10D04FF46A
:1082D0008070FFF7D5FEFFF719FF03461846FFF73A
:1082E0006DFFFFF75FFF0346002B01D0FFF7D6FFBE
:1082F00000BF80BD80B582B000AF00237B608022CC
:108300000021164819F09CFE154B00221A60154BEF
:1083100000221A6006210D20FFF73EFE0D20FFF718
:1083200021FE0D20FFF7EAFDFFF7FEFE0120FFF71B
:10833000D7FEFFF7A5FF00BFFFF728FF034683F036
:108340000103DBB2002BF7D1FFF778FF7860786884
:108350001AF06CF900BF0837BD4680BD40180020F8
:10836000C0180020C418002080B500AFFFF796FFAA
:108370000D20FFF7DDFD0D20FFF7F4FD00210D209E
:10838000FFF70AFE00BF80BD90B585B000AF7860F2
:108390000B467B800023FB730023BB81294B1B789A
:1083A000DBB283F00103DBB2002B05D1264B274A59
:1083B000C721274819F0A6FD224B01221A707B68BD
:1083C000002B02D07B88002B02D10723FB7331E006
:1083D000FFF7BCFE0346BB73BA7B7988BB89CB1A17
:1083E0009A4205DD7B88DAB2BB89DBB2D31ABB7354
:1083F000BB7B002B19D00023BB600BE0BA89BB68A4
:1084000013447A68D418FFF7F9FE03462370BB685B
:108410000133BB60BB7BBA689A42EFD3FFF730FFF2
:10842000BB7B9AB2BB891344BB81BA897B889A42D1
:10843000CED300BF034B00221A70FB7B18461437C3
:10844000BD4690BD3C1800200C3C0200383C0200A8
:10845000203C020080B400AF00BFBD465DF8047B45
:10846000704780B400AF00BFBD465DF8047B704725
:1084700080B400AF00BFBD465DF8047B704780B498
:1084800000AF00BFBD465DF8047B704780B500AF0C
:1084900000F008F800BF80BD80B500AF00F018F80C
:1084A00000BF80BD80B582B000AF0121002010F078
:1084B00039FF78607B68002B03DB044B01221A70C4
:1084C00000E000BF00BF0837BD4680BDC8180020CF
:1084D00080B400AF034B00221A7000BFBD465DF8A8
:1084E000047B7047C818002080B582B000AF0346F7
:1084F000FB71FB7983F00103DBB2002B02D000F0AB
:10850000A3F901E000F012FA00BF0837BD4680BDB4
:1085100080B582B000AF0346FB71FB7983F00103A5
:10852000DBB2002B01D000F0E3F900BF0837BD46F5
:1085300080BD80B500AF00F00BFA00BF80BD80B4F5
:1085400000AF01231846BD465DF8047B704780B438
:1085500083B000AF78607B6818460C37BD465DF885
:10856000047B704780B483B000AF78607B681846A6
:108570000C37BD465DF8047B7047000080B584B0C1
:1085800000AF78600B46FB707868FFF7EBFFF86090
:10859000FB78032B24D801A252F823F0CD850000EC
:1085A000C5850000AD850000E18500004FF4007234
:1085B0000E490F4818F0A4F9FDF7B2FE03460D4A24
:1085C00013610EE00B4B0122DA750AE0094B012220
:1085D0001A76F86818F085F90346064A936000E0B9
:1085E00000BF00BF1037BD4680BD00BF541900203A
:1085F0004C3C0200541B002080B582B000AF786074
:108600000B46FB70FFF70CFB00BF0837BD4680BD73
:1086100080B582B000AF0346FB71FB79083B062BA7
:1086200022D801A252F823F04B86000059860000A0
:108630006186000069860000698600006986000086
:108640004586000014F014FE0FE00A4B00221A8445
:10865000094B01221A7508E0074B00221A7504E045
:10866000054B01225A7500E000BF00BF0837BD4628
:1086700080BD00BFCC180020541B002080B582B004
:1086800000AFFDF74DFE0246094B1B69D31A7B6014
:108690007B68002B02DB7B680A2B01DD012300E0F5
:1086A000002303F00103DBB218460837BD4680BD46
:1086B000541B002080B582B000AF3B1D1A4601213B
:1086C0000C4818F081F90346002B0ED17B68002B73
:1086D00006D0FFF7D3FF0346002B01D0012300E0B3
:1086E000002303F00103DBB200E000231846083743
:1086F000BD4680BD4C3C020080B582B000AF224B2D
:108700001B7B002B06D0204B1B7DDBB2002B01D046
:10871000012300E00023FB71FB7903F00103FB71EF
:10872000194B5B7BFA799A421AD0174AFB7953733B
:10873000FB79002B0AD013F0C7FC034683F001033A
:10874000DBB2002B0CD014F08DFD09E013F0CCFC53
:108750000346002B02D014F0ADFD01E014F088FDBB
:10876000094B5B7DDBB2002B09D0074B00225A7509
:1087700013F0AAFC0346002B01D014F07FFD00BFCC
:108780000837BD4680BD00BF541B002080B500AF38
:10879000104B1B7EDBB2002B19D00E4B9B68002BBD
:1087A00009D00C4B9B689BB219460B48F8F7C9FDE2
:1087B000084B00229A604FF400720749074818F0EE
:1087C0009FF80346002B02D1024B00221A7600BF0D
:1087D00080BD00BF541B0020541900204C3C0200F7
:1087E00080B500AF164B1B68002B19D0FFF762FF56
:1087F0000346002B14D0124B1B68114A928819466D
:10880000104818F01FF80346002B17D10C4B01221B
:108810009A750B4B00221A60094B00229A800DE0DA
:10882000074BDB7DDBB2002B08D0054B0022DA754D
:10883000034B00229A75F8F793FDFFE700BF80BD58
:10884000541B00204C3C020080B582B000AF1C22BB
:108850000021214819F0F4FB16F0D6FA1F4814F055
:10886000DDFB78607B68002B06D01D4B1D4A40F273
:1088700013111D4819F046FB16F0EAFB78607B687F
:10888000002B06D0164B174A40F21711164819F064
:1088900039FB1648FFF75BFE3860386814F0FEFFBE
:1088A00078607B68002B06D00D4B0E4A4FF48E711A
:1088B0000D4819F027FB14F0AFFC78607B68002BA3
:1088C00006D0074B074A40F21F11074819F01AFB60
:1088D00000BF0837BD4680BD541B0020A83C0200E5
:1088E000703C0200B43C0200843C02004C3C02009C
:1088F00080B500AF13F0F8FB0346002B08D014F04E
:10890000D9FC00BF14F050FF0346002BFAD106E05B
:1089100013F0DAFB0346002B01D014F0A9FC15F08C
:108920009BF814F015FC00BF80BD000080B400AFC0
:10893000064B00229A75054B00221A60034B002259
:108940009A8000BFBD465DF8047B7047541B002031
:1089500080B500AF00BF14F027FF0346002BFAD10B
:10896000FFF7CAFEFFF712FFFFF73AFF00BF80BD17
:1089700080B400AF044B01221A7300231846BD4691
:108980005DF8047B704700BF541B002080B584B0A5
:1089900000AF78600B467B800023FB73184B9B7DF8
:1089A000DBB2002B01D000F02FF8154B1B68002B19
:1089B00002D00523FB731DE0FFF77CFE034683F026
:1089C0000103DBB2002B06D00D4A7B6813600C4A12
:1089D0007B8893800EE07B881A467968094817F0F7
:1089E00031FF0346002B02D00123FB7302E0044B4E
:1089F00001229A75FB7B18461037BD4680BD00BF2B
:108A0000541B00204C3C020080B500AF09E000BFC1
:108A100014F0CAFE0346002BFAD1FFF76DFEFFF7F4
:108A2000DFFE094B9B7DDBB2002B07D0064BDB7DC5
:108A3000DBB283F00103DBB2002BE8D1FFF7D0FEFD
:108A40000023184680BD00BF541B002080B483B0B3
:108A500000AF7860034B18460C37BD465DF8047BC9
:108A6000704700BF701B002080B582B000AF7860F7
:108A70007868FFF7EBFF034618460837BD4680BD10
:108A800080B483B000AF78607B68113318460C3730
:108A9000BD465DF8047B704780B500AF00F0F6FD81
:108AA0000346184680BD80B483B000AF78600123D0
:108AB00018460C37BD465DF8047B704780B582B020
:108AC00000AF7860786800F031F80346184600F08F
:108AD00046FE00BF0837BD4680BD80B582B000AFFE
:108AE0007860786800F022F80346184600F0FEFD32
:108AF00000BF0837BD4680BD80B582B000AF78604A
:108B0000786800F013F80346184600F0FAFD00BF3D
:108B10000837BD4680BD000080B400AF024B184648
:108B2000BD465DF8047B7047C43C020080B483B04E
:108B300000AF78607B6818460C37BD465DF8047B53
:108B4000704780B584B000AFF860B9601346FB7120
:108B5000FB68FA79B968184602F03DFD00BF10378E
:108B6000BD4680BD80B582B000AF78607868FFF701
:108B70007BFF03461846FEF7F6F90346184608370A
:108B8000BD4680BD80B582B000AF78600B46FB70FB
:108B90007868FFF769FF0246FB7819461046FEF732
:108BA000EDF900BF0837BD4680BD80B582B000AF8B
:108BB00078607868FFF758FF03461846FEF7DCF840
:108BC000034618460837BD4680BD80B582B000AF69
:108BD00078607868FFF748FF03461846FEF7A8F963
:108BE000034618460837BD4680BD80B582B000AF49
:108BF00078600B46FB707868FFF736FF0246FB781B
:108C000019461046FEF7C8F900BF0837BD4680BDBB
:108C100080B582B000AF78600B467B807868FFF744
:108C200023FF02467B8819461046FEF7C3F9034628
:108C300018460837BD4680BD80B582B000AF786069
:108C400039607868FFF710FF02463B681946104606
:108C5000FEF7D0F9034618460837BD4680BD80B5FB
:108C600082B000AF78600B467B807868FFF7FCFE2F
:108C700002467B8819461046FEF7D3F9034618468C
:108C80000837BD4680BD80B582B000AF78603960DE
:108C90007868FFF7E9FE02463B6819461046FEF782
:108CA000E0F9034618460837BD4680BD80B582B05E
:108CB00000AF78607868FFF7D7FE03461846FEF7E6
:108CC000E7F900BF0837BD4680BD80B582B000AF70
:108CD00078607868FFF7C8FE03461846FEF7E3F9A8
:108CE00000BF0837BD4680BD80B483B000AF786058
:108CF0007B689B8818460C37BD465DF8047B70473F
:108D000080B483B000AF78607B68063318460C37B8
:108D1000BD465DF8047B704780B483B000AF7860D7
:108D20007B685B6918460C37BD465DF8047B70476D
:108D300080B483B000AF78607B685B68002B14BFA1
:108D400001230023DBB218460C37BD465DF8047BD7
:108D5000704780B582B000AF78607B6810331846EA
:108D600002F00EFF034618460837BD4680BD80B5A9
:108D700082B000AF78607B6810331846FFF7CCFFF5
:108D8000034618460837BD4680BD80B582B000AFA7
:108D900078607B6810331846FFF7A6FF0346184635
:108DA0000837BD4680BD80B483B000AF78607B6873
:108DB0005B8818460C37BD465DF8047B704780B46D
:108DC00083B000AF78607B681B7818460C37BD46CF
:108DD0005DF8047B704780B582B000AF78607B6837
:108DE00010331846FFF78CFF034618460837BD4678
:108DF00080BD80B483B000AF78607B6814331846C0
:108E00000C37BD465DF8047B704780B582B000AF7B
:108E1000786039607868FFF789FE03461846FFF7E7
:108E2000E8FF03463968184601F050FB0346184630
:108E30000837BD4680BD80B582B000AF78607868E5
:108E4000FFF774FE03461846FFF7D3FF03461846A4
:108E5000FFF76EFF034618460837BD4680BD80B554
:108E600082B000AF78600B467B807868FFF75EFECB
:108E700003461846FFF7BDFF02467B881946104699
:108E800001F0B2FB034618460837BD4680BD80B5E9
:108E900082B000AF78607868FFF748FE0346184656
:108EA000FFF7EEFD03461846FFF75CFE0346184643
:108EB0000837BD4680BD80B584B000AF78600B46F2
:108EC000FB700023FB737868FFF730FEB860B8686A
:108ED000FFF78FFF03461846FFF72AFF034683F08C
:108EE0000103DBB2002B02D00D23FB7308E0B8684E
:108EF000FFF7C6FD0246FB7819461046FFF742FE13
:108F0000FB7B18461037BD4680BD80B584B000AFEE
:108F100078600023FB737868FFF708FEB860B868D4
:108F2000FFF767FF03461846FFF702FF034683F08B
:108F30000103DBB2002B02D00D23FB7308E0B868FD
:108F4000FFF79EFD03461846FFF72FFE0346FB730F
:108F5000FB7B18461037BD4680BD80B582B000AFA0
:108F600078607868FFF7E2FD03461846FFF741FF97
:108F70000346184601F058FB034618460837BD461D
:108F800080BD80B582B000AF78607868FFF7CEFD15
:108F900003461846FFF72DFF03461846FFF7E7FE86
:108FA000034618460837BD4680BD80B582B000AF85
:108FB000786039607868FFF7B9FD03461846FFF717
:108FC00018FF03463968184601F073FB034618463C
:108FD0000837BD4680BD80B582B000AF7860786844
:108FE000FFF7A4FD03461846FFF703FF03461846A4
:108FF000FFF7AFFE034618460837BD4680BD80B573
:1090000084B000AFF8607B600B46FB7213463B8177
:10901000F868FFF78BFD03461846FFF7EAFE3A892A
:10902000F97A7B6801F08CFB034618461037BD4681
:1090300080BD80B584B000AF78600B46FB70002324
:10904000FB737868FFF772FDB860B868FFF7D1FE70
:1090500003461846FFF76CFE034683F00103DBB2BC
:10906000002B02D00D23FB7308E0B868FFF708FD62
:109070000246FB7819461046FFF7B7FDFB7B184602
:109080001037BD4680BD80B584B000AF78600B4618
:109090007B800023FB737868FFF748FDB860B868F1
:1090A000FFF7A7FE03461846FFF742FE034683F08C
:1090B0000103DBB2002B02D00D23FB730AE0B8687A
:1090C000FFF7DEFC02467B8819461046FFF7A0FD3D
:1090D0000346FB73FB7B18461037BD4680BD80B549
:1090E00086B000AF786039600023FB757868FFF7C1
:1090F0001DFD38613869FFF77CFE03461846FFF70F
:1091000017FE034683F00103DBB2002B02D00D23D0
:10911000FB7512E0396807F1080301221846FFF7D2
:1091200010FD3869FFF7ACFC024607F10803194649
:109130001046FFF781FD0346FB75FB7D1846183787
:10914000BD4680BD80B584B000AF78600B467B80A3
:109150000023FB737868FFF7E9FCB860B868FFF795
:1091600048FE03461846FFF7E3FD034683F001037C
:10917000DBB2002B02D00D23FB730AE0B868FFF7C7
:109180007FFC02467B8819461046FFF768FD0346C0
:10919000FB73FB7B18461037BD4680BD80B586B09B
:1091A00000AF786039600023FB757868FFF7BEFC7C
:1091B00038613869FFF71DFE03461846FFF7B8FD12
:1091C000034683F00103DBB2002B02D00D23FB75B5
:1091D00012E0396807F1080301221846FFF7B1FCD5
:1091E0003869FFF74DFC024607F10803194610469F
:1091F000FFF749FD0346FB75FB7D18461837BD4652
:1092000080BD80B584B000AF78600023FB737868C0
:10921000FFF78CFCB860B868FFF7EBFD0346184613
:10922000FFF786FD034683F00103DBB2002B02D07B
:109230000D23FB7306E0B868FFF722FC03461846CF
:10924000FFF734FDFB7B18461037BD4680BD80B567
:1092500084B000AF78600023FB737868FFF766FC8A
:10926000B860B868FFF7C5FD03461846FFF760FD14
:10927000034683F00103DBB2002B02D00D23FB7306
:1092800006E0B868FFF7FCFB03461846FFF71DFD34
:10929000FB7B18461037BD4680BDF0B587B002AFE6
:1092A000F8607B600B46FB721346BB72F868FFF7F1
:1092B0003DFC03461846FFF79CFD0546786800F024
:1092C000E1F80646B86A00F0DDF80446F86A00F0F6
:1092D000D9F80346BA7AF97A0193009433462846BE
:1092E00001F087FA034618461437BD46F0BD80B535
:1092F00082B000AF786039607868FFF717FC0346EA
:109300001846FFF776FD03463968184601F0C4FA9F
:10931000034618460837BD4680BD80B582B000AF11
:109320007860FDF741F902460B46104619460837AA
:10933000BD4680BD80B582B000AF78607868FFF729
:10934000F5FB03461846FFF754FD03461846FFF7A2
:1093500036FD034618460837BD4680BD80B582B04D
:1093600000AF78600B46FB707868FFF7DFFB0346C1
:109370001846FFF73EFD0246FB781946104601F0FD
:10938000F9F8034618460837BD4680BD80B582B05F
:1093900000AF78607868FFF7C9FB03461846FFF70F
:1093A00028FD03461846FFF7FEFC0346184608371B
:1093B000BD4680BD80B582B000AF78600B467B8033
:1093C0007868FFF7B3FB03461846FFF712FD024625
:1093D0007B881946104601F0AAF80346184608375C
:1093E000BD4680BD80B582B000AF78607868FFF779
:1093F0009DFB03461846FFF7FCFC03461846FFF7A3
:10940000EAFC034618460837BD4680BD90B583B0D8
:1094100000AF786039607868FFF788FB034618462C
:10942000FFF7E7FC0446386800F037F803461946B2
:10943000204601F0BBF8034618460C37BD4690BDE8
:1094400080B582B000AF78607868FFF76FFB0346A5
:109450001846FFF7CEFC03461846FFF796FC034676
:1094600018460837BD4680BD80B582B000AF786031
:1094700039603B6819467868FDF732FB00BF083752
:10948000BD4680BD80B483B000AF78607B6818466D
:109490000C37BD465DF8047B704780B483B000AFE5
:1094A00078607B6818460C37BD465DF8047B7047D2
:1094B00080B400AF01231846BD465DF8047B7047B9
:1094C00080B500AFFFF7F4FF0346184680BD80B5B6
:1094D00000AF00F0C7F90346184680BD80B500AF65
:1094E000FFF7F5FF0346184680BD80B483B000AF98
:1094F00078607B68043318460C37BD465DF8047B02
:10950000704780B582B000AF78607868FFF7CBFA1B
:10951000034683F00103DBB2002B0BD17868FFF721
:1095200005FB03461846FFF7E0FF0346184600F028
:109530007FFA00E000BF00BF0837BD4680BD80B4A1
:1095400083B000AF0346FB7100BF0C37BD465DF82A
:10955000047B704780B483B000AF78607B680022E2
:109560001A607B6818460C37BD465DF8047B70476F
:1095700080B582B000AF7860396039687868F7F7F5
:1095800039FF7B68184600F00EF97B6818460837EB
:10959000BD4680BD80B582B000AF786039607B6821
:1095A00039681846FFF7E4FF7B6818460837BD4660
:1095B00080BD80B582B000AF786039607B68396863
:1095C0001846FFF7D5FF7B6818460837BD4680BDB3
:1095D00080B582B000AF7860396039687868F7F795
:1095E00009FF7B6818460837BD4680BD80B582B04C
:1095F00000AF7860396039687868F7F7FBFE7B6800
:10960000013339681846FFF7E3FF7B6818460837CF
:10961000BD4680BD80B483B000AF78607B682433E2
:1096200018460C37BD465DF8047B704780B582B0A4
:1096300000AF78607B6804331846FFF78BFF7B68C8
:10964000083379681846FFF7A5FF7B680C33796803
:109650001846FFF7AEFF7B681033184600F0B2F8EB
:109660007B68113379681846FFF7C0FF7B681433B5
:109670007968184600F0E3FE7B68002283F88C20AE
:109680007B6818460837BD4680BD000090B583B0A2
:1096900000AF00F01DF878607B6893F88C30002BE9
:1096A0000DD10A4B19469020F7F7C5FE0446204617
:1096B000FFF7BCFF7C60786800F035F800E000BF81
:1096C0007B6818460C37BD4690BD00BF701B00205C
:1096D00080B483B000AF044B7B607B6818460C37C6
:1096E000BD465DF8047B7047701B002080B582B0DA
:1096F00000AF78607868FCF7A5FF00BF0837BD466B
:1097000080BD80B582B000AF78607B6811331846A9
:1097100003F0EAF97B681433184600F0B7FE00BF87
:109720000837BD4680BD80B483B000AF78607B68E9
:10973000012283F88C2000BF0C37BD465DF8047B06
:10974000704780B582B000AF78607B6810331846F0
:1097500000F06CF87B6818460837BD4680BD80B5C0
:1097600082B000AF78607B6893F88C3083F001039F
:10977000DBB2002B12D17B68002283F88C20786842
:10978000FFF748FF0346184602F0A2FA03461846C0
:10979000FFF7D5FE7868FFF7D4FF00E000BF00BFF9
:1097A0000837BD4680BD80B483B000AF78607B6869
:1097B00000221A607B6818460C37BD465DF8047BB2
:1097C0007047000080B584B000AF7860154B1B88EF
:1097D0004FF6FF72934200D1FEE7124B1B88002B1D
:1097E00014D107F10C0304211846FEF7CDFD034602
:1097F000002B14BF01230023DBB2002B00D0FEE7B7
:10980000FB681946084800F03FF800E000BF054B30
:109810001B8801339AB2034B1A807B6818461037B5
:10982000BD4680BD001C0020041C002080B483B015
:1098300000AF78600A4B1B88002B00D1FEE7084B75
:109840001B88013B9AB2064B1A80054B1B88002BE4
:1098500000BF7B6818460C37BD465DF8047B704737
:10986000001C002080B500AF054B1B88002B00D1E9
:10987000FEE7044800F020F80346184680BD00BF0C
:10988000001C0020041C002080B483B000AF78606E
:1098900039603B68002B04D03B686FF00042934274
:1098A00001D101233B607B683A681A6000BF0C3726
:1098B000BD465DF8047B704780B489B000AF786026
:1098C0007B681B681A464FF0000348F24E3101FBDB
:1098D00003F0002101FB02F1014448F24E30A2FBEB
:1098E000002319440B46C7E90423C7E904233B6955
:1098F000FB60FB685B08FB60D7E904014FF00002E6
:109900004FF000030A0000231346BB60BA68FB68EF
:109910001344FB61FB69002B06DAFB6923F000436B
:10992000FB61FB690133FB617B68FA691A60FB69C3
:1099300018462437BD465DF8047B704780B582B079
:1099400000AF786039603A687B689A4200D8FEE7D9
:10995000FFF7BDFD024639687B68CB1AB2FBF3F115
:1099600003FB01F3D21A7B68134418460837BD463F
:1099700080BD80B483B000AF78607B685B68002BEB
:1099800014BF01230023DBB218460C37BD465DF837
:10999000047B704780B582B000AF78607B681B683D
:1099A0007868984700BF0837BD4680BD80B582B053
:1099B00000AF78607868FFF7DCFF034683F00103AF
:1099C000DBB2002B07D0786800F058F803467968BE
:1099D000184600F004F800BF0837BD4680BD80B5CA
:1099E00082B000AF786039607B681B68002B0FD1B4
:1099F0007B683A681A607B681B687A6812685A60EC
:109A00003868FFF723F803461846F7F753FC0BE0D6
:109A10007B681B685A683B685A607B681B683A68B9
:109A20005A607B683A681A6000BF0837BD4680BD3F
:109A300080B584B000AF78607B681B68FB607B6892
:109A400000221A60FB68002B14D0FB685B68BB60C7
:109A5000BA68FB689A4202D10023FB6003E0BB684E
:109A60005A68FB685A60BB6800225A60B868FFF702
:109A700091FFE7E700BF1037BD4680BD80B582B0DB
:109A800000AF78607868FEF7E1FF03461846FFF7FD
:109A90002CFD034618460837BD4680BD80B582B010
:109AA00000AF786039603968786800F011F87B6839
:109AB00018460837BD4680BD80B483B000AF7860DB
:109AC0007B681B6818460C37BD465DF8047B704701
:109AD00080B483B000AF786039607B683A681A6000
:109AE00000BF0C37BD465DF8047B704780B483B07F
:109AF00000AF786039607B681A683B681B68D31ACE
:109B000018460C37BD465DF8047B704780B584B0BD
:109B100000AF786039607B681A683B681A4407F1C7
:109B20000C0311461846FFF7B9FFFB6818461037BB
:109B3000BD4680BD80B582B000AF786039607B687B
:109B40001A683B681B681946104600F0B4FA0346D1
:109B500018460837BD4680BD80B582B000AF78603A
:109B6000396039687868FFF7E5FF034683F0010341
:109B7000DBB218460837BD4680BD80B483B000AF65
:109B800078607B685B6818460C37BD465DF8047BDF
:109B9000704780B483B000AF78607B689B687A6858
:109BA0009A4214BF01230023DBB218460C37BD468E
:109BB0005DF8047B704780B582B000AF78607B6849
:109BC0001B687868984700BF0837BD4680BD000015
:109BD00080B582B000AF78607B680449184600F019
:109BE000ADF900BF0837BD4680BD00BF1C3D020077
:109BF00080B582B000AFFCF793FB02463B1D1146D7
:109C00001846FFF74BFF7B6818460837BD4680BDF6
:109C100080B582B000AF786039607B683968044AEB
:109C2000184600F0A8F800BF0837BD4680BD00BF49
:109C3000283D020080B582B000AF786039607B6853
:109C40003968044A184600F0F2F800BF0837BD46EC
:109C500080BD00BF283D020080B582B000AF7860B3
:109C60007B680449184600F069F900BF0837BD4613
:109C700080BD00BF283D020080B582B000AFFCF778
:109C800078FB02463B1D11461846FFF707FF7B682D
:109C900018460837BD4680BD80B483B000AF034688
:109CA000FB7100BF0C37BD465DF8047B704780B484
:109CB00083B000AF78607B68083318460C37BD4628
:109CC0005DF8047B704780B483B000AF78607B6838
:109CD0000C3318460C37BD465DF8047B704780B5E1
:109CE0008AB000AFF860B9607A60F868FFF745FFA6
:109CF00003467B613A1D07F1140311461846FFF72E
:109D000019FF034687F82630B868FFF736FF034689
:109D1000BB613A1D07F1180311461846FFF70AFF09
:109D200003461A4697F82630934214BF01230023B6
:109D3000DBB2002B04D097F8263087F8273014E0E8
:109D4000F868FFF71AFF0346FB61B868FFF715FFD5
:109D500003463B6207F1200207F11C031146184637
:109D6000FFF7E8FE034687F8273097F827301846B4
:109D70002837BD4680BD80B58AB000AFF860B960B5
:109D80007A6000237B627B689B689847024607F1F4
:109D9000180311461846FFF781FE7A68B968F8681B
:109DA00000F045F8FB683B62386A00F094F903461E
:109DB0007B61386A00F0A2F903463B6107F11002AB
:109DC00007F114031146184600F0A7F90346002BCB
:109DD00016D007F11403184600F0BEF9F861BA690D
:109DE000F969B868FFF77BFF0346002B07D1FB69D1
:109DF0007B6207F11403184600F0A3F9DEE700BF09
:109E00007B6A002B09D1FB68B968184600F0B0F9ED
:109E10007968F86800F043F805E0FB687A6AB96889
:109E2000184600F0B7F900BF2837BD4680BD80B5A1
:109E300084B000AFF860B9607A60B868FFF7A9FE37
:109E4000034683F00103DBB2002B23D1FB681846E5
:109E500000F0B6F90246BB6893420CBF0123002311
:109E6000DBB2002B08D0FB68184600F0B5F9796822
:109E7000F86800F014F808E0FB68B968184600F0CC
:109E8000C3F903461846FFF707FFB968B86800F042
:109E9000D6F900E000BF00BF1037BD4680BDB0B5A9
:109EA00086B000AF786039607B68184600F0D5F95D
:109EB0000346002B08D03B685C687868FEF7C6FD57
:109EC00003461846A04735E07B68184600F078F94D
:109ED00078613B689B689847024607F10C0311467E
:109EE0001846FFF7DBFD7B691A1D07F10C031146CD
:109EF0001846FFF71FFE0346002B09D07B69043389
:109F000007F10C0211461846FFF7F0FD034600E08A
:109F100000233B613B681C687868FEF797FD0546A7
:109F200007F10C031846FFF7C7FD03463A691946C7
:109F30002846A04700BF1837BD46B0BD80B584B0E5
:109F400000AF786039607B68184600F039F9F86036
:109F5000FB68002B1DD03B689B689847024607F1C1
:109F6000080311461846FFF799FDFB681A1D07F113
:109F7000080311461846FFF7EFFD0346002B08D0F3
:109F80003A68F9687868FFF752FFF868FFF713FE40
:109F900004E039687868FFF782FF00BF1037BD46DC
:109FA00080BD80B582B000AF78607868FEF77BFD39
:109FB000034683F00103DBB2002B0BD17868FEF778
:109FC000B5FD03461846FFF772FE03461846FFF735
:109FD000FFFD00E000BF00BF0837BD4680BD80B573
:109FE00082B000AF78603960FFF746FE03463A68FA
:109FF0001946786800F004F800BF0837BD4680BDF8
:10A0000080B584B000AFF860B9607A607B68002BDF
:10A0100000DAFEE707F1080379681846FFF776FDD6
:10A0200003461946F86800F004F800BF1037BD4633
:10A0300080BD80B582B000AF786039607B683A68D7
:10A040005A60786800F01AF9034679681846FFF7F5
:10A05000DFFD00BF0837BD4680BD80B582B000AFD0
:10A060007860786800F00AF9034679681846FFF7C7
:10A07000E1FD00BF0837BD4680BD80B582B000AFAE
:10A0800078607868FEF70FFD034683F00103DBB2CA
:10A09000002B0BD17868FEF749FD03461846FFF701
:10A0A00012FE03461846FFF7D7FD00E000BF00BFD1
:10A0B0000837BD4680BD80B483B000AF786039609A
:10A0C0007A683B68D31ADB0FDBB218460C37BD4603
:10A0D0005DF8047B704780B584B000AF7860786825
:10A0E00000F06EF8024607F10C031146184600F026
:10A0F000D5F8FB6818461037BD4680BD80B584B0E2
:10A1000000AF786007F10C030021184600F0C6F894
:10A11000FB6818461037BD4680BD80B483B000AFE1
:10A12000786039607B681A683B681B689A4214BF84
:10A1300001230023DBB218460C37BD465DF8047BD3
:10A14000704780B582B000AF7860786800F0B5F8ED
:10A1500000BF0837BD4680BD80B483B000AF7860D3
:10A160007B681B6818460C37BD465DF8047B70475A
:10A1700080B582B000AF786039607B681B68194693
:10A18000386800F05CF87B683A681A6000BF0837EE
:10A19000BD4680BD80B584B000AFF860B9607A601C
:10A1A000786800F09AF803461946B86800F047F856
:10A1B000B968786800F043F800BF1037BD4680BD2D
:10A1C00080B483B000AF78607B681B6818460C379A
:10A1D000BD465DF8047B704780B584B000AF786001
:10A1E0007B681B68FB607B681B68002B07D07B6863
:10A1F0001B68184600F071F802467B681A60FB681D
:10A2000018461037BD4680BD80B584B000AF786079
:10A21000396007F108031A463968786800F069F870
:10A220000346FB73FB7B002B04D1BB68194678689F
:10A2300000F073F8FB7B18461037BD4680BD80B434
:10A2400083B000AF786039607B683A689A6000BF7D
:10A250000C37BD465DF8047B704780B483B000AF17
:10A2600078607B681B68002B0CBF01230023DBB2E6
:10A2700018460C37BD465DF8047B704780B582B048
:10A2800000AF78607868FEF7E1FB03461846FFF7F9
:10A290001AFD034618460837BD4680BD80B582B01A
:10A2A00000AF786039607B683968184600F056F86E
:10A2B0007B6818460837BD4680BD80B582B000AFC8
:10A2C00078607B681B68184600F007F802467B68D8
:10A2D0001A6000BF0837BD4680BD80B483B000AFB0
:10A2E00078607B689B6818460C37BD465DF8047B38
:10A2F000704780B584B000AFF860B9607A60F868E4
:10A3000000F03BF803467A68B968184600F040F858
:10A31000034618461037BD4680BD80B584B000AFF7
:10A32000786039603B68002B04D17868FFF754FFF0
:10A33000F8600EE03868FFF7D0FFF860FB68002B8C
:10A3400007D0F868FFF7C9FF034619463868FFF7DA
:10A3500076FFFB6818461037BD4680BD80B483B0D9
:10A3600000AF786039607B683A681A607B6818468D
:10A370000C37BD465DF8047B704780B483B000AFF6
:10A3800078607B6818460C37BD465DF8047B7047E3
:10A3900080B586B000AFF860B9607A601723FB75AE
:10A3A0007B6800221A60FB681B683B613B69002BDD
:10A3B0000ED03A69BB689A4202D10023FB7507E0D0
:10A3C0007B683A691A60386900F007F83861EDE790
:10A3D000FB7D18461837BD4680BD80B483B000AF02
:10A3E00078607B689B6818460C37BD465DF8047B37
:10A3F000704780B483B000AF0346FB7100BF0C37D9
:10A40000BD465DF8047B704780B582B000AF7860D0
:10A41000786800F009F80346184600F05BFA7B689C
:10A4200018460837BD4680BD80B483B000AF786061
:10A430007B6818460C37BD465DF8047B704780B5D5
:10A4400082B000AF7860396039687868F6F7D2FF7B
:10A450007B680B221A707B684FF6FF725A807B680C
:10A4600000225A607B6800229A607B680022DA60D2
:10A470007B6810333968184601F0EEFA786800F00E
:10A4800005F87B6818460837BD4680BD80B582B0A8
:10A4900000AF78607B680022DA607B6800229A60F7
:10A4A0007B6800225A607B680B221A707B684FF62B
:10A4B000FF725A807B6800225A607B68103318460E
:10A4C00001F014FB00BF0837BD4680BD80B584B0E5
:10A4D00000AF786039600023FB733B68002B14BF2A
:10A4E00001230023BB73BB7B002B0FD07B68103391
:10A4F000184601F0AEFB0346FB73FB7B002B14BF39
:10A5000001230023DBB2002B09D00BE07B68103362
:10A51000184601F0DDFB03461846FFF76AFF7B682B
:10A520003A685A60FB7B18461037BD4680BD80B53F
:10A5300084B000AF78600B467B800023FB737868A3
:10A54000FEF7F6FB034683F00103DBB2002B02D0DB
:10A550000D23FB7309E07B6810337A881146184697
:10A5600001F02CFB7B687A885A80FB7B18461037F9
:10A57000BD4680BD80B584B000AF78600B46FB70EF
:10A580000023FB737868FEF7D3FB034683F00103D7
:10A59000DBB2002B02D00D23FB7302E07B68FA785C
:10A5A0001A70FB7B18461037BD4680BD80B584B05D
:10A5B00000AF786039600023FB737868FEF7B8FB62
:10A5C000034683F00103DBB2002B02D00D23FB73A3
:10A5D00005E07B6810333968184601F019FBFB7BF6
:10A5E00018461037BD4680BD80B584B000AF786096
:10A5F0000B467B800023FB737868FEF799FB0346CC
:10A6000083F00103DBB2002B02D00D23FB7306E0C5
:10A610007B6810337A881146184601F0E2FAFB7B1A
:10A6200018461037BD4680BD80B584B000AF786055
:10A630000023FB737868FEF77BFB034683F001037E
:10A64000DBB2002B02D00D23FB7312E07B6803F119
:10A6500010027B681B781946104601F071FB034617
:10A66000FB73FB7B002B14BF01230023DBB2002B09
:10A6700000BFFB7B18461037BD4680BD90B585B046
:10A6800000AFF860B9601346FB71FB685B68002B94
:10A690000BD0FB79002B08D1FB685C68F868FEF7EB
:10A6A000D5F9FB791A46B968A04700BF1437BD46F3
:10A6B00090BD80B584B000AF786039600023FB7333
:10A6C0007868FEF735FB034683F00103DBB2002B0D
:10A6D00002D00D23FB7313E07B681033184601F0A2
:10A6E0008FFB0346FB73FB7B002B14BF012300236E
:10A6F000DBB2002B03D17B683A689A6000E000BFB0
:10A70000FB7B18461037BD4680BD90B585B000AFC5
:10A71000F860B9607A60FB70FB689B68002B0BD017
:10A72000FB689C68F868FEF791F9B968FB787A686D
:10A73000A047FB6800229A6000BF1437BD4690BD59
:10A7400080B586B000AFF8607B600B46FB721346A5
:10A750003B810023FB75F868FEF7EAFA034683F0B5
:10A760000103DBB2002B02D00D23FB7515E0FB6863
:10A7700010333A89F97A184601F0A6FE0346FB75B4
:10A78000FB7D002B14BF01230023DBB2002B03D180
:10A79000FB687A68DA6000E000BFFB7D1846183776
:10A7A000BD4680BD90B583B000AF78600B46FB70AE
:10A7B0007868FEF7BDFA0346002B05D07B68DB689E
:10A7C000002B01D0012300E00023002B0DD07B687B
:10A7D000DC687868FEF73AF9024697F903301946C3
:10A7E0001046A0477B680022DA6000BF0C37BD46E8
:10A7F00090BD90B595B002AFF8607B600B46FB72E0
:10A800001346BB72002387F8473007F1340318461C
:10A81000FFF7FAFD07F124031846FFF7F5FD07F1EE
:10A8200014031846FFF7F0FDF868FEF781FA0346B7
:10A8300083F00103DBB2002B03D00D2387F84730F0
:10A8400024E007F1340300227968184600F0FEFE88
:10A8500007F124030022B96D184600F0F7FE07F156
:10A8600014030022F96D184600F0F0FEFB6803F1B6
:10A87000100007F13404BA7AF97A07F1140301934E
:10A8800007F124030093234601F0DCFF97F84730DB
:10A8900018464C37BD4690BD80B584B000AF786097
:10A8A00039600023FB737868FEF742FA034683F0B1
:10A8B0000103DBB2002B02D00D23FB7305E07B68A4
:10A8C00010333968184602F020F8FB7B1846103721
:10A8D000BD4680BD80B582B000AF786010220021F7
:10A8E000786817F0ADFB00BF0837BD4680BD80B467
:10A8F00083B000AF0346FB80FB8818460C37BD468B
:10A900005DF8047B704780B483B000AF78607B68EB
:10A910001B781AB27B6801331B781B021BB21343EE
:10A920001BB29BB218460C37BD465DF8047B7047DE
:10A9300080B483B000AF78607B681B781A467B6870
:10A9400001331B781B021A437B6802331B781B04FC
:10A950001A437B6803331B781B06134318460C37D6
:10A96000BD465DF8047B704780B483B000AF78606B
:10A9700039607B68DAB23B681A707B681A0A3B68F8
:10A980000133D2B21A707B681A0C3B680233D2B220
:10A990001A707B681A0E3B680333D2B21A7000BF7C
:10A9A0000C37BD465DF8047B704780B582B000AFC0
:10A9B00078607B681B889BB21846FFF798FF0346B8
:10A9C000DB119BB2DBB29BB218460837BD4680BD97
:10A9D00080B483B000AF78607B681B7803F07F039E
:10A9E000DBB218460C37BD465DF8047B704780B576
:10A9F00082B000AF7860786800F09AF8034603F4FC
:10AA00000073002B14BF01230023DBB21846083764
:10AA1000BD4680BD80B483B000AF78607B681B68A2
:10AA200018460C37BD465DF8047B704780B582B090
:10AA300000AF78607868FFF7EDFF034618460837E7
:10AA4000BD4680BD80B582B000AF7860786800F008
:10AA500071FD0346184600F058FC0346184600F006
:10AA600074FD034618460837BD4680BD80B582B0E8
:10AA700000AF7860786800F05DFD0346184600F08E
:10AA80005DFC0346184600F060FD03461846083793
:10AA9000BD4680BD80B483B000AF78600223184605
:10AAA0000C37BD465DF8047B704780B483B000AFBF
:10AAB0000346FB80FB8803F44063002B14BF012393
:10AAC0000023DBB218460C37BD465DF8047B7047A7
:10AAD00080B483B000AF78607B689B6818460C3701
:10AAE000BD465DF8047B704780B483B000AF7860EA
:10AAF0000B46FB707A68937EF97861F304139376C2
:10AB000000BF0C37BD465DF8047B704780B483B04E
:10AB100000AF78600B46FB707A68937EF97861F33A
:10AB20000003937600BF0C37BD465DF8047B704789
:10AB300080B582B000AF78607B681B681846FFF76D
:10AB4000E2FE034618460837BD4680BD80B584B096
:10AB500000AF0346FB800123FB73FB881846FDF71B
:10AB60004AF90346002B35D0FA884CF6404313408F
:10AB70004CF6404293422AD04CF64042934230DC9D
:10AB80004CF24002934222D04CF24002934228DC25
:10AB9000B3F5404F1BD0B3F5404F22DC48F24002E2
:10ABA000934214D048F2400293421ADCB3F5004FAE
:10ABB0000DD0B3F5004F14DCB3F5446F07D0B3F5F7
:10ABC000446F0EDC002B02D0B3F5046F09D10023D3
:10ABD000FB7307E0FB881846FFF767FF0346FB732C
:10ABE00000E000BFFB7B18461037BD4680BD80B536
:10ABF00084B000AF0346FB800023FB73FB8803F4A3
:10AC00004043002B21D0FB8803F04003002B1CD1D4
:10AC1000FB881846FDF7EFF8034683F00103DBB22B
:10AC2000002B0BD1FB8803F44063B3F5406F05D1D3
:10AC3000FB8803F44043B3F5404F01D0012300E00B
:10AC40000023002B01D00123FB73FB7B1846103738
:10AC5000BD4680BD80B584B000AF78607B689B88BE
:10AC6000022B02D8FF23FB7310E07868F9F75EFB34
:10AC7000034683F00103DBB2002B02D0FF23FB73FA
:10AC800004E0786800F058FA0346FB73FB7B184633
:10AC90001037BD4680BD80B584B000AF78603960A4
:10ACA0000023FB737868FFF7D5FF0346BB73BB7BBC
:10ACB000FF2B02D10623FB7309E07B681A68BB7B7C
:10ACC00013441B7803F00703DAB23B681A70FB7B6E
:10ACD00018461037BD4680BD80B584B000AF78609F
:10ACE00039600023FB737868FFF7B4FF0346BB733A
:10ACF000BB7BFF2B02D10623FB7309E07B681A683C
:10AD0000BB7B13441B7803F01803DAB23B681A705C
:10AD1000FB7B18461037BD4680BD80B584B000AFC0
:10AD2000786039600023FB737868FFF793FF034670
:10AD3000BB73BB7BFF2B02D10623FB730CE0BB7BF9
:10AD40000133BB737B681A68BB7B13441846FFF75B
:10AD5000EFFD02463B681A60FB7B18461037BD4684
:10AD600080BD80B584B000AF786039607868FFF747
:10AD700071FF0346FB73FB7BFF2B00D1FEE7FB7BE0
:10AD80000133FB737B681A68FB7B134419463868F0
:10AD9000FFF7EAFD01217868FFF7B8FE00BF103722
:10ADA000BD4680BD80B485B000AF0346FB71002373
:10ADB000FB73FB79182B41D801A252F823F000BF96
:10ADC00025AE00003DAE00003DAE00003DAE0000EF
:10ADD0003DAE00003DAE00003DAE00003DAE0000C7
:10ADE0002BAE00003DAE00003DAE00003DAE0000C9
:10ADF0003DAE00003DAE00003DAE00003DAE0000A7
:10AE000031AE00003DAE00003DAE00003DAE0000A2
:10AE10003DAE00003DAE00003DAE00003DAE000086
:10AE200037AE00000023FB7308E00023FB7305E04E
:10AE30000423FB7302E00823FB7300BFFB7B18466F
:10AE40001437BD465DF8047B704700BF80B584B001
:10AE500000AF786039600023FB737868FFF7FAFE73
:10AE60000346BB73BB7BFF2B02D10623FB7316E0AB
:10AE70007B681A68BB7B13441B7803F01803DBB2B2
:10AE80001846FFF78FFF03467B737B681B68BA7B0E
:10AE9000511D7A7B0A4413441A783B681A70FB7B75
:10AEA00018461037BD4680BD80B584B000AF7860CD
:10AEB0000B46FB707868FFF7CDFE0346FB73FB7B08
:10AEC000FF2B00D1FEE77B681A68FB7B13441B78DD
:10AED00003F01803DBB21846FFF764FF0346BB73A9
:10AEE0007B681B68FA7B511DBA7B0A441344FA78CD
:10AEF0001A7000BF1037BD4680BD80B582B000AF6C
:10AF00007860786800F001FA02467B681B68D31A03
:10AF1000DBB218460837BD4680BD80B584B000AFAF
:10AF200078607868FFF7B6FD0346FB737868FFF733
:10AF300091FE0346BB73BB7BFF2B0DD07B681A6869
:10AF4000BB7B13441B78184600F00CF803461A46E6
:10AF5000FB7B1344FB7300E000BFFB7B18461037FC
:10AF6000BD4680BD80B485B000AF0346FB710023B1
:10AF7000FB73FB7903F00703072B1FD801A252F8DC
:10AF800023F000BFA5AF0000ABAF0000B1AF0000E1
:10AF9000B7AF0000A5AF0000ABAF0000B1AF00003D
:10AFA000B7AF00000023FB7308E00423FB7305E048
:10AFB0000823FB7302E01023FB7300BFFB7B1846E2
:10AFC0001437BD465DF8047B704700BFB0B582B052
:10AFD00000AF78607B689C887868FFF78EFF034637
:10AFE0009DB27868FFF799FF03469BB22B449BB252
:10AFF000E31A9BB218460837BD46B0BD80B584B091
:10B0000000AF7860786800F097F80346FB73FB7B2D
:10B01000FF2B2BD07868F9F789F90346002B27D04E
:10B02000FB7B7A689288934202DBFF23FB7320E06C
:10B030007B681A68FB7B13441B78BB73BB7B184689
:10B0400000F01CF803467B737B7BFF2B02D1FF23B0
:10B05000FB730EE0FA7B7B7B1344FB73FB7B7A680C
:10B060009288934205DDFF23FB7302E000BF00E0FE
:10B0700000BFFB7B18461037BD4680BD80B485B04D
:10B0800000AF0346FB710523FB73FB7903F0070355
:10B09000002B02D1FF23FB7346E0FB7903F018037A
:10B0A000182B41D801A252F823F000BF29B10000AB
:10B0B00029B1000029B1000029B1000029B1000028
:10B0C00029B1000029B1000029B1000011B1000030
:10B0D00029B1000029B1000029B1000029B1000008
:10B0E00029B1000029B1000029B1000019B1000008
:10B0F00029B1000029B1000029B1000029B10000E8
:10B1000029B1000029B1000029B1000021B10000DF
:10B11000FB7B0133FB7307E0FB7B0533FB7303E031
:10B12000FB7B0933FB7300BFFB7B18461437BD461E
:10B130005DF8047B704700BF80B584B000AF7860D5
:10B140007868FFF7A7FC034602337A689288934237
:10B15000ACBF01230023DBB2002B02D0FF23FB7323
:10B1600008E07868FFF7E4FC0346184600F007F8AB
:10B170000346FB73FB7B18461037BD4680BD80B588
:10B1800084B000AF0346FB800323FB73FB881846A3
:10B19000FFF7DCFC0346002B02D0FB7B0233FB7382
:10B1A000FB8803F44063B3F5406F0BD0B3F5406FF9
:10B1B0000CDC002B0DD0B3F5006F07D1FB7B023305
:10B1C000FB7307E0FB7B0833FB7303E0FF23FB7398
:10B1D00024E000BFFB881846FFF709FD0346002B5B
:10B1E00002D0FB7B0233FB73FB8803F44043B3F5CF
:10B1F000404F0BD0B3F5404F0CDC002B0DD0B3F516
:10B20000004F07D1FB7B0233FB7307E0FB7B083366
:10B21000FB7303E0FF23FB7300E000BFFB7B1846DA
:10B220001037BD4680BD80B584B000AF78607868C7
:10B23000FFF7E4FE0346FB81FB89FF2B5CD07868B7
:10B24000FFF7D5FB0346002B3CD07868FFF765FE7F
:10B2500003467B737B681A68FB891344BB60FB89D8
:10B260000233FB81FA897B7B13447A68928893428C
:10B2700002DDFF23FB8142E0B868FFF7A9FB03462C
:10B280009AB2FB891344FB81FA897B7B13447A6869
:10B290009288934202DDFF23FB8130E0B868FFF71C
:10B2A00084FB03467F2B0CBF01230023DBB2002B62
:10B2B00007D1FA897B7B13447A689288934201DA3A
:10B2C000C8E700BF7868FCF772FD034683F001030E
:10B2D000DBB2002B09D07868FFF72AFC034603F0A5
:10B2E0000703032B01D1012300E00023002B05D02D
:10B2F000FB890133FB8102E000BF00E000BFFB8956
:10B30000DBB218461037BD4680BD80B584B000AFB3
:10B3100078607868FFF787FF0346FB72FB7AFF2BA4
:10B3200002D10023FB6004E07B681A68FB7A1344B7
:10B33000FB60FB6818461037BD4680BDB0B582B0D3
:10B3400000AF78607B681C687B689B881D467868C6
:10B35000FFF7E3FD0346EB1A234418460837BD46C2
:10B36000B0BD80B582B000AF78607B68184602F04F
:10B37000A1F87B6818460837BD4680BD80B582B00D
:10B3800000AF78607B68184602F0E4F87B681846E6
:10B390000837BD4680BDB0B5E4B002AF3B1D1860B4
:10B3A0003B4619600023C7F8803107F108031846AF
:10B3B000FFF7D7FF3B1D1B681846F8F7B7FF03469A
:10B3C00083F00103DBB2002B40F0A4803B1D1B681F
:10B3D00007F27F1211461846FFF75DFC0346002B6B
:10B3E00014BF01230023DBB2002B40F095803B1DEE
:10B3F0001B6807F5C07211461846FFF78EFC03461E
:10B40000002B14BF01230023DBB2002B40F0868009
:10B41000D7F8801197F87F2107F5B8733846006890
:10B4200002F029F83B1D1868FFF752FB024607F1AE
:10B4300008031146184601F000FD3B1D1B68184625
:10B44000FFF76BFD03461C463B1D1B681846FFF7C4
:10B4500021FB0346E31A87F887313B1D1B6818461A
:10B46000FFF74BFD03461C463B1D1B681846FFF7C4
:10B47000ADFD0346194697F8872107F108000D2313
:10B48000019307F5B873009313460A46214601F06D
:10B49000E9FC3B1D1B681846FFF7C8FA04463B1D34
:10B4A0001B681846FFF729FD03461A4607F10803F3
:10B4B0002146184601F03DFE3B1D1B681846FFF76C
:10B4C000C1FA04463B1D1B681846FFF7BBFA054648
:10B4D0003B1D1B681846FFF779FD03461A4607F126
:10B4E00008000023009313462A46214601F091FEEE
:10B4F0003B1D1B681846FFF7B9FA024607F108031F
:10B500001146184601F07AFF3B1D01211868FFF72C
:10B51000EBFA04E000BF02E000BF00E000BF00BFA4
:10B5200007F108031846FFF729FF00BF07F5C477A6
:10B53000BD46B0BD80B483B000AF78607B6818466C
:10B540000C37BD465DF8047B704780B483B000AF14
:10B5500078607B6818460C37BD465DF8047B704701
:10B5600080B485B000AFF860B9601346FB80FB681B
:10B57000BA681A60FB68FA889A8000BF1437BD4623
:10B580005DF8047B704780B483B000AF78607B685F
:10B5900018460C37BD465DF8047B704780B483B015
:10B5A00000AF78607B6818460C37BD465DF8047BB9
:10B5B000704790B482B000AF786039607A683B68B9
:10B5C0001446186859689A68DB680FC400BF0837CA
:10B5D000BD4690BC704780B586B000AFF860B960DA
:10B5E0001346FB71FB79002B02D0012B06D01AE029
:10B5F0000822B968F86816F0FBFC14E0BB68073352
:10B60000BB600823FB75FB7D002B0BD0BA68531E73
:10B61000BB60FB68591CF96012781A70FB7D013B16
:10B62000FB75F0E700BF00BF1837BD4680BD80B591
:10B6300082B000AF78607868FEF7F6FE03461846E1
:10B64000FFF748F900BF0837BD4680BD80B584B01C
:10B6500000AFF860B9601346FB71B968F868FFF78E
:10B66000A8FF00BF1037BD4680BD80B582B000AFD7
:10B67000786039607868FFF791FF03461846FFF756
:10B6800082FF0346102219463868FFF769FF00BFA2
:10B690000837BD4680BD80B584B000AF78603960A2
:10B6A0007B681A683B68D21A07F10C0311461846EA
:10B6B000FEF7F4F9FB6818461037BD4680BD80B52B
:10B6C00084B000AFF860B9607A60B968F868F5F7DF
:10B6D00091FEFB687A681A60FB68FA689A60FB68FA
:10B6E00018461037BD4680BD80B584B000AFF86005
:10B6F000B9607A60FB687A68B9681846FFF7DFFFBF
:10B70000FB6818461037BD4680BD80B483B000AFDB
:10B710000346FB7100BF0C37BD465DF8047B7047E4
:10B7200080B483B000AF78607B689B7918460C3793
:10B73000BD465DF8047B704780B483B000AF78608D
:10B740007B681B7E18460C37BD465DF8047B70474E
:10B7500080B483B000AF78607B685B7E18460C379E
:10B76000BD465DF8047B704780B483B000AF78605D
:10B770000B46FB707A68937EF97861F34103937608
:10B7800000BF0C37BD465DF8047B704780B483B0C2
:10B7900000AF78607B689B7EC3F38003DBB2184602
:10B7A0000C37BD465DF8047B704780B483B000AFB2
:10B7B000786039603A687B689A6000BF0C37BD4694
:10B7C0005DF8047B704780B483B000AF78607B681D
:10B7D0009B7EC3F30013DBB218460C37BD465DF801
:10B7E000047B704780B582B000AF786039607868BC
:10B7F000FDF73AF9034639681846FCF7FDF800BF33
:10B800000837BD4680BD80B582B000AF78607868EB
:10B81000FDF72AF903461846FBF79AFB034618463C
:10B820000837BD4680BD80B582B000AF78600B465A
:10B830007B807868FDF718F902467B881946104628
:10B84000FBF795F900BF0837BD4680BDF0B58BB05A
:10B8500004AFF8607B600B46FB721346BB7200239B
:10B86000FB75F868FDF700F906467D683B6B7A6B5F
:10B87000BC7AF87AF97D0291019200932B46224618
:10B8800001463046FCF764F800BF1C37BD46F0BDEA
:10B8900080B582B000AF78607868FDF7E5F80346C0
:10B8A0001846FBF71DFA034618460837BD4680BD0B
:10B8B00080B582B000AF78607868FDF7D5F80346B0
:10B8C0001846FBF72BFA034618460837BD4680BDDD
:10B8D00080B582B000AF78600B46FB707868FDF7EA
:10B8E000C3F80246FB7819461046FBF75DFA03469B
:10B8F00018460837BD4680BD80B582B000AF78607D
:10B900007868FDF7B1F803461846FBF703FB0346DA
:10B9100018460837BD4680BD80B582B000AF78605C
:10B920000B46FB7013463B807868FDF79DF83A881C
:10B93000FB781946FBF7C2FB034618460837BD469D
:10B9400080BD80B483B000AF78607B683433184624
:10B950000C37BD465DF8047B704780B483B000AF00
:10B9600078607B685B6D18460C37BD465DF8047BDC
:10B97000704780B483B000AF78607B681B7803F0B9
:10B980000C03002B14BF01230023DBB218460C3735
:10B99000BD465DF8047B704780B483B000AF78602B
:10B9A0007B681B7803F02003002B14BF01230023C6
:10B9B000DBB218460C37BD465DF8047B704780B497
:10B9C00083B000AF78607B681B7803F00403002B22
:10B9D00014BF01230023DBB218460C37BD465DF8C7
:10B9E000047B704780B483B000AF78607B681B78BD
:10B9F00003F00103002B14BF01230023DBB2184620
:10BA00000C37BD465DF8047B704780B483B000AF4F
:10BA100078607B681B7803F00203002B14BF0123BE
:10BA20000023DBB218460C37BD465DF8047B704737
:10BA300080B483B000AF78607B681B7803F040036C
:10BA4000002B14BF01230023DBB218460C37BD4680
:10BA50005DF8047B7047000080B582B000AF78606D
:10BA6000396039687868F5F7C5FC786800F069FFD7
:10BA700003461846FFF7C7FE03461A467B681A704E
:10BA8000786800F05EFF03461846FFF735FF024670
:10BA90007B685A617B6818333968184600F08BFF61
:10BAA0007B680022DA617B6800221A627B6824339B
:10BAB0001846FEF7A9FC7B6834331846FEF7A4FC51
:10BAC0007B6844331846FEF79FFC7B685C33064A6C
:10BAD00039681846FFF708FE786800F007F87B68B9
:10BAE00018460837BD4680BD69C6000080B584B0E1
:10BAF00000AF78607B6800225A707B6800229A70E1
:10BB00007B680022DA707B684FF6FE729A807B6851
:10BB10000633184600F025FF7A68937B43F0010353
:10BB200093737B687F22DA7307F10C0300211846B8
:10BB3000FDF7B4FF7B68FA681A617B68002283F81E
:10BB400059207B6824331846FFF771FD7B68343336
:10BB50001846FFF76CFD7B6844331846FFF767FD16
:10BB60007B6800225A657B68002283F858207B6836
:10BB70005C331846FEF771FA00BF1037BD4680BD32
:10BB800080B485B000AF78607B681B78FB73FB7B6B
:10BB900043F00403FB73FB7B43F02003FB73FB7B4D
:10BBA00043F04003FB73FB7B63F07F03FB73FB7B82
:10BBB00018461437BD465DF8047B704780B582B0E7
:10BBC00000AF78600B467B80786800F0BAFE0246D2
:10BBD0007B8819461046FFF726FE00BF0837BD4692
:10BBE00080BD80B582B000AF78600B467B807B68FB
:10BBF0007A889A80786800F0A4FE02467B689B8869
:10BC00001946104600F0ECFF00BF0837BD4680BD66
:10BC100080B584B000AF786039607B683A680633DD
:10BC20001168526819605A60396807F108030122E7
:10BC30001846FCF786FF786800F083FE024607F19D
:10BC400008031946104600F0B9FF00BF1037BD4683
:10BC500080BD80B584B000AF78600023FB737B6843
:10BC60005B78002B26D1786800F06BFE03461846FF
:10BC7000FFF70EFE0346FB73FB7B002B14BF012373
:10BC80000023DBB2002B17D1786800F05AFE034680
:10BC90001846FCF78AFF0346FB73FB7B002B14BF9F
:10BCA00001230023DBB2002B08D10121786800F0CA
:10BCB000B5FD04E000BF02E000BF00E000BFFB7B79
:10BCC000002B00D0FEE7FB7B18461037BD4680BD39
:10BCD00080B584B000AF78607B685C331846FEF7AF
:10BCE000BCF9786800F02DFE03461846FCF75DFFAE
:10BCF0000346FB73FB7B002B14BF01230023DBB245
:10BD0000002B15D1786800F01CFE03461846FFF79B
:10BD1000CFFD0346FB73FB7B002B14BF01230023E5
:10BD2000DBB2002B06D10021786800F077FD02E03D
:10BD300000BF00E000BFFB7B18461037BD4680BD4A
:10BD400080B584B000AF78600B46FB70786800F077
:10BD5000F8FD0246FB7819461046FFF7B9FD034689
:10BD6000FB73FB7B002B04D10221786800F056FDA9
:10BD700000E000BFFB7B18461037BD4680BD80B594
:10BD800084B000AFF860B9601346FB71FB68DB69F3
:10BD9000002B0CD0BB68002B09D0FB79002B06D1FF
:10BDA000FB68DB69FA68126A0021B8689847F8688E
:10BDB00000F0B0FC034683F00103DBB2002B0BD094
:10BDC000BB68002B08D0BB68DB7DC3F34003DBB24C
:10BDD000002B01D0012300E00023002B05D0BB681D
:10BDE0001B691946F86800F076FDFB681833FA798C
:10BDF000B968184600F0EDFD00BF1037BD4680BDA4
:10BE000080B584B000AF78600023FB737B685B78FB
:10BE1000072B0CDC032B07DA002B05D0002B06DBED
:10BE2000013B012B03D802E00D23FB730FE0786880
:10BE300000F012F87B6800229A707B680022DA70AA
:10BE40007B68002283F85920786800F08BF8FB7B30
:10BE500018461037BD4680BD90B587B000AF7860FA
:10BE600000237B617B685B691846F8F75FFA03463D
:10BE700083F00103DBB2002B67D17B685B69184656
:10BE8000FFF7A1FC0346002B61D17B685B691A4672
:10BE900007F10F0319461046FEF71EFF0346002B5D
:10BEA00014BF01230023DBB2002B52D17B685B69F6
:10BEB0001846F8F76FFA034683F00103DBB2002B54
:10BEC00009D07B685B691A467B6893F8583019463D
:10BED0001046FEF7E9FF786800F01CFC034683F08B
:10BEE0000103DBB2002B36D1FB7B082B35D17B68FD
:10BEF0005C697868FFF725FD034619462046FFF781
:10BF000054FC7B685B691846F8F744FA034683F0F3
:10BF10000103DBB2002B0DD07868FFF71EFD3861FE
:10BF20007B685B6939691846FEF71BFF39697868D9
:10BF300000F0D1FC7868FCF7E3FE78617B685B6910
:10BF400079691846FFF727FA08E000BF06E000BF4E
:10BF500004E000BF02E000BF00E000BF00BF1C37EC
:10BF6000BD4690BD90B589B000AF78607B689B7886
:10BF70000333FB777B685B691B69002B62D0072169
:10BF8000786800F04BFC786800F032FC0346002B28
:10BF900054D07868FCF75AFD03461846FBF7CBFCF3
:10BFA00002460B4607F1080311461846FDF776FDD9
:10BFB0007B685B695A6907F1140311461846FDF75F
:10BFC0006DFD7B685B691A6907F114031146184619
:10BFD000FDF79CFD03463B6107F1100380211846E5
:10BFE000FFF759FB0346FB6007F10C0207F108035A
:10BFF00011461846FDF79EFD0346002B1AD07B68BC
:10C0000003F15C047B685B695A6907F11803114608
:10C010001846FDF743FD07F1180380211846FFF786
:10C020003AFB01467B685B691B691A462046FDF7AF
:10C03000E7FF22E0786800F068F81EE0786800F01A
:10C0400064F81AE00321786800F0E8FB786800F0F3
:10C0500077FB034683F00103DBB2002B03D0786843
:10C0600000F053F809E0FB7F052B01D90523FB778E
:10C07000FB7F1946786800F004F800BF2437BD46FE
:10C0800090BD90B585B000AF78600B46FB70FB7833
:10C09000012202FA03F319460020FDF74FFCF86075
:10C0A000FA6813469B0013449B01FB607B689B7BF3
:10C0B000C3F30003DBB2002B12D0786800F041FC20
:10C0C00004467B685B691846FFF72AFB034619465E
:10C0D0002046FFF7FDFB03461846FFF716FB0AE074
:10C0E000786800F02EFC03461846FCF75EFD034618
:10C0F0001846FFF70AFB7B685C33F9681846FDF7C2
:10C100006EFF00BF1437BD4690BD90B585B000AF3F
:10C1100078607B685B78032B03D07B685B78072BA8
:10C1200059D17B681B7803F01003002B16D1786877
:10C1300000F007FC04467B685B691846FFF7F0FADD
:10C14000034619462046FFF7C3FB0346002B14BFE6
:10C1500001230023DBB2002B00D0FEE70421786826
:10C1600000F05CFB7B68DB69002B08D07B68DB6937
:10C170007A68526910467A68126A0121984778688D
:10C1800000F0DFFB02467B685B691946104600F051
:10C190003AFD0346FB73FB7B0D2B18D17B685B6973
:10C1A0001B69002B13D07B685B6900221A617B68D6
:10C1B0005B6900225A61786800F0C3FB02467B6825
:10C1C0005B691946104600F01EFD0346FB73FB7BBE
:10C1D000002B02D0FEE700BF00E000BF00BF143715
:10C1E000BD4690BD80B582B000AF78603960786898
:10C1F00000F0BCFA0346002B08D03B681846FBF75A
:10C20000E6FD0346002B01D0012300E00023002BB4
:10C2100006D07B685C334FF47A511846FDF7DFFE99
:10C2200000BF0837BD4680BD90B589B002AFF86049
:10C23000B9607A60FB700123FB75FB685C331846BC
:10C24000FDF70BFFFB780F2B39D801A252F823F032
:10C2500095C20000BFC20000BFC20000BFC2000004
:10C26000BFC20000BFC20000BFC20000BFC20000CA
:10C27000BFC20000BFC20000BFC20000C1C20000B8
:10C28000BFC20000BFC2000095C2000091C2000002
:10C290000023FB75B868FFF779FA0346002B11D02D
:10C2A000FB6803F11804BB681846FFF739FA034628
:10C2B0001A46FB7D1946204600F09EFB02E0FEE791
:10C2C00000BF00E000BFB968F86800F085F8FB7DAA
:10C2D00083F00103DBB2002B0FD0F86800F030FAD6
:10C2E0000346002B09D0FB689C78B868FFF724FA56
:10C2F00003469C4201D2012300E00023002B09D019
:10C30000FB689B780133DAB2FB689A70F868FFF734
:10C3100029FE5DE0FB6800229A70FB78002B0FD0AD
:10C32000F86800F039FA0346002B09D0FB68DC7886
:10C33000B868FFF70DFA03469C4201D2012300E0E2
:10C340000023BB75FB6803F11800FB68DB78F97804
:10C35000BA7D019200930B467A68B96800F05AFBE7
:10C36000BB7D002B28D0FB68DB780133DAB2FB6899
:10C37000DA700121B868FFF7F7F9FB780E2B17D1B7
:10C380000621F86800F04AFAFB6893F8593019461C
:10C39000F868FFF776FEFB6893F85930042B28BF46
:10C3A0000423DBB20133DAB2FB6883F859200FE0D3
:10C3B000F868FFF7D7FD0BE00221F86800F02EFACD
:10C3C000FB6803F11800FB787A68B96800F03AFB63
:10C3D00000BF1C37BD4690BD80B584B000AF78600B
:10C3E00039600023FB73786800F094F90346002B52
:10C3F00012D13B681846F7F799FF034683F0010313
:10C40000DBB2002B08D13868F7F7C4FF034683F08E
:10C410000103DBB2002B01D0012300E00023002B3D
:10C4200034D13B6807F10E0211461846FEF754FC62
:10C430000346002B14BF01230023DBB2002B06D0E0
:10C44000FB7B83F00103DBB2002B21D0FEE7BB7B3B
:10C45000082B1FD13B6807F1080211461846FEF76A
:10C460005CFC0346002B14BF01230023DBB2002B2E
:10C4700006D0FB7B83F00103DBB2002B0CD0FEE780
:10C48000BB681946786800F026FA06E000BF04E0B1
:10C4900000BF02E000BF00E000BF00BF1037BD4694
:10C4A00080BD80B584B000AF7860786800F049FA4C
:10C4B00003461846FCF789FB0346FB7397F90F30D8
:10C4C00018461037BD4680BD90B585B000AF786086
:10C4D0000B46FB7013463B800023FB737B685B7845
:10C4E000072B0CDC032B07DA002B05D0002B06DB17
:10C4F000013B012B03D802E00D23FB734BE078686E
:10C50000FFF783FA0346002B10D0786800F019FA81
:10C510003A88FB781946FFF7FFF903461846FFF7FC
:10C52000F4F80521786800F079F934E0786800F0D3
:10C5300049F90346002B2CD0786800F002FA024635
:10C54000FB7819461046FFF7C3F90346002B14BFCA
:10C5500001230023DBB2002B00D0FEE70521786821
:10C5600000F05CF97B687F22DA73FDF741FB03463C
:10C57000BB603A887C6807F1080311461846FDF74E
:10C58000C5FA20617B685C3300211846FDF727FD62
:10C5900001E00C23FB73FB7B18461437BD4690BDAE
:10C5A00090B585B000AF78607868FFF72EFA034643
:10C5B000002B00D0FEE77868FFF773FF0346FB739C
:10C5C00097F90F307F2B0ED07B6893F90F307F2BBC
:10C5D00006D07B6893F90F3097F90F209A4202DD5D
:10C5E0007B68FA7BDA73FDF703FB0346BB607B686D
:10C5F00003F1100207F1080311461846FDF79AFAF5
:10C600000346002B0FD07B6803F15C047B685C332E
:10C610001846FDF7B2FA03464FF4FA32194620469F
:10C62000FDF7EEFC06E07B6893F90F301946786859
:10C6300000F004F800BF1437BD4690BD80B582B04D
:10C6400000AF78600B46FB700221786800F0E6F8D6
:10C650007B68183397F903201146184600F005FA55
:10C6600000BF0837BD4680BD80B582B000AF78609E
:10C67000786800F083F90346184600F005F800BF1B
:10C680000837BD4680BD000090B583B000AF78602C
:10C690007B685B78033B042B36D801A252F823F069
:10C6A000BDC60000C5C6000001C70000F9C60000F5
:10C6B000B5C600007868FFF728FD26E07868FFF728
:10C6C00024FD22E0786800F03CF904467B685B6951
:10C6D0001846FFF725F8034619462046FFF7F8F8F5
:10C6E00003461846FFF711F87B6859690E230022AC
:10C6F0007868FFF799FD08E07868FFF733FC04E0FD
:10C700007868FFF74DFF00E000BF00BF0C37BD4663
:10C7100090BD00BF80B584B000AF78600123FB738B
:10C720007868FFF739F90346002B02D00023FB732A
:10C7300001E00123FB73FB7B18461037BD4680BD2B
:10C7400080B584B000AF78600123FB737868FFF791
:10C7500010F90346002B02D00023FB7301E00023F5
:10C76000FB73FB7B18461037BD4680BD80B584B097
:10C7700000AF78600123FB737868FFF733F9034655
:10C78000002B02D00023FB7301E00023FB73FB7B33
:10C7900018461037BD4680BD80B584B000AF7860C4
:10C7A0000123FB737868FFF70AF90346002B02D0D8
:10C7B0000023FB7301E00123FB73FB7B184610375A
:10C7C000BD4680BD80B584B000AF78600123FB73A7
:10C7D0007868FFF71AF90346002B02D00023FB7399
:10C7E00001E00023FB73FB7B18461037BD4680BD7C
:10C7F00080B584B000AF78600123FB737868FFF7E1
:10C8000017F90346002B02D00023FB7301E001233C
:10C81000FB73FB7B18461037BD4680BD80B483B0E8
:10C8200000AF78600B46FB707B685B78FA789A42C1
:10C8300002D07B68FA785A7000BF0C37BD465DF8AD
:10C84000047B704790B587B002AFF8607B600B4601
:10C85000FB721346BB72FB7A102B23D0102B20DC0B
:10C86000002B1FD0082B1CD1FB68BA7A83F8582004
:10C87000FB687A6803F1240413460FCB84E80F00A9
:10C88000FB683A6A03F1340413460FCB84E80F00C7
:10C89000FB687A6A03F1440413460FCB84E80F0067
:10C8A00001E0FEE700BFF868FFF734FF0346002B06
:10C8B0000CD1F86800F045F8BA7AF97A7B6A0193EE
:10C8C0003B6A00937B68FEF7C1FF00E000BF00BF3A
:10C8D0001437BD4690BD80B582B000AF7860396036
:10C8E0007B6818333968184600F0D3F87B685B6DB5
:10C8F0003A689A4204D33B685A1C7B685A6500E048
:10C9000000BF00BF0837BD4680BD80B582B000AF14
:10C91000786039607B683A685A657868FFF7FAFE94
:10C920000346002B08D1786800F00BF803463968FD
:10C930001846FEF757FF00E000BF00BF0837BD46AE
:10C9400080BD80B582B000AF78607868FCF77EF873
:10C9500003461846FCF794F8034618460837BD46C8
:10C9600080BD80B582B000AF786008220021786871
:10C9700015F066FB00BF0837BD4680BD80B582B0AC
:10C9800000AF78607868FCF761F803461846FCF75A
:10C9900041FE034618460837BD4680BD80B485B0C9
:10C9A00000AFF860B9607A60FB7000BF1437BD4615
:10C9B0005DF8047B704780B582B000AF7860396065
:10C9C00039687868F4F716FD7B6818460837BD4665
:10C9D00080BD80B584B000AFF860B9601346FB71CC
:10C9E000F86800F061F8FB791A46B968FDF746FE71
:10C9F00000BF1037BD4680BD80B483B000AF786003
:10CA00000B46FB701346BB7000BF0C37BD465DF88C
:10CA1000047B704780B586B002AFF860B9607A6079
:10CA2000FB70F86800F040F8FA783B7F01933B7E9A
:10CA3000009313467A68B968FFF7B0FF00BF10375C
:10CA4000BD4680BD80B584B000AFF860B9607A6043
:10CA5000FB70F86800F028F8FB787A68B968FDF791
:10CA600054FE00BF1037BD4680BD80B582B000AF18
:10CA700078600B46FB70786800F016F8024697F96C
:10CA8000033019461046FDF78DFE00BF0837BD463E
:10CA900080BD80B483B000AF7860396000BF0C37D0
:10CAA000BD465DF8047B704780B582B000AF78600A
:10CAB0007868FBF7CBFF03461846FCF79AF9034664
:10CAC00018460837BD4680BD80B582B000AF78609B
:10CAD0007868FBF7C9FF03461846FAF7E7F80346FC
:10CAE00018460837BD4680BD80B592B002AF786069
:10CAF00000217868FCF779F87868FCF7D7F878684F
:10CB0000FCF7E3F87868FFF7DFFF0346002B17D048
:10CB10007868FCF74AF80346002B14BF0123002372
:10CB2000DBB2002B00D0FEE77868FEF7C1FE0346BB
:10CB3000002B14BF01230023DBB2002B00D0FEE743
:10CB40004FF6FF717868FEF76EFE07F108030022CA
:10CB50001A605A6007F108031946786800F02EF849
:10CB60004FF6FE71786800F03BF807F110031846A5
:10CB7000FDF74AFC07F120031846FDF745FC07F1D5
:10CB800030031846FDF740FC07F1100207F13003AF
:10CB9000019307F1200300931346002200217868D7
:10CBA000FEF754FE00217868FEF71CFE002178682D
:10CBB000FBF7E8FF00BF4037BD4680BD80B582B0BF
:10CBC00000AF786039607868FBF74EFF02463B683B
:10CBD00019461046F9F7E2FF00BF0837BD4680BD91
:10CBE00080B582B000AF78600B467B807868FBF739
:10CBF0003BFF02467B8819461046F9F7F1FF00BF5C
:10CC00000837BD4680BD80B582B000AF786039601E
:10CC10007868FBF729FF02463B6819461046FAF789
:10CC2000EDF8034618460837BD4680BD80B483B092
:10CC300000AF78607B6893F88C3018460C37BD469F
:10CC40005DF8047B704780B483B000AF78607B6888
:10CC5000123318460C37BD465DF8047B704780B52B
:10CC600086B000AFF860B9601346FB71F868FBF757
:10CC70005DFF7861BB683B617869FFF7D7FF0346CA
:10CC800083F00103DBB2002B08D17869FFF7DBFFEB
:10CC9000FB791A46396900F069FD00E000BF00BF6A
:10CCA0001837BD4680BD80B584B000AF786039606C
:10CCB0007868FBF73BFFF8603B68BB60F868FFF7FC
:10CCC000B5FF034683F00103DBB2002B08D1F868FF
:10CCD000FFF7B9FF0346B968184600F05AFD00E0B7
:10CCE00000BF00BF1037BD4680BD80B588B000AF23
:10CCF000F860B9607A60FB70F868FBF717FFF861BD
:10CD0000BB68BB617B687B61F869FFF78FFF0346F7
:10CD100083F00103DBB2002B08D1F869FFF793FF22
:10CD2000FB787A69B96900F045FD00E000BF00BFFB
:10CD30002037BD4680BD80B584B000AF78600B461B
:10CD4000FB707868FBF7F2FEF860F868FFF76EFF9B
:10CD5000034683F00103DBB2002B0AD1F868FFF72A
:10CD600072FF024697F903301946104600F035FD70
:10CD700000E000BF00BF1037BD4680BD80B483B067
:10CD800000AF7860034B18460C37BD465DF8047B56
:10CD9000704700BF00F8FF0780B582B000AF786031
:10CDA0007868FFF7EBFF034618460837BD4680BD9D
:10CDB00080B483B000AF7860FF2318460C37BD46BF
:10CDC0005DF8047B704780B483B000AF7860FF23C8
:10CDD00018460C37BD465DF8047B704780B483B0BD
:10CDE00000AF786039607B681B0EDAB23B681A705E
:10CDF0007B681A0C3B680133D2B21A707B681A0A3E
:10CE00003B680233D2B21A703B6803337A68D2B2FD
:10CE10001A7000BF0C37BD465DF8047B704780B5C3
:10CE200082B000AF786039607B683968184600F0DE
:10CE300060FB00BF0837BD4680BD80B586B000AF3F
:10CE40007860396007F10C0319463868FEF70DFC6D
:10CE500007F10C0319467868FFF7E1FF00BF1837A8
:10CE6000BD4680BD80B588B000AFF860B9607A601B
:10CE7000FB70BB6A3B610023FB77FB7803F0010387
:10CE8000002B05D1FB78032B02D9FB78102B00D99E
:10CE9000FEE70023FB757B68BB61BB69002B06D0F6
:10CEA000FB7D0133FB75BB691B0ABB61F5E7FB7DAD
:10CEB000012B01D80223FB7597F82C300D2B02D9DA
:10CEC0000D2387F82C30FA7D97F82C30C3F10F032F
:10CED0009A4204DA97F82C30C3F10F03FB7597F8E8
:10CEE0002C20FB7DC3F10F039A4204DDFB7DC3F1CF
:10CEF0000F0387F82C30BB68002B01D0402200E0E4
:10CF00000022FB78023B5B10DBB2DB00DBB2134399
:10CF1000DAB2FB7D013BDBB21343DAB2FB6883F884
:10CF20002021FB6803F2211397F82C203969184659
:10CF300015F05EF87B68BB610F23BB75BA7D97F86F
:10CF40002C309A420ED9BB7DBA69D1B2FA6813442B
:10CF50000A4683F82021BB691B0ABB61BB7D013BEC
:10CF6000BB75EBE7F868FB6803F59071FB6803F5A8
:10CF700090731A4600F0D5FABB68002B00F095803C
:10CF8000BB68B3F57F4F25D2FB7F5A1CFA77194651
:10CF9000FA680A4492F82011BA68120AD2B2184606
:10CFA00081EA0203DAB2FB68034483F82021FB7FA5
:10CFB0005A1CFA771946FA680A4492F82011BA689E
:10CFC000D2B2184681EA0203DAB2FB68034483F85E
:10CFD00020216AE0FB7F5A1CFA771946FA680A4456
:10CFE00092F820211946D343DAB2FB680B4483F848
:10CFF0002021FB7F5A1CFA771946FA680A4492F8F6
:10D000002021194682F00103DB43DAB2FB680B44AE
:10D0100083F82021FB7F5A1CFA771946FA680A44E4
:10D0200092F82011BA68120ED2B2184681EA0203B1
:10D03000DAB2FB68034483F82021FB7F5A1CFA779D
:10D040001946FA680A4492F82011BA68120CD2B252
:10D05000184681EA0203DAB2FB68034483F8202110
:10D06000FB7F5A1CFA771946FA680A4492F8201195
:10D07000BA68120AD2B2184681EA0203DAB2FB6831
:10D08000034483F82021FB7F5A1CFA771946FA687B
:10D090000A4492F82011BA68D2B2184681EA020313
:10D0A000DAB2FB68034483F82021FB7D013BDAB24E
:10D0B000FB6883F83021FB6803F2311397F82C20CA
:10D0C0003969184614F094FF97F82C30013303F5B2
:10D0D0009873FA68D01897F82C30C3F10F031A46EA
:10D0E000002114F0ADFFFB6897F82C2083F8642131
:10D0F000FB68BA68C3F85021FB680022C3F85421CA
:10D10000FB687A68C3F85821FB680022C3F85C21E9
:10D11000FB7F9AB2FB68A3F86021FB681022A3F89A
:10D120006221FB68FA7883F8652100BF2037BD468D
:10D1300080BD80B586B000AFF860B9607A60BB682A
:10D140003B61FB68D3F854217B681A44FB68D3F831
:10D1500050319A4200D9FEE700237B617A697B68EF
:10D160009A422FD2FB68B3F86031102B0DD1F868CA
:10D17000FB6803F59071FB6803F590731A4600F0A5
:10D18000D0F9FB680022A3F86021FB68B3F8603196
:10D190005A1C91B2FA68A2F860111946FA680A445A
:10D1A00092F8201138697A6902441278184681EAA7
:10D1B0000203DAB2FB68034483F820217B69013360
:10D1C0007B61CBE7FB68D3F854217B681A44FB688A
:10D1D000C3F85421FB68D3F85421FB68D3F85031CD
:10D1E0009A4212D1FB68B3F86031002B09D0F8687D
:10D1F000FB6803F59071FB6803F590731A4600F025
:10D2000090F9FB680022A3F8602100BF1837BD46E3
:10D2100080BD80B58AB000AFF860B9607A603B60CD
:10D22000BB68BB617B687B61FB68D3F85C213B68B2
:10D230001A44FB68D3F858319A4200D9FEE700231C
:10D240003B623A6A3B689A4280F0A480FB68B3F87C
:10D250006231102B37D10F23FB61FB6893F86431E7
:10D260001A46FB69934220DDFA68FB69134403F513
:10D2700098731B780133D9B2FA68FB69134403F53C
:10D2800098730A461A70FA68FB69134403F5987399
:10D290001B78002B14BF01230023DBB2002B03D12A
:10D2A000FB69013BFB61D8E700BFF868FB6803F549
:10D2B0009871FB6803F5A0731A4600F032F9FB6819
:10D2C0000022A3F8622197F83030002B1BD1BA69F5
:10D2D0003B6A13441B7887F82730FB68B3F8623148
:10D2E0005A1C91B2FA68A2F862111A46FB681344FC
:10D2F00093F840117A693B6A134497F827204A4013
:10D30000D2B21A7019E07A693B6A13441A78FB6842
:10D31000B3F86231591C88B2F968A1F86201194664
:10D32000FB680B4493F84031534087F82730BA69C3
:10D330003B6A134497F827201A70FB68B3F86031F2
:10D34000102B0DD1F868FB6803F59071FB6803F5AD
:10D3500090731A4600F0E5F8FB680022A3F86021FC
:10D36000FB68B3F860315A1C91B2FA68A2F86011F8
:10D370001946FA680A4492F82021194697F827308E
:10D380005340DAB2FB680B4483F820213B6A013337
:10D390003B6256E7FB68D3F85C213B681A44FB68A4
:10D3A000C3F85C21FB68D3F85C21FB68D3F85831E3
:10D3B0009A421FD3FB68B3F86031002B09D0F8689C
:10D3C000FB6803F59071FB6803F590731A4600F053
:10D3D000A8F8FB6893F86431013303F59873FA6891
:10D3E000D018FB6893F86431C3F10F031A4600218B
:10D3F00014F026FE00BF2837BD4680BD80B584B03E
:10D4000000AF786039603B68BB607B68D3F85C2113
:10D410007B68D3F858319A4200D0FEE778687B6881
:10D4200003F598717B6803F5A0731A4600F079F84C
:10D430000023FB607B6893F865311A46FB689342D2
:10D4400015DA7A68FB68134403F5907319787A68E3
:10D45000FB68134403F5A0731A78FB68B8680344AB
:10D460004A40D2B21A70FB680133FB60E2E700BFAA
:10D470001037BD4680BD80B584B000AFF860B9609C
:10D480003B601346FB71FB6808221946386814F0AC
:10D49000AFFD3B6808333B603968B868FFF79EFC16
:10D4A0003B6804333B603B68FA791A7000BF103761
:10D4B000BD4680BD80B582B000AF78607B6803F167
:10D4C00008027B681A607B684FF48C729A807B68D4
:10D4D000184600F06DF80346002B14BF012300230B
:10D4E000DBB2002B00D0FEE77B6818460837BD464C
:10D4F00080BD80B582B000AF786039607B683A68E3
:10D500001146184600F073F80346002B14BF0123A0
:10D510000023DBB2002B00D0FEE700BF0837BD467A
:10D5200080BD80B584B000AFF860B9607A60FB68F8
:10D530007A68B968184600F09BF80346002B14BFC0
:10D5400001230023DBB2002B00D0FEE700BF103721
:10D55000BD4680BD80B582B000AF78607B6818465C
:10D5600000F0B6F80346002B14BF01230023DBB202
:10D57000002B00D0FEE77B6818460837BD4680BD0B
:10D5800080B483B000AF78607B681B6818460C37A6
:10D59000BD465DF8047B704780B483B000AF78600F
:10D5A0007B689B8818460C37BD465DF8047B704746
:10D5B00080B584B000AF78600023FB737B68002BDC
:10D5C00002D10723FB730DE07B689B88B3F58C7F4A
:10D5D00002D20123FB7305E07B681B68BB60B8685F
:10D5E00000F0ECFEFB7B18461037BD4680BD90B5C1
:10D5F00087B000AF786039600023FB7507F108033E
:10D600003968184600F09BF87B68002B02D107238D
:10D61000FB7528E07B689B88B3F58C7F02D20123E1
:10D62000FB7520E07B681B683B6107F10803184627
:10D63000FFF7A6FF044607F108031846FFF7ACFF03
:10D640000346DB001A462146386900F0DBF8034642
:10D65000002B14BF01230023DBB2002B02D00123D7
:10D66000FB7500E000BFFB7D18461C37BD4690BD32
:10D6700080B586B000AFF860B9607A600023FB75B2
:10D68000FB68002B02D10723FB751CE0FB689B881D
:10D69000B3F58C7F02D20123FB7514E0FB681B6895
:10D6A0003B617B68BA680121386900F0C7FE034618
:10D6B000002B14BF01230023DBB2002B02D0012377
:10D6C000FB7500E000BFFB7D18461837BD4680BDE6
:10D6D00080B584B000AF78600023FB737B68002BBB
:10D6E00002D10723FB730DE07B689B88B3F58C7F29
:10D6F00002D20123FB7305E07B681B68BB60B8683E
:10D7000000F06AFEFB7B18461037BD4680BD80B432
:10D7100083B000AF78607B681B6818460C37BD4645
:10D720005DF8047B704780B483B000AF78607B689D
:10D730009B8818460C37BD465DF8047B704780B562
:10D7400082B000AF786039603868FFF7E0FF0246CA
:10D750007B681A603868FFF7E6FF03461A467B6865
:10D760009A807B6818460837BD4680BD80B584B076
:10D7700000AFF860B9601346FB71F868FFF7FEF878
:10D78000FB791A46B968FEF7FAFA00BF1037BD46B2
:10D7900080BD80B582B000AF786039607868FFF7EF
:10D7A000EDF8034639681846FEF71CFD00BF083740
:10D7B000BD4680BD80B584B000AFF860B9607A60C6
:10D7C000FB70F868FFF7DAF8FB787A68B968FEF75B
:10D7D0002BFD00BF1037BD4680BD80B582B000AFC5
:10D7E00078600B46FB707868FFF7C8F8024697F937
:10D7F000033019461046FEF721FF00BF0837BD462B
:10D8000080BD0000E0B1D9B1C02A08B507D0B2F59B
:10D81000807F12D0802A0DD06FF01F0008BD0C232E
:10D82000036000F108034360D208184600F07AFB59
:10D83000002008BD0A230360F3E70E230360F0E72E
:10D840006FF02000704700BF10B504461046D4E9C1
:10D850000032063B9B0000F037FA002010BD00BFED
:10D8600010B504461046D4E90032063B9B0000F098
:10D8700003F8002010BD00BF2DE9F14F03F11C0497
:10D8800002EB840C4FEA930B8A68CB6808684968FE
:10D8900000F046F93CE9F0006040694072407B408E
:10D8A0000BF1060E4EE083EA134480EA134582EA48
:10D8B000134746BA96EA3444604000F00F1684EAF3
:10D8C000063420F00F1684EA161054BA94EA0106C2
:10D8D000724002F00F1486EA043622F00F1486EA32
:10D8E00014124CBA6540694001F00F1485EA043502
:10D8F00021F00F1485EA14115CBA67407B4003F0F5
:10D900000F1487EA043723F00F1487EA141344BA7C
:10D9100044404DBA4D4056BA56405FBA5F4087EA20
:10D92000174886EA174B84EA17464FEA38488BEACD
:10D930001B4485EA1B4788EA1B4580EA344069405E
:10D9400072407B4000F0703400F0803500F00F3002
:10D9500040EA440040EAD50080EA900404F0332411
:10D9600080EA8400604001F0703401F0803501F0FD
:10D970000F3141EA440141EAD50181EA910404F002
:10D98000332481EA8401614002F0703402F0803572
:10D9900002F00F3242EA440242EAD50282EA9204DD
:10D9A00004F0332482EA8402624003F0703403F00E
:10D9B000803503F00F3343EA440343EAD50383EA97
:10D9C000930404F0332483EA84036340C943DB43B4
:10D9D00081EA000483EA044686EA020183EA0143FD
:10D9E00082EA334583EA144383EA040484EA0007A5
:10D9F0007FEA040A8AEA024A8AEA010B87EA1148A6
:10DA00008AEA374A80EA060181EA1A418AEA030A69
:10DA100004EA0A00454088EA040707EA0B0041408F
:10DA20008AEA0B0608EA060084EA34428AEA3A46A1
:10DA300002EA060358404540414087EA37438BEAF3
:10DA40003B4003EA000985EA090582EA03094640EA
:10DA500009EA0606714085EA010005EA35464640B6
:10DA600006EA314181EA304181EA364606EA30462B
:10DA700086EA354634400F4086EA010508EA050883
:10DA800086EA3640024088EA020881EA31421340C1
:10DA90005C4080EA020309EA030987EA0907674054
:10DAA00088EA040806EA0A0601EA0B018AEA0B047E
:10DAB00025408AEA3A44204045408BEA3B4B02EA43
:10DAC0000B02564084EA0B04234059406E406940E3
:10DAD00087EA364080EA384080EA060380EA10444C
:10DAE00081EA134585EA344585EA17427D4082EA9A
:10DAF000354180EA05403CE9F000604069407240F1
:10DB00007B40BEF1010E3FF6CEAE00F05FF810BCD8
:10DB100020606160A260E360BDE8F08F00F002BAAF
:10DB200080EA101404F0F01480EA0410604081EAE6
:10DB3000111404F0F01481EA0411614082EA121415
:10DB400004F0F01482EA0412624083EA131404F031
:10DB5000F01483EA0413634080EA102404F47F4441
:10DB600080EA0420604081EA112404F47F4481EAC1
:10DB70000421614082EA122404F47F4482EA0422F0
:10DB8000624083EA132404F47F4483EA042363405D
:10DB900081EA500404F0553480EA4400614083EA8D
:10DBA000520404F0553482EA4402634082EA90044D
:10DBB00004F0333480EA8400624083EA910404F084
:10DBC000333481EA84016340704700BF82EA9004E5
:10DBD00004F0333480EA8400624083EA910404F064
:10DBE000333481EA8401634081EA500404F05534FF
:10DBF00080EA4400614083EA520404F0553482EA2A
:10DC00004402634080EA102404F47F4480EA042044
:10DC1000604081EA112404F47F4481EA04216140D8
:10DC200082EA122404F47F4482EA0422624083EAF6
:10DC3000132404F47F4483EA0423634080EA10142D
:10DC400004F0F01480EA0410604081EA111404F03A
:10DC5000F01481EA0411614082EA121404F0F01415
:10DC600082EA0412624083EA131404F0F01483EA97
:10DC700004136340704700BF2DE9F04F4FF2F002EC
:10DC800080EA1031114080EA0130484041088208A2
:10DC9000C3084FF0000EA3E000F0113001F0113185
:10DCA00002F0113203F0113340EA410040EA8200F1
:10DCB00040EAC3004FF2F00280EA1031114080EADE
:10DCC00001304840BDE8F08F2DE9F14F94464FEA0E
:10DCD000930B8A68CB6808684968FFF721FF0BF14E
:10DCE000060E33E083EA134480EA134582EA1347C1
:10DCF00046BA96EA3444604000F00F1684EA0634CF
:10DD000020F00F1684EA161054BA94EA0106724005
:10DD100002F00F1486EA043622F00F1486EA141279
:10DD20004CBA6540694001F00F1485EA043521F0D2
:10DD30000F1485EA14115CBA67407B4003F00F149E
:10DD400087EA043723F00F1487EA1413BCE8F000C5
:10DD50006040694072407B4000F0E03400F01035D4
:10DD600000F00F3040EA540040EAC50080EA900419
:10DD700004F0332480EA8400604001F0E03401F0D4
:10DD8000103501F00F3141EA540141EAC50181EA41
:10DD9000910404F0332481EA8401614002F0E0340C
:10DDA00002F0103502F00F3242EA540242EAC50294
:10DDB00082EA920404F0332482EA8402624003F08F
:10DDC000E03403F0103503F00F3343EA540343EA21
:10DDD000C50383EA930404F0332483EA8403634095
:10DDE00081EA324787EA134581EA354690EA06041C
:10DDF00084EA034B82EA1B4280EA044484EA054435
:10DE000083EA144A85EA14448BEA044B84EA3744D3
:10DE100081EA0B4181EA164104EA0A00454082EAA0
:10DE200004082BEA080041408AEA0B0602EA0600D1
:10DE300084EA34438AEA3A4603EA060778404540D2
:10DE4000414088EA38478BEA3B4007EA000985EA07
:10DE5000090583EA0709464006EA0906714085EA92
:10DE6000010005EA3546464006EA314181EA304183
:10DE700081EA364606EA304686EA3546344008EA04
:10DE8000010886EA01052A4086EA364003405A40E6
:10DE900081EA31431F407C4080EA030709EA070911
:10DEA00088EA0908544088EA020806EA0A0601EAF4
:10DEB0000B018AEA0B0215408AEA3A4210404540BB
:10DEC0008BEA3B4003405E404240174079404D4062
:10DED0004E40E443F64386EA18435D4085EA054038
:10DEE00083EA134386EA034183EA384284EA114312
:10DEF00083EA04435FEA3343BEF1010E3FF6F2AE1C
:10DF00003FF5CAAEBCE8F0006040694072407B401B
:10DF1000FFF75CFE10BC20606160A260E360BDE8BA
:10DF2000F08F00BF2DE9F04102F11C0506460746BF
:10DF300000EB850851F8040B46F8040B043AF9D1BC
:10DF40004FF0010CFFF798FE5FEA302080EA0C00EA
:10DF50004FEA4C0C4FEA1C2140F21B1201FB02F26B
:10DF60008CEA020C1ECF41404A4053405C401EC622
:10DF70002000464510D02C2DE4D03C2D06D1FFF7D3
:10DF80007BFE06CF41404A4006C6100006CF414006
:10DF90004A4006C61000D5E736E90F00FFF7C0FD7E
:10DFA00086E80F00043DF7D1BDE8F08190B4ADF5EF
:10DFB000016D00AF0023C7F80C380123C7F80838FB
:10DFC00026E007F58063D7F80C28D7F8081843F83F
:10DFD00022103B46D7F80828D7F80C1843F822102F
:10DFE000D7F808385A00D7F8083803F08003002B18
:10DFF00001D01B2300E000235A40D7F808385340D3
:10E00000DBB2C7F80838D7F80C380133C7F80C383A
:10E01000D7F80C38FF2BD4DD0023C7F80C380123C8
:10E02000C7F808381BE0D7F80828D849D7F80C38C3
:10E0300041F82320D7F808385A00D7F8083803F0F9
:10E040008003002B01D01B2300E000235340DBB2F0
:10E05000C7F80838D7F80C380133C7F80C38D7F8A8
:10E060000C38092BDFDDCA4B63221A70C94B002222
:10E0700083F863200123C7F80C386DE03B46D7F8DE
:10E080000C2853F82230C3F1FF0207F5806353F8E0
:10E090002230C7F80838D7F80838C7F80438D7F856
:10E0A00004385A00D7F80438DB111343DBB2C7F841
:10E0B0000438D7F80828D7F804385340C7F8083888
:10E0C000D7F804385A00D7F80438DB111343DBB211
:10E0D000C7F80438D7F80828D7F804385340C7F8E9
:10E0E0000838D7F804385A00D7F80438DB1113433E
:10E0F000DBB2C7F80438D7F80828D7F804385340FB
:10E10000C7F80838D7F804385A00D7F80438DB11B4
:10E110001343DBB2C7F80438D7F8043883F063033D
:10E12000D7F808285340C7F80838D7F80838D9B2C4
:10E13000974AD7F80C3813440A461A70D7F80C38A7
:10E14000D9B2944AD7F8083813440A461A70D7F857
:10E150000C380133C7F80C38D7F80C38FF2B8DDD9D
:10E160000023C7F80C3806E1894AD7F80C38134465
:10E170001B78C7F80838D7F808385A00D7F8083895
:10E1800003F08003002B01D01B2300E00023534049
:10E19000DBB2C7F80438D7F80428D7F8083853405A
:10E1A000DBB2C7F80038D7F808381A02D7F80438B5
:10E1B0005A40D7F808381B045A40D7F800381B06D5
:10E1C0005A407549D7F80C3841F82320724AD7F8DD
:10E1D0000C3852F823304FEA33627049D7F80C38C4
:10E1E00041F823206D4AD7F80C3852F823304FEA13
:10E1F00033626B49D7F80C3841F82320684AD7F8C6
:10E200000C3852F823304FEA33626649D7F80C389D
:10E2100041F823205F4AD7F80C3813441B78C7F81D
:10E220000838D7F80838002B18D03B469A6B3B4685
:10E23000D7F8081853F821301A445B4B82FB03349B
:10E240001319D911D317C91A0B461B025B1AD11A1D
:10E2500007F5806353F82130184600E00020D7F816
:10E260000838002B18D03B465A6A3B46D7F80818A6
:10E2700053F821301A444C4B82FB03341319D91143
:10E28000D317C91A0B461B025B1AD11A07F5806314
:10E2900053F821301B0200E000235840D7F808381B
:10E2A000002B18D03B465A6B3B46D7F8081853F85A
:10E2B00021301A443C4B82FB03341319D911D31774
:10E2C000C91A0B461B025B1AD11A07F5806353F873
:10E2D00021301B0400E000235840D7F80838002BF9
:10E2E00018D03B46DA6A3B46D7F8081853F8213075
:10E2F0001A442D4B82FB03341319D911D317C91AB1
:10E300000B461B025B1AD11A07F5806353F82130C4
:10E310001B0600E0002380EA03022449D7F80C38EA
:10E3200041F82320214AD7F80C3852F823304FEA1D
:10E3300033621F49D7F80C3841F823201C4AD7F81C
:10E340000C3852F823304FEA33621A49D7F80C38A8
:10E3500041F82320174AD7F80C3852F823304FEAF7
:10E3600033621549D7F80C3841F82320D7F80C3818
:10E370000133C7F80C38D7F80C38FF2B7FF7F4AE11
:10E3800000BF07F50167BD4690BC7047083E0020FE
:10E39000081C0020082D0020081D00200821002056
:10E3A000082500200829002081808080082E002078
:10E3B0000832002008360020083A002080B582B0DC
:10E3C00000AF78604FF48C720021786813F038FE4B
:10E3D00000BF0837BD4680BD80B582B000AF786011
:10E3E0007B68002B05D04FF48C71786800F042F800
:10E3F00000E000BF0837BD4680BD00BF80B584B0D7
:10E4000000AFF860B9607A607A68B968F868FFF7B9
:10E410001BFA00BF1037BD4680BD00BF80B584B079
:10E4200000AFF860B9607A607A68B968F868FFF799
:10E4300017FA00BF1037BD4680BD00BF80B584B05D
:10E4400000AFF860B9607A603B60BB68012B06D111
:10E450003A687968F868FFF7F7F9034605E03A6823
:10E460007968F868FFF7FCF9034618461037BD468F
:10E4700080BD00BF38B131B10144002203460130F4
:10E4800081421A70FAD1704780B483B000AF03465E
:10E49000FB7100BF0C37BD465DF8047B704780B44C
:10E4A00083B000AF78600B467B807B689B887A885E
:10E4B0009A4294BF01230023DBB218460C37BD46B5
:10E4C0005DF8047B704780B582B000AF78600B4682
:10E4D000FB7001217868FFF7E2FF0346002B0ED0A6
:10E4E0007B681B68591C7A681160FA781A707B681F
:10E4F0009B88013B9AB27B689A80002300E003234B
:10E5000018460837BD4680BD80B483B000AF786040
:10E510000B467B807B681A687B885B421A447B6869
:10E520001A607B689A887B8813449AB27B689A80C9
:10E5300000BF0C37BD465DF8047B704780B483B0E4
:10E5400000AF03460A46FB8013467B71FB881B1213
:10E550001AB2F9887B794B40DBB2064931F81330A7
:10E560001BB253401BB29BB218460C37BD465DF838
:10E57000047B7047343D020080B485B000AF034691
:10E58000FB71FB79F82B09D0F82B0ADC7E2B08DC19
:10E590007D2B03DA112B01D0132B02D10123FB7346
:10E5A00002E00023FB7300BFFB7B18461437BD4617
:10E5B0005DF8047B704780B483B000AF7860396049
:10E5C0007B683A681A607B6800229A807B681846EC
:10E5D0000C37BD465DF8047B704780B582B000AF54
:10E5E00078607B684FF6FF729A807B681B687E219B
:10E5F0001846FFF768FF034618460837BD4680BD3A
:10E6000080B584B000AF78600B46FB700023FB73CD
:10E61000FB781846FFF7B0FF0346002B27D07B6836
:10E620001B6802211846FFF73AFF034683F00103F7
:10E63000DBB2002B02D00323FB7336E07B681B6840
:10E640007D211846FFF73FFF03461846FFF71CFFE2
:10E650007B681A68FB7883F02003DBB2194610460A
:10E66000FFF731FF03461846FFF70EFF10E07B6807
:10E670001B68FA7811461846FFF725FF0346FB731F
:10E68000FB7B002B14BF01230023DBB2002B0BD13B
:10E690007B689B88FA7811461846FFF74FFF0346C0
:10E6A0001A467B689A8000E000BFFB7B1846103753
:10E6B000BD4680BD80B586B000AF78600023FB7595
:10E6C0007B681A6807F1080392E8030083E80300F7
:10E6D0007B689B88BB827B689B887B827B8ADB43D1
:10E6E0007B827B8ADBB219467868FFF789FF034695
:10E6F000FB75FB7D002B14BF01230023DBB2002B35
:10E7000020D17B8A1B12DBB219467868FFF778FFAD
:10E710000346FB75FB7D002B14BF01230023DBB2F6
:10E72000002B11D17B681B687E211846FFF7CBFEBA
:10E730000346FB75FB7D002B14BF01230023DBB2D6
:10E74000002B02E000BF00E000BFFB7D002B0BD0E0
:10E750007B681B681A4607F10803186810609B88DD
:10E7600093807B68BA8A9A80FB7D18461837BD462D
:10E7700080BD80B485B000AFF860B9607A603B605E
:10E78000FB6800221A70FB68BA685A60FB687A68F6
:10E790009A60FB683A68DA60FB6800221A82FB68BC
:10E7A00000225A82FB6818461437BD465DF8047B88
:10E7B000704780B586B000AFF860B9601346FB8043
:10E7C000FB885A1EFA80002B14BF01230023DBB202
:10E7D000002B00F0BC80BB685A1CBA601B78BB756C
:10E7E000FB681B78022B78D0022BE9DC002B02D0CF
:10E7F000012B0FD0AAE0BB7D7E2B40F0A680FB68EA
:10E8000001221A70FB6800225A82FB684FF6FF72E1
:10E810001A829AE0BB7D7D2B02D07E2B04D02AE0A9
:10E82000FB6802221A7057E0FB685B8A002B1AD043
:10E830000623FB75FB685B8A012B0DD9FB681B8ADD
:10E840004FF2B802934207D1FB685B680221184679
:10E85000FFF75AFE0023FB75FB689B68FA68D268D5
:10E86000F97D10469847FB6800225A82FB684FF6F4
:10E87000FF721A8230E0FB685B6801211846FFF7DF
:10E880000EFE0346002B1CD0FB681B8ABA7D114686
:10E890001846FFF753FE03461A46FB681A82FB68C8
:10E8A0005B68BA7D11461846FFF70DFE0346184611
:10E8B000FFF7EAFDFB685B8A01339AB2FB685A8274
:10E8C00009E0FB689B68FA68D26803211046984704
:10E8D000FB6800221A7000BF38E0FB685B6801210A
:10E8E0001846FFF7DCFD0346002B23D0BB7D83F0E9
:10E8F0002003BB75FB681B8ABA7D11461846FFF7DB
:10E900001DFE03461A46FB681A82FB685B68BA7DE7
:10E9100011461846FFF7D7FD03461846FFF7B4FD2A
:10E92000FB685B8A01339AB2FB685A82FB6801225A
:10E930001A700BE0FB689B68FA68D26803211046E6
:10E940009847FB6800221A7000E000BF38E700BF5C
:10E950001837BD4680BD80B483B000AF0346FB715D
:10E9600000BF0C37BD465DF8047B704780B584B0AE
:10E9700000AFF860B9601346FB80FB68BA681A60A4
:10E98000FB88BA681A44FB685A60FB68FA881A81E7
:10E9900000220021F86800F057F800220021F868F2
:10E9A00000F064F8F86800F005F8FB6818461037C6
:10E9B000BD4680BD80B582B000AF78607B681A68C4
:10E9C0007B681A627B68196801230122786800F06D
:10E9D0005FF802467B685A627B6802221A777B687E
:10E9E0001A687B689A627B681A687B68DA627B685F
:10E9F00000221A637B68002283F834207B6800229F
:10EA000083F835207B684FF6FF72DA867B681A68D8
:10EA10007B689A637B68196801230122786800F09B
:10EA200037F802467B68DA637B681A687B681A6489
:10EA30007B681A687B685A647B681A687B689A648A
:10EA400000BF0837BD4680BD80B485B000AFF86018
:10EA5000B9607A60FB68BA68DA60FB687A681A6144
:10EA600000BF1437BD465DF8047B704780B485B0A5
:10EA700000AFF860B9607A60FB68BA685A61FB68F9
:10EA80007A689A6100BF1437BD465DF8047B704711
:10EA900080B487B000AFF860B96011461A460B46E3
:10EAA000FB8013467B71BB687B617B79022B27D08F
:10EAB000022B29DC002B02D0012B10D024E0FB8894
:10EAC0007A6913447B61FB685B687A699A4218D360
:10EAD000FB681B895B427A6913447B61F3E7FB881F
:10EAE0005B427A6913447B61FB681B687A699A42CE
:10EAF00009D2FB681B891A467B6913447B61F3E7E3
:10EB0000FEE700BF00E000BF7B6918461C37BD462A
:10EB10005DF8047B704780B487B000AFF860B960DF
:10EB20007A60FB7000237B61FB78022B34D0022BD0
:10EB300033DC002B02D0012B17D02EE07A68BB68A3
:10EB40009A4204D37A68BB68D31A7B6125E0FB68DC
:10EB50005A68BB68D31A7B61FB681B687A68D31A52
:10EB60001A467B6913447B6117E07A68BB689A4256
:10EB700004D8BA687B68D31A7B610EE0FB685A68D8
:10EB80007B68D31A7B61FB681B68BA68D31A1A4684
:10EB90007B6913447B6100E0FEE77B699BB218460A
:10EBA0001C37BD465DF8047B704780B584B000AF6C
:10EBB000F860B96011461A460B46FB8013467B711C
:10EBC000FB881B12DAB2BB681A707B790122B96824
:10EBD000F868FFF75DFF0346FA88D2B21A7000BFEB
:10EBE0001037BD4680BD80B586B000AFF860B96013
:10EBF0001346FB71BB681B789BB21B02FB82FB793F
:10EC00000122B968F868FFF743FF03461B789AB200
:10EC1000FB8A1344FB82FB8A18461837BD4680BD29
:10EC200080B584B000AF78600B46FB700023FB73A7
:10EC30007B681B7F022B00D1FEE77B68D96A7B686B
:10EC40001B7F01227868FFF723FFB8607B681B7F7A
:10EC5000002B01D1012200E000227B68083253F82A
:10EC60002230BA689A4207D07B68DB6AFA781A7059
:10EC70007B68BA68DA6204E00323FB73786800F00B
:10EC80008DF8FB7B18461037BD4680BD80B584B03B
:10EC900000AF78600023FB730023BB817B689A6A16
:10ECA0007B68DB6A9A4230D17B681B7F1A467B689F
:10ECB000083253F822207B689B6A9A4205D1BB89AF
:10ECC0006FEA43436FEA5343BB8102237B817B8915
:10ECD000002B11D000217868FFF7A2FF0346FB73D9
:10ECE000FB7B002B14BF01230023DBB2002B0ED1D2
:10ECF0007B89013B7B81EAE77B68996A7B681B7FA4
:10ED0000BA897868FFF751FF02E000BF00E000BF5A
:10ED1000FB7B18461037BD4680BD80B584B000AF80
:10ED200078600B467B807B68996A7B68DA6A7B68CF
:10ED30001B7F7868FFF7EFFE0346FB81FB89012B01
:10ED400024D9FB89023BFB817B68996A7B681B7F26
:10ED50001A467868FFF747FF0346BB81FB89C3F378
:10ED60000D039AB2BB891343BB81BA897B881343D5
:10ED7000BB817B68996A7B681B7FBA897868FFF7DB
:10ED800014FF7B68DA6A7B689A6203E07B689A6AA0
:10ED90007B68DA6200BF1037BD4680BD80B582B0A7
:10EDA00000AF78607B681B7F022B10D07B681B7FD5
:10EDB0001A467B68083253F822207B68DA627B6847
:10EDC000DA6A7B689A627B6802221A7700E000BFE9
:10EDD000786800F0BCFB00BF0837BD4680BD80B43A
:10EDE00083B000AF78600B46FB707B681B7FFA78BE
:10EDF0009A420CBF01230023DBB218460C37BD46F4
:10EE00005DF8047B704780B582B000AF78600B4638
:10EE1000FB707868FFF7C2FFFB78002B05D0012B51
:10EE200007D17B6801221A7703E07B6800221A77FA
:10EE300000BF7B681B7F1A467B68083253F822208C
:10EE40007B68DA627B68DA6A7B689A6200BF08379F
:10EE5000BD4680BD80B584B000AF78600B46FB70C6
:10EE60000023FB737B681B7F022B02D10D23FB73F6
:10EE700015E07868FFF70AFF0346FB73FB7B002B66
:10EE800014BF01230023DBB2002B07D1FB78194606
:10EE90007868FFF7C5FE0346FB7300E000BFFB7B0D
:10EEA00018461037BD4680BD80B586B000AFF8600B
:10EEB000B9601346FB800023FB75FB681B7F022BA8
:10EEC00002D10D23FB752EE0F868FFF7DFFE034645
:10EED000FB75FB7D002B14BF01230023DBB2002B4D
:10EEE0001CD1FB885A1EFA80002B14BF012300237B
:10EEF000DBB2002B14D0BB685A1CBA601B781946D1
:10EF0000F868FFF78DFE0346FB75FB7D002B14BFF1
:10EF100001230023DBB2002B04D1E2E700BF02E0B3
:10EF200000BF00E000BFFB7D18461837BD4680BD1E
:10EF300080B584B000AF786039600023FB737B68D4
:10EF40001B7F022B02D10D23FB7316E07868FFF7BD
:10EF50009DFE0346FB73FB7B002B14BF01230023A4
:10EF6000DBB2002B08D17B68DA6A3B681A607B68E9
:10EF70009A6A3B685A6000E000BFFB7B1846103776
:10EF8000BD4680BD80B588B000AFF860B9607A60DA
:10EF90007B800023FB77FB681B7F022B02D10D23B4
:10EFA000FB7741E0BB685A68FB689B6A9A4202D0D3
:10EFB0000723FB7738E0FB68996AFB68DA6AFB682D
:10EFC0001B7FF868FFF7A7FD0346FB82FB68996A81
:10EFD000BB681A68FB681B7FF868FFF79CFD034657
:10EFE000BB82BA8A7B881A44FB8A9A4202DD0723D5
:10EFF000FB7719E0BB681B68BB617B88002B12D0D4
:10F000007B681A78BB691A707B6801337B607B88E8
:10F01000013B7B80FB681B7F0122B969F868FFF721
:10F0200037FDB861E9E700BFFB7F18462037BD46D2
:10F0300080BD80B584B000AF786039600023FB816B
:10F040007B681B7F022B2BD03B685A687B689B6ACE
:10F050009A4227D17B68996A7B68DA6A7B681B7F52
:10F060007868FFF758FD0346BB817B68996A3B6867
:10F070001A687B681B7F7868FFF74DFD03467B812C
:10F080007A89BB899A420FD23B6819687B68DA6A31
:10F090007B681B7F7868FFF73EFD0346FB8104E039
:10F0A00000BF02E000BF00E000BFFB891846103738
:10F0B000BD4680BD80B584B000AF78603960002364
:10F0C000FB737B681B7F022B02D10D23FB7329E0AE
:10F0D0003B685A687B689B6A9A4202D00723FB739D
:10F0E00020E07B68996A7B68DA6A7B681B7F7868B6
:10F0F000FFF711FD0346BB817B68996A3B681A687C
:10F100007B681B7F7868FFF706FD03467B817A8961
:10F11000BB899A4202D30723FB7303E03B681A685A
:10F120007B68DA62FB7B18461037BD4680BD90B520
:10F1300085B000AF78600023FB737B681B7F022BD8
:10F1400002D10D23FB7326E000217868FFF7E5FD6F
:10F150007B681B7F1A467B68083253F822207B6845
:10F160001A637B681B7F1A467B68996A7B68083242
:10F1700043F822107B68DB68002B09D07B68DC68D1
:10F180007B6818697B68196B7B681A7F7B68A0476E
:10F190007B6802221A77FB7B18461437BD4690BD68
:10F1A00080B483B000AF78607B681B6B18460C3767
:10F1B000BD465DF8047B704780B483B000AF7860D3
:10F1C0000B46FB70FA787B680E3253F82220F978F0
:10F1D0007B68083153F821309A4214BF0123002381
:10F1E000DBB218460C37BD465DF8047B704780B52E
:10F1F00082B000AF786001217868FFF7DDFF034639
:10F2000083F00103DBB2002B0BD000217868FFF7FD
:10F21000D3FF034683F00103DBB2002B01D00123AF
:10F2200000E0002318460837BD4680BD80B582B097
:10F2300000AF78607B6893F83530002B0CD101214A
:10F240007868FFF7B9FF0346002B01D0012200E0E8
:10F2500000227B6883F8342000BF0837BD4680BD9C
:10F2600080B584B000AF78600023FB737B685A6C74
:10F270007B681A647B681A6C7B6893F83430194693
:10F280007B68083153F821309A4202D11723FB736F
:10F2900044E07B68196C7B6893F834301A467868D0
:10F2A000FFF7A1FC0346BB81B7F90C30002B0EDA47
:10F2B0007B681A6C7B6893F8343019467B680E3192
:10F2C00053F821309A4202D01723FB7326E07B6863
:10F2D000196CBB89C3F30D039BB202339AB27B68EE
:10F2E00093F834307868FFF7D3FB02467B685A64A2
:10F2F0007B68196C7B6893F8343002227868FFF7DA
:10F30000C7FB02467B689A647B689A6C7B685B6C7F
:10F310009A42ABD07B68012283F83520FB7B002B1F
:10F3200003D07B68032283F83520FB7B1846103717
:10F33000BD4680BD80B584B000AF78600023FB730C
:10F340007868FFF754FF0346002B02D01723FB73A6
:10F3500015E07868FFF76AFF7B6893F834301A4647
:10F360007B680E3253F822207B685A647B685A6CA3
:10F370007B681A647868FFF773FF0346FB73FB7BB7
:10F3800018461037BD4680BD80B483B000AF7860AA
:10F390007B6893F83530032B04D07B6893F83530C5
:10F3A000002B01D1012300E0002318460C37BD4695
:10F3B0005DF8047B7047000080B584B000AF7860D2
:10F3C0000023FB737B6893F83530032B30D801A200
:10F3D00052F823F0E5F30000EBF3000031F40000F5
:10F3E000E5F300000023FB7322E07B689B6C1B7835
:10F3F000FB737B68996C7B6893F8343001227868E2
:10F40000FFF746FB02467B689A647B689A6C7B68D0
:10F410005B6C9A420BD11723BB73BB7B002B06D0CE
:10F420007868FFF71DFF03461846FFF794FA00BF00
:10F43000FB7B18461037BD4680BD00BF90B589B034
:10F4400000AF78600023FB777868FFF7D0FE0346B3
:10F45000002B02D01723FB7774E07868FFF7E6FEF5
:10F460007B6893F834301A467B680E3253F82230AA
:10F470003B617B6893F834301A467B680E3253F850
:10F480002230BB610023FB757B6893F834301A4649
:10F490007B68083253F82230BA699A422ED07B68D2
:10F4A00093F834301A46B9697868FFF79CFB034635
:10F4B000FB81B7F90E30002B0ADA7B6893F8343001
:10F4C0001A467B680E3253F82230BA699A4214D138
:10F4D000FB89C3F30D039BB202339AB27B6893F8A6
:10F4E0003430B9697868FFF7D3FAB861FB7D01332E
:10F4F000FB75FB7D0A2BC7D9FEE700BF7B6893F83D
:10F5000034301A467B680E32B96943F822107868A5
:10F5100000F01DF87B68002283F835207B684FF6E9
:10F52000FF72DA867B685B69002B0AD07B685C69B6
:10F530007B6898697B6893F834207B683969A047B9
:10F5400000E000BFFB7F18462437BD4690BD80B564
:10F5500082B000AF786001217868FFF72DFE034686
:10F5600083F00103DBB2002B0BD001217868FFF799
:10F5700036FC034683F00103DBB2002B01D00123EC
:10F5800000E00023002B0ED07B68996B0123012241
:10F590007868FFF77DFA02467B685A627B685A6A90
:10F5A0007B68DA6328E000217868FFF705FE0346F0
:10F5B00083F00103DBB2002B0BD000217868FFF74A
:10F5C0000EFC034683F00103DBB2002B01D00123C4
:10F5D00000E00023002B0ED07B68D96B00230122B2
:10F5E0007868FFF755FA02467B681A627B681A6AE8
:10F5F0007B689A6300E000BF00BF0837BD4680BD4E
:10F6000080B483B000AF78607B689A887B689A8109
:10F6100000BF0C37BD465DF8047B704780B483B0F3
:10F6200000AF78607B689A897B689B889A4234BF78
:10F6300001230023DBB218460C37BD465DF8047B7E
:10F64000704780B483B000AF78607B6800221A6096
:10F650007B6800229A807B680022DA807B68002227
:10F660001A817B6800229A727B680022DA727B68BA
:10F6700000229A817B680022DA817B6818460C3769
:10F68000BD465DF8047B704780B584B000AFF8607C
:10F69000B9601346FB80FB68BA681A60FB681B6898
:10F6A000002B01D0FA8800E00022FB689A80F868FD
:10F6B00000F007F8F868FFF7A3FF00BF1037BD465A
:10F6C00080BD80B582B000AF78607B680022DA80B0
:10F6D0007B689A887B681A817B6800229A727868B6
:10F6E000FFF78EFF00BF0837BD4680BD80B584B0F0
:10F6F00000AF786039600023FB7307F10E031946F1
:10F70000786800F021F80346FB73FB7B002B14BFE5
:10F7100001230023DBB2002B10D1BB7B002B03D1D4
:10F720003B6800221A700AE0BB7B012B03D13B68C7
:10F7300001221A7003E00623FB7300E000BFFB7B8D
:10F7400018461037BD4680BD80B485B000AF7860E4
:10F7500039600023FB737B68DB8801337A68128988
:10F76000934202D90623FB730DE07B681B687A681D
:10F77000D28813441A783B681A707B68DB8801339F
:10F780009AB27B68DA80FB7B18461437BD465DF879
:10F79000047B704780B584B000AF78603960002387
:10F7A000FB7307F10E0319467868FFF7CDFF034698
:10F7B000FB73FB7B002B14BF01230023DBB2002B68
:10F7C00004D1BB7B5AB23B681A7000E000BFFB7BE0
:10F7D00018461037BD4680BD80B485B000AF786054
:10F7E00039600023FB737B68DB8802337A681289F7
:10F7F000934202D90623FB731AE07B681B687A6880
:10F80000D28813441B781AB27B6819687B68DB883E
:10F8100001330B441B781B021BB213431BB29AB279
:10F820003B681A807B68DB8802339AB27B68DA8097
:10F83000FB7B18461437BD465DF8047B704780B4E7
:10F8400085B000AF786039600023FB737B68DB888C
:10F8500004337A681289934202D90623FB732AE0A3
:10F860007B681B687A68D28813441B7819467B68CA
:10F870001A687B68DB88013313441B781B0241EA5A
:10F8800003027B6819687B68DB8802330B441B78B2
:10F890001B041A437B6819687B68DB8803330B44BD
:10F8A0001B781B061A433B681A607B68DB880433AD
:10F8B0009AB27B68DA80FB7B18461437BD465DF848
:10F8C000047B70472DE9B00F91B000AF78633963C6
:10F8D000002387F83F307B6BDB8803F108027B6BEA
:10F8E0001B899A4203D9062387F83F30B9E07B6B26
:10F8F0001A687B6BDB8813441B78DCB24FF0000581
:10F900007B6B1A687B6BDB88013313441B78DAB29C
:10F910004FF000034FF000004FF00001190241EAE0
:10F920001261100244EA0003BB6245EA0103FB6274
:10F930007B6B1A687B6BDB88023313441B78DAB26B
:10F940004FF000034FF000004FF00001190441EAAE
:10F9500012411004D7E90A45234603433B622B4674
:10F960000B437B627B6B1A687B6BDB88033313442E
:10F970001B78DAB24FF00003110AF9611306BB617C
:10F98000D7E908452346D7E90601024613433B6100
:10F990002B460A4613437B617B6B1A687B6BDB88C3
:10F9A000043313441B78D8B24FF000014FF000022B
:10F9B0004FF0000303000022D7E90445214611431C
:10F9C000B96029461943F9607B6B1A687B6BDB8849
:10F9D000053313441B78D8B24FF000014FF00002FA
:10F9E0004FF0000303020022D7E90245214641EA15
:10F9F000020A294641EA030B7B6B1A687B6BDB88A2
:10FA0000063313441B78D8B24FF000014FF00002C8
:10FA10004FF00003030400224AEA02084BEA0309FC
:10FA20007B6B1A687B6BDB88073313441B78D8B277
:10FA30004FF000014FF000024FF0000303060022D8
:10FA400048EA0201396049EA03037B603B6BD7E96E
:10FA50000012C3E900127B6BDB8808339AB27B6B20
:10FA6000DA8097F83F3018464437BD46BDE8B00FFE
:10FA7000704780B586B000AF786039600023FB75B1
:10FA80007B681B687A68D28898187B681B891A463D
:10FA90007B68DB88D31A194607F10C031A4600F07D
:10FAA000B0FC38613B69002B02DC0623FB750AE0E1
:10FAB0007B68DA883B699BB213449AB27B68DA8030
:10FAC000FA683B681A60FB7D18461837BD4680BD52
:10FAD00080B487B000AFF860B9601346FB800023A4
:10FAE000FB75FB68DB881A46FB881344FA681289A9
:10FAF000934202DD0623FB750DE0FB681B68FA6884
:10FB0000D2881A44BB681A60FB68DA88FB88134401
:10FB10009AB2FB68DA80FB7D18461C37BD465DF85B
:10FB2000047B704780B584B000AFF860B9607A603C
:10FB3000FB681A89FB68DB88D31A9AB27B681A8043
:10FB40007B681B881A46B968F868FFF7C1FF03464F
:10FB500018461037BD4680BD80B586B000AFF8604E
:10FB6000B9607A600023FB7507F114031946F86841
:10FB7000FFF732FE0346FB75FB7D002B14BF01230C
:10FB80000023DBB2002B13D1BB8A1A46B968F86890
:10FB9000FFF79EFF0346FB75FB7D002B14BF01237F
:10FBA0000023DBB2002B05D1BA8A7B681A8002E001
:10FBB00000BF00E000BFFB7D18461837BD4680BD82
:10FBC00080B483B000AF78607B68DA887B689A8104
:10FBD0007B681A897B68DA817B689A7A7B68DA723B
:10FBE00000BF0C37BD465DF8047B704780B584B01C
:10FBF00000AF78600023FB737868FFF70FFD0346C2
:10FC000083F00103DBB2002B02D00D23FB730BE06A
:10FC10007B689A897B68DA807B68DA897B681A81DD
:10FC20007B68DA7A7B689A72FB7B18461037BD4690
:10FC300080BD80B582B000AF78600B46FB707B68FA
:10FC4000002283F824207B681B68FA781146184646
:10FC5000FFF7D9F8002318460837BD4680BD80B5A8
:10FC600086B000AFF8600B467A60FB720023FB752C
:10FC7000FB7A03F00F03002B0ED00121F868FFF789
:10FC8000D8FF0346FB75FB7D002B14BF0123002327
:10FC9000DBB2002B0ED02DE00021F868FFF7C9FF82
:10FCA0000346FB75FB7D002B14BF01230023DBB251
:10FCB000002B1CD1FB7A1946F868F2F77CF8034652
:10FCC000FB75FB7D002B14BF01230023DBB2002B4F
:10FCD0000FD17968F86800F021FA0346FB75FB7DC7
:10FCE000002B14BF01230023DBB2002B02E000BF76
:10FCF00000E000BFFB7D18461837BD4680BD80B5CB
:10FD000086B000AFF8607A603B600B46FB72002360
:10FD1000FB75FB7A7A681946F868FFF7A0FF03467F
:10FD2000FB75FB7D002B14BF01230023DBB2002BEE
:10FD30001AD1F86800F01BFB0346FB75FB7D002B16
:10FD400014BF01230023DBB2002B0FD13968F86800
:10FD500000F0E4F90346FB75FB7D002B14BF012383
:10FD60000023DBB2002B02E000BF00E000BFFB7D00
:10FD700018461837BD4680BD80B584B000AF7860A6
:10FD800039600023FB73786800F016FB0346FB73B1
:10FD9000FB7B002B14BF01230023DBB2002B1BD104
:10FDA0000021786800F0BAF90346FB73FB7B002B57
:10FDB00014BF01230023DBB2002B0FD13968786810
:10FDC00000F0ACF90346FB73FB7B002B14BF01234F
:10FDD0000023DBB2002B02E000BF00E000BFFB7B92
:10FDE00018461037BD4680BD80B584B000AF78603E
:10FDF0000023FB737B6893F82430002B0DD07868C8
:10FE000000F063FA0346FB73FB7B002B14BF012356
:10FE10000023DBB2002B08D1ECE77B681B68184697
:10FE2000FFF785F90346FB7300E000BFFB7B184634
:10FE30001037BD4680BD80B584B000AF78600B46FA
:10FE40007B800023FB737B681B687A88D2B21146E3
:10FE50001846FEF7FFFF0346FB73FB7B002B14BF26
:10FE600001230023DBB2002B13D17B681A687B8847
:10FE70001B0A9BB2DBB219461046FEF7EBFF0346A6
:10FE8000FB73FB7B002B14BF01230023DBB2002B91
:10FE900000E000BFFB7B18461037BD4680BD80B533
:10FEA00084B000AF786039600023FB737B681B6807
:10FEB0003A68D2B211461846FEF7CCFF0346FB73F0
:10FEC000FB7B002B14BF01230023DBB2002B38D1B6
:10FED0007B681A683B681B0ADBB219461046FEF7BE
:10FEE000B9FF0346FB73FB7B002B14BF01230023E8
:10FEF000DBB2002B27D17B681A683B681B0CDBB296
:10FF000019461046FEF7A6FF0346FB73FB7B002B4A
:10FF100014BF01230023DBB2002B16D17B681A68C3
:10FF20003B681B0EDBB219461046FEF793FF0346F3
:10FF3000FB73FB7B002B14BF01230023DBB2002BE0
:10FF400004E000BF02E000BF00E000BFFB7B1846FA
:10FF50001037BD4680BD90B587B000AFF860C7E9E7
:10FF600000230023FB75FB681B683A78114618468E
:10FF7000FEF770FF0346FB75FB7D002B14BF0123CA
:10FF80000023DBB2002B40F0B780FB681C68D7E988
:10FF900000014FF000024FF00003020A42EA016242
:10FFA0000B0AD3B219462046FEF754FF0346FB75F1
:10FFB000FB7D002B14BF01230023DBB2002B40F09C
:10FFC0009D80FB681C68D7E900014FF000024FF0EC
:10FFD0000003020C42EA01420B0CD3B21946204640
:10FFE000FEF738FF0346FB75FB7D002B14BF012392
:10FFF0000023DBB2002B40F08380FB681C68D7E94C
:020000021000EC
:1000000000014FF000024FF00003020E42EA01220D
:100010000B0ED3B219462046FEF71CFF0346FB75B4
:10002000FB7D002B14BF01230023DBB2002B69D121
:10003000FB681C68D7E900014FF000024FF0000395
:100040000A000023D3B219462046FEF703FF0346F9
:10005000FB75FB7D002B14BF01230023DBB2002BBB
:1000600052D1FB681C68D7E900014FF000024FF045
:1000700000030A0A0023D3B219462046FEF7EAFE1F
:100080000346FB75FB7D002B14BF01230023DBB26D
:10009000002B3BD1FB681C68D7E900014FF0000240
:1000A0004FF000030A0C0023D3B219462046FEF796
:1000B000D1FE0346FB75FB7D002B14BF01230023FB
:1000C000DBB2002B24D1FB681C68D7E900014FF09C
:1000D00000024FF000030A0E0023D3B21946204657
:1000E000FEF7B8FE0346FB75FB7D002B14BF012312
:1000F0000023DBB2002B0CE000BF0AE000BF08E0E9
:1001000000BF06E000BF04E000BF02E000BF00E067
:1001100000BFFB7D18461C37BD4690BD80B586B03C
:1001200000AF7860396007F10C033A680621184681
:1001300000F0D1F978617B699AB207F10C03194696
:100140007868F1F778FE034618461837BD4680BD3B
:1001500080B586B000AFF860B9601346FB8000231D
:10016000FB75FB881946F868FFF765FE0346FB75CB
:10017000FB7D002B14BF01230023DBB2002B0FD12A
:10018000FB881A46B968F868F1F755FE0346FB7517
:10019000FB7D002B14BF01230023DBB2002B00E00A
:1001A00000BFFB7D18461837BD4680BD80B584B0C2
:1001B00000AF78603960386812F090FAB860BB68B8
:1001C0004FF6FE72934202D94FF6FF73BB60BB68D5
:1001D0009BB21A4639687868F1F72DFE0346FB7327
:1001E000FB7B002B14BF01230023DBB2002B0FD1BC
:1001F0007B681B6800211846FEF72CFE0346FB7344
:10020000FB7B002B14BF01230023DBB2002B00E09B
:1002100000BFFB7B18461037BD4680BD80B584B05B
:1002200000AF78600023FB737B6893F82430032BC6
:1002300002D90D23FB7343E07B6818687B6893F851
:100240002430DB007A68134404331946FEF770FE4D
:100250000346FB73FB7B002B14BF01230023DBB29F
:10026000002B28D17B681B6800211846FEF7F2FDA1
:100270000346FB73FB7B002B14BF01230023DBB27F
:10028000002B1AD17B681B6800211846FEF7E2FD9F
:100290000346FB73FB7B002B14BF01230023DBB25F
:1002A000002B0CD17B6893F824300133DAB27B68E1
:1002B00083F8242004E000BF02E000BF00E000BF9C
:1002C000FB7B18461037BD4680BD80B584B000AFBB
:1002D00078600023FB737B6893F82430002B02D1F5
:1002E0000D23FB733EE07B6893F82430013BDAB2C8
:1002F0007B6883F824207B6818687B6893F8243037
:10030000DB007A68134404331946FEF792FE034675
:10031000BB81BB89012B02D80D23FB7322E0BB8973
:10032000023BBB81BB89DBB23B72BB891B0A9BB220
:10033000DBB27B727B6818687B6893F82430DB0043
:100340007A681344191D07F108020223FEF71AFE0A
:100350000346FB73FB7B002B14BF01230023DBB29E
:10036000002B00BFFB7B18461037BD4680BD80B513
:1003700084B000AF78600023FB737B681A687B68E9
:10038000283319461046FEF7D3FD0346FB73FB7B6B
:10039000002B14BF01230023DBB2002B06D17B68A6
:1003A00093F824207B6883F8252000E000BFFB7BC6
:1003B00018461037BD4680BD80B584B000AF786068
:1003C0000023FB737B681A687B6828331946104644
:1003D000FEF770FE0346FB73FB7B002B14BF01236B
:1003E0000023DBB2002B06D17B6893F825207B68C5
:1003F00083F8242000E000BFFB7B18461037BD4681
:1004000080BD80B489B000AFF860B9607A60002325
:10041000FB610023BB6100237B61BB68002B02D022
:100420007B691F2B03D94FF0FF33FB611BE0FB6897
:100430001B7803F07F027B6902FA03F3BA69134366
:10044000BB617B6907337B61FB690133FB61FB683F
:100450000133FB60BB68013BBB60FB68013B1B7861
:100460005BB2002BD9DBFB69002B05DD7B68002B21
:1004700002D07B68BA691A60FB6918462437BD460A
:100480005DF8047B704780B485B000AF78607B680E
:100490007F2B02D80123FB6016E07B68B3F5804F09
:1004A00002D20223FB600FE07B68B3F5001F02D28B
:1004B0000323FB6008E07B68B3F1805F02D2042372
:1004C000FB6001E00523FB60FB6818461437BD465E
:1004D0005DF8047B704780B586B000AFF860B96006
:1004E0007A607868FFF7CFFF3861BB683A699A4253
:1004F0001FDC00237B610EE07B68DAB2FB68591CCD
:10050000F96062F07F02D2B21A707B68DB097B600F
:100510007B6901337B613B69013B7A699A42EBD18C
:100520007B68DAB2FB68591CF96002F07F02D2B234
:100530001A703B6918461837BD4680BD80B483B039
:1005400000AF0346FB71FB79054A012101FA03F371
:10055000C2F8043500BF0C37BD465DF8047B704718
:1005600000F0014080B483B000AF0346FB71FB791B
:10057000054A012101FA03F3C2F8083500BF0C3720
:10058000BD465DF8047B704700F0014080B485B043
:1005900000AF0346B9607A60FB730949FB7BA23365
:1005A000BA6841F83320064AFB7BA233DB001344D0
:1005B0007A685A6000BF1437BD465DF8047B704707
:1005C00000F0014080B483B000AF03463960FB7196
:1005D0000649FB7903F511733A6841F8232000BFFF
:1005E0000C37BD465DF8047B704700BF00F001404A
:1005F00080B483B000AF78600B46FB70FB787A68FC
:10060000134418460C37BD465DF8047B704780B430
:1006100085B000AF78600B467B807B887A68134496
:1006200000221A607B887A6813441B68FB60FB68B1
:1006300000BF1437BD465DF8047B704780B483B0BB
:1006400000AF786039607B68D3F800223B681A43BA
:100650007B68C3F8002200BF0C37BD465DF8047B01
:10066000704780B485B000AFF8600B467A60FB72CB
:10067000FA7AFB6802F5A872796843F8221000BF85
:100680001437BD465DF8047B704780B483B000AF7B
:100690000346FB80FB8803F1804303F58053184633
:1006A0000C37BD465DF8047B7047000080B483B012
:1006B00000AF78600B46FB700C4A7B6803F5A273B1
:1006C00052F8233023F48012FB781B0503F48013C7
:1006D00006491A437B6803F5A27341F8232000BF43
:1006E0000C37BD465DF8047B704700BF00600040DA
:1006F00080B584B000AF03463960FB710023FB6016
:1007000010E0FA79FB6842FA03F303F00103002BCF
:1007100005D03B68002B09D03B68013B3B60FB6880
:100720000133FB60FB68032BEBD900E000BFFB68E3
:10073000002B01D1002314E0FB68012B01D1012320
:100740000FE0FB68022B01D102230AE0FB68032BB8
:1007500001D1032305E0054B054A7821054811F036
:10076000D1FB18461037BD4680BD00BF383F0200A0
:1007700010400200403F020080B588B000AFF86032
:10078000B9603B601346FB71FB68002B05D1764BCB
:10079000764AA721764811F0B5FBBB68002B05D13E
:1007A000744B724AA821724811F0ACFBFB681B7BAA
:1007B000002B29D0FB685B7BFF2B05D16E4B6B4A6E
:1007C000AC216B4811F09EFB6C4B1B78FF2B06D1C4
:1007D000FB685B7BFB76694AFB7E13701FE0FB685E
:1007E0005A7B664B1B789A420CD1654A634B1B7847
:1007F00003F5117352F82330002B03D1FB685B7BA8
:10080000FB760CE00823AAE0FB79002B03D05D4BBC
:1008100093F8203002E05B4B93F82130FB76BB6805
:100820005B78FA799A4206D0BB68DB789A00564B1F
:100830001344FB6105E0BB68DB789A00534B13441B
:10084000FB61FB689B7B002B1BD0012B7FD14C4AAB
:10085000FB7EA233DB0013445B68002B05D0FB7EDC
:10086000F9691846FFF7AEFE06E0FB681968FB7EE3
:10087000FA691846FFF78AFEFB7E1846FFF75EFE10
:100880006CE0FB681B7A002B05D1414B374AE22113
:10089000374811F037FBFB681B7A00211846FFF739
:1008A00027FF3861FB681A683B6950339B0013448B
:1008B0001946FB7EFA691846FFF768FEFB7E18466C
:1008C000FFF73CFEFB6818683B69D9B2FB685A68C1
:1008D0003B68D31A1A46FFF7C4FE2A4B5B7F002BF6
:1008E00006D0284BDB7F9A00284B13447B6105E040
:1008F000244BDB7F9A00244B13447B61FB681B7AFB
:1009000001211846FFF7F4FE38611E4B93F82200D0
:10091000FB681A683B6950339B0013447A69194697
:10092000FFF734FE174B93F822301846FFF706FE08
:10093000FB6818683B69D9B2FB685A683B68D21AF1
:10094000104B9B68D31A1A46FFF78BFE06E0114B3B
:10095000064A4FF48C71064811F0D4FA0023184669
:100960002037BD4680BD00BFA03F020030400200DE
:10097000403F0200A83F0200B83F020030000020C4
:1009800000F001400C00002060600040306000403A
:10099000E43F0200383F020080B584B000AF7860C9
:1009A0000B46FB707B68002B06D11D4B1D4A40F2A5
:1009B00025111D4811F0A6FA7B681B7B002B03D084
:1009C0007B685B7BFB730AE0FB78002B03D0174B43
:1009D00093F8203002E0154B93F82130FB73FB7B3A
:1009E0001846FFF7BFFDFB7B002200211846FFF7EA
:1009F000CDFDFB7B00211846FFF7E4FD7B689B7B68
:100A0000012B06D90A4B074A40F23D11064811F066
:100A100079FA00BF002318461037BD4680BD00BFDD
:100A2000A03F020048400200403F02000C000020AE
:100A3000383F020080B584B000AF78603960174B52
:100A40001B7D83F00103DBB2002B01D00F2320E0DC
:100A50007B68002B0CD0114B1B6801221049786871
:100A6000FFF78AFEF860FB68002B01D0FB6810E0FE
:100A70003B68002B0CD0094B1B68002208493868E2
:100A8000FFF77AFEF860FB68002B01D0FB6800E0FE
:100A9000002318461037BD4680BD00BF0C00002063
:100AA0002000002080B584B000AF78603960174B1B
:100AB0001B7E83F00103DBB2002B01D00F2320E06B
:100AC0007B68002B0CD0114B5B68012210497868C1
:100AD000FFF752FEF860FB68002B01D0FB6810E0C6
:100AE0003B68002B0CD0094B5B6800220849386832
:100AF000FFF742FEF860FB68002B01D0FB6800E0C6
:100B0000002318461037BD4680BD00BF0C000020F2
:100B10002400002080B584B000AF78603960144BA9
:100B20001B7D83F00103DBB2002B01D00F231AE001
:100B30007B68002B09D001217868FFF72DFFF86052
:100B4000FB68002B01D0FB680DE03B68002B09D04F
:100B500000213868FFF720FFF860FB68002B01D008
:100B6000FB6800E0002318461037BD4680BD00BF7B
:100B70000C00002080B584B000AF78603960144B61
:100B80001B7E83F00103DBB2002B01D00F231AE0A0
:100B90007B68002B09D001217868FFF7FDFEF86023
:100BA000FB68002B01D0FB680DE03B68002B09D0EF
:100BB00000213868FFF7F0FEF860FB68002B01D0D9
:100BC000FB6800E0002318461037BD4680BD00BF1B
:100BD0000C00002080B582B000AF0346FB711C4BB7
:100BE0001B7D002B15D0FB7903F00103002B10D0E7
:100BF000174B5B7D002B06D0154BDB7D0021184683
:100C0000FFF754FD05E0124BDB7D01211846FFF78D
:100C10004DFD0F4B1B7E002B15D0FB7903F002031B
:100C2000002B10D00A4B5B7E002B06D0084BDB7EDE
:100C300000211846FFF73AFD05E0054BDB7E012158
:100C40001846FFF733FD00BF0837BD4680BD00BF23
:100C50000C00002080B500AF224B93F820301846DE
:100C6000FFF780FC1F4B93F820300022002118462C
:100C7000FFF78CFC1B4B93F8203000211846FFF740
:100C8000A1FC184B93F821301846FFF76BFC154B6D
:100C900093F82130002200211846FFF777FC114B12
:100CA00093F8213000211846FFF78CFC0E4B1B787F
:100CB000FF2B14D00C4B1B781846FFF753FC0A4B44
:100CC0001B78002200211846FFF760FC064B1B78BA
:100CD00000211846FFF776FC034BFF221A7000BF75
:100CE00080BD00BF0C0000203000002080B588B01F
:100CF00000AFF860B9601346FB712C4B1B7F83F08B
:100D00000103DBB2002B01D000234AE0274B5B7FBD
:100D1000002B06D0254BDB7F9A00254B1344FB614B
:100D200005E0224BDB7F9A00224B1344FB61BB683A
:100D3000D9B21E4BDB6801331A46F868FFF791FC05
:100D40001A4B93F82200BB6850339B00FA68134497
:100D5000FA691946FFF71AFC4FF48870FFF795FC03
:100D6000B8610021F868FFF743FC03467B614FF44C
:100D70008071F868FFF762FCFB797A69B9691846F7
:100D8000FFF704FCFB7900211846FFF71BFCFB79F9
:100D90001846FFF7D3FB4FF4A071F868FFF737FC54
:100DA000012318462037BD4680BD00BF0C0000203F
:100DB000606000403060004080B483B000AF034604
:100DC000FB71FB79054A012101FA03F3C2F80435EE
:100DD00000BF0C37BD465DF8047B704700F0014052
:100DE00080B483B000AF0346FB71FB79054A012153
:100DF00001FA03F3C2F8083500BF0C37BD465DF8B1
:100E0000047B704700F0014080B485B000AF03461A
:100E1000B9607A60FB730949FB7BA233BA6841F879
:100E20003320064AFB7BA233DB0013447A685A6006
:100E300000BF1437BD465DF8047B704700F00140E9
:100E400080B483B000AF03463960FB710649FB797B
:100E500003F511733A6841F8232000BF0C37BD46F3
:100E60005DF8047B704700BF00F0014080B584B09E
:100E700000AFB9607A603B600346FB73FB7B7A6826
:100E8000B9681846FFF7C0FFFB7B39681846FFF7C3
:100E9000D7FF00BF1037BD4680BD000080B483B0CF
:100EA00000AF03460A46FB711346BB710A4ABB7981
:100EB00003F5007352F82310FB7901229A4006488B
:100EC000BB790A4303F5007340F8232000BF0C37B9
:100ED000BD465DF8047B704700F0014080B483B0EC
:100EE00000AF0346FB71054AFB79012142F833103C
:100EF00000BF0C37BD465DF8047B704700F0014031
:100F000080B483B000AF0346FB71064AFB79DB0077
:100F1000134401225A6000BF0C37BD465DF8047BC4
:100F2000704700BF00F0014080B483B000AF0346BB
:100F3000FB71FB79DB00043303F1804303F5F833E5
:100F400018460C37BD465DF8047B704780B582B00B
:100F500000AF0F4B00221A600E4B00221A7000F0F7
:100F600099FDF5F7C1FA786000F0C6FD38603A687F
:100F700079680D20FFF748FF0D20FFF71DFF0121C5
:100F80000E20FFF78BFF00BF0837BD4680BD00BFB6
:100F9000403E00203D3E002080B500AF00F082FDC5
:100FA0000D20FFF71DFF002200210D20FFF72CFF71
:100FB0000120FFF7A5FF0023002200210E20FFF7EC
:100FC00055FF00BF80BD000080B500AF054B00227B
:100FD0001A7000F071FD00F09BFDF5F73FFA00BFBD
:100FE00080BD00BF3C3E002080B500AF00F07AFD20
:100FF000F5F773FA00BF80BD90B583B000AF78609D
:1010000000F0CCFD04460120FFF78EFF0346224688
:1010100079680E20FFF72AFF0120FFF75FFF00BF6E
:101020000C37BD4690BD00002DE9B04F92B000AF27
:101030007863002387F847307B6B002B05D1754B15
:10104000754A9921754810F05DFF754B1B78DBB22E
:10105000002B00F0D88000F0ADFD3864714B5A6869
:101060003B6C9B1AFB63704B1B78002B00F0BE801F
:101070006E4B1B6818464FEAE071FB6B1A464FF047
:10108000000302FB01F500FB03F42C44A0FB022348
:10109000E1180B46DB0FD9B2644B1A686FF480037A
:1010A0009A42D4BF01230023DBB24B40DBB2002BBA
:1010B00054D05E4B1B6818464FEAE071FB6B1A4632
:1010C0004FF0000302FB01F500FB03F42C44A0FBEE
:1010D000020163181946554B1B681A464FEAE27322
:1010E00012F58004BC6243F10003FB62D7E90A8970
:1010F0004B46DB0F1A464FF00003444614193C6080
:101100004C4643EB04047C604FF000024FF00003B8
:10111000D7E90089444662084C4642EAC4724C460C
:101120006310524263EB430384183C6241EB0303B8
:101130007B623E4B1B681A464FEAE27312F5800150
:10114000B96143F10003FB61D7E90623D7E9080140
:1011500010F00CFD02460B46134648E0334B1B686B
:1011600018464FEAE071FB6B1A464FF0000302FB92
:1011700001F500FB03F42C44A0FB0201631819469F
:101180002A4B1B681A464FEAE27312F5800A43F1B4
:10119000000B4FEADB731A464FF0000312EB0A080C
:1011A00043EB0B094FF000024FF000034FEA5802E7
:1011B00042EAC9724FEA690384183C6141EB0303B8
:1011C0007B611A4B1B681A464FEAE27312F58001E5
:1011D000B96043F10003FB60D7E90223D7E90401BA
:1011E00010F0C4FC02460B46134600E00023BB632C
:1011F0000C4B1A68FB6B1A44BB6BD21A7B6B1A60E0
:10120000012387F8473097F8473018464837BD46DE
:10121000BDE8B08F64400200C44002007840020084
:101220003C3E0020343E00203D3E0020403E002059
:1012300080B588B000AF3B1D0433184600F080FC39
:101240000346002B00F09780F5F75CF903467B60BE
:101250004D4B1B78DBB2002B68D07A684B4B1B6878
:10126000D31AFB61BA68494B5B68D31ABB61FB694F
:1012700003F500139B0D7B61BA69FB69D31A3B61CF
:101280003B69DB0FDAB27B69DB0FDBB25340DBB2C9
:10129000002B0BD07B69DA0F13445B105B421A46BC
:1012A0003B691A447B6992FBF3F309E07B69DA0F2F
:1012B00013445B101A463B691A447B6992FBF3F3B3
:1012C000FB60334B1B78002B2AD0324B1A68134635
:1012D000DB009A1AFB681344DB0F03F00103DBB257
:1012E000002B0DD02B4B1A681346DB009A1AFB68B3
:1012F0001344043B002B00DA0733DB101A460CE0E2
:10130000244B1A681346DB009A1AFB681344043313
:10131000002B00DA0733DB101A461E4B1A6002E07E
:101320001C4AFB6813601A4B01221A70164B0022EC
:101330001A70BFF35F8F00BF144B1A463B1D93E832
:10134000030082E80300BFF35F8F00BF0E4B012252
:101350001A7000F0DDFB0D4B1A680D4B1B78002B4B
:1013600002D04FF0807301E04FF48003194610461D
:10137000F5F79CF803E000F0CBFBF5F76FF800BF42
:101380002037BD4680BD00BF3C3E0020343E0020DB
:101390003D3E0020403E002080B582B000AF3B467D
:1013A0001846FFF741FE0346FB71FB7983F001030A
:1013B000DBB2002B02D000233B6005E03B68002B32
:1013C00002D13B6801333B603B6818460837BD4695
:1013D00080BD80B584B000AF0346FB7106F0AAFE65
:1013E00003461A46FB79934214BF01230023FB7383
:1013F000FB79184606F0ACFEFB7B002B01D001F018
:101400000FFC00BF1037BD4680BD80B500AF06F0B1
:1014100091FE0346184680BD80B582B000AF0346FA
:10142000FB7197F90730184606F0C6FE00BF083773
:10143000BD4680BD80B500AF06F0A0FE03465BB29E
:10144000184680BD80B500AF01F0F6FB00BF80BD3F
:1014500080B582B000AF7860786806F0C7FE00BF44
:101460000837BD4680BD80B582B000AF786078682F
:1014700006F0D8FE00BF0837BD4680BD80B582B0FB
:1014800000AF7860786806F0EBFE00BF0837BD4615
:1014900080BD80B483B000AF0346FB71FB799B082D
:1014A000DBB25E3BDBB25BB218460C37BD465DF883
:1014B000047B704780B483B000AF0346FB71FB79B7
:1014C0005E33DBB218460C37BD465DF8047B7047CF
:1014D00080B485B000AF78600B46FB700A23FB60D8
:1014E000FB7801335B001A46FB681344FB60FB6822
:1014F0001B017A68D31A18461437BD465DF8047B81
:10150000704780B500AF01F079FF06F0ADF800F04C
:10151000FCF906F087FC06F055FD01F081FAF4F7BE
:101520004BFF06F08DFD01F0FBFAF6F7EFF901F045
:101530000BFB00F0B3FB00F0EDFD06F06FFFF6F7DC
:101540000DFCFFF703FD01F00BF900BF80BD80B576
:1015500000AF01F021F9FFF71FFDF6F706FC00F0E0
:101560001FFEF6F7DAF9F4F72EFF00F0D5F906F0D2
:101570008DF800BF80BD000080B500AF06F098F880
:101580000346092B22D801A252F823F0B515010019
:10159000B5150100B9150100B9150100BD1501000F
:1015A000BD150100BD150100C1150100C5150100E3
:1015B000C915010002230AE0032308E0042306E022
:1015C000052304E0062302E0072300E00123184678
:1015D00080BD00BF80B582B000AF012001F0BBFA32
:1015E0000346FB71FB7918460837BD4680BD80B5C0
:1015F00082B000AF002001F0AEFA034683F0010391
:10160000DBB2FB71FB7918460837BD4680BD80B55B
:1016100082B000AF012300220021012001F0ABFACB
:101620000346FB71FB7918460837BD4680BD80B57F
:1016300086B002AF78600B46FB70FB780022019207
:10164000002200927A680021002001F0ACFA0346E3
:10165000FB73FB7B18461037BD4680BD80B588B054
:1016600002AFF8607A603B600B46FB72F97A97F83C
:10167000203000933B687A68F86802F007FB034665
:10168000FB75FB7D18461837BD4680BD80B584B01C
:1016900000AF78607968002001F0A2FA0346FB737E
:1016A000FB7B18461037BD4680BD000080B584B076
:1016B00000AF78607B68FB60FB6893F8803083F054
:1016C0000103DBB2002B06D10C4B0D4A4FF4F8712D
:1016D0000C4810F017FC786801F094FA0346FB728E
:1016E000FB7A002B06D1084B054A4FF4FB710548E5
:1016F00010F008FC00BF1037BD4680BDEC40020072
:101700004C410200044102004441020080B500AF98
:1017100001F09EFA0346184680BD80B582B000AF46
:101720000023FB71FB1D184601F09EFA034683F06F
:101730000103DBB2002B01D07F23FB7197F9073047
:1017400018460837BD4680BD80B500AF06F0B4FC32
:101750000346184680BD80B582B000AF0346FB71DA
:10176000FB79184606F0B6FC00BF0837BD4680BDC1
:1017700080B582B000AF0346FB71FB79184601F0DB
:1017800059FE00BF0837BD4680BD80B584B002AFAA
:1017900078600B46FB70F978002300930023002249
:1017A000786801F057FE034618460837BD4680BDED
:1017B00080B582B000AF78600B46FB70FB780022EA
:1017C0001946786801F075FE034618460837BD468D
:1017D00080BD80B582B000AF0346FB71FB7900216C
:1017E000184601F087FE00BF0837BD4680BD80B5B2
:1017F00082B000AF7860786806F044FD01F01CFA12
:1018000000BF0837BD4680BD80B582B000AF7860AC
:10181000786806F075FD00BF0837BD4680BD80B50D
:1018200082B000AF7860786801F0D4FF00BF08375D
:10183000BD4680BD80B582B000AF78600B46FB70BE
:101840001346BB70FFF7A8FD0346BA7897F903105B
:101850007868F5F71DFE00BF0837BD4680BD80B52E
:1018600088B002AFF860B96011461A460B46FB71AA
:101870001346BB71BB68002B03D0FFF78DFD0346F9
:1018800000E000237B61B97997F907207B69009319
:101890000B46B968F868F5F727FF00BF1837BD4653
:1018A00080BD80B483B000AF0346FB7100BF0C372E
:1018B000BD465DF8047B704780B483B000AF03463B
:1018C000FB7100BF0C37BD465DF8047B704780B4E8
:1018D00083B000AF0346FB7100BF0C37BD465DF817
:1018E000047B704780B582B000AF0346FB71FB7983
:1018F000002B01D100F0B1FDFB79012B01D100F0EB
:1019000023F800BF0837BD4680BD80B400AF00BFDC
:10191000BD465DF8047B704780B400AF00BFBD4694
:101920005DF8047B7047000080B500AF024807F007
:1019300055FE00BF80BD00BF3400002080B500AF61
:1019400007F088FE00BF80BD80B400AF00BFBD4679
:101950005DF8047B704780B483B000AF78600B46BD
:10196000FB70FB787A68134401221A6000BF0C37C1
:10197000BD465DF8047B704780B483B000AF7860EB
:101980000B46FB70FB787A68134418460C37BD464B
:101990005DF8047B704780B483B000AF78600B467D
:1019A000FB707B68D3F8043523F00302FB7803F067
:1019B00003031A437B68C3F8042500BF0C37BD46F8
:1019C0005DF8047B704780B483B000AF78600B464D
:1019D000FB707B68D3F8083523F00302FB7803F033
:1019E00003031A437B68C3F8082500BF0C37BD46C4
:1019F0005DF8047B704780B483B000AF78600B461D
:101A0000FB707B68D3F8103523F00F02FB7803F0EE
:101A10000F031A437B68C3F8102500BF0C37BD467F
:101A20005DF8047B704780B485B000AFF8600B466A
:101A30007A60FB72FA7AFB6802F5A872796843F85B
:101A4000221000BF1437BD465DF8047B704780B498
:101A500083B000AF78600B46FB70FA787B6802F5C4
:101A6000A87253F8223018460C37BD465DF8047B47
:101A70007047000080B500AF44210548FFF76BFFB9
:101A800001210348FFF7E3FF0346184680BD00BF6E
:101A90000080004080B400AF00BFBD465DF8047B0D
:101AA0007047000080B500AF10210248FFF753FFD8
:101AB00000BF80BD0080004080B500AF0021084815
:101AC000FFF769FF03210648FFF77DFF0421044863
:101AD000FFF791FF00210248FFF73DFF00BF80BDE7
:101AE0000080004080B500AF10210248FFF733FFAF
:101AF00000BF80BD0080004080B500AF4821034892
:101B0000FFF73AFF0346184680BD00BF0080004043
:101B100080B582B000AFFFF7ADFF0346013B7B60AD
:101B2000054A7B6813607A6802210448FFF77BFF4F
:101B300000BF0837BD4680BD443E00200080004005
:101B400080B584B000AF78600023FB7302210E489B
:101B5000FFF77DFFB8607B68002B05D10B4B0C4A6B
:101B60007B210C4810F0CEF90B4B1B68BA689A42E7
:101B700004D07B68BA681A600123FB73FB7B1846AC
:101B80001037BD4680BD00BF0080004068410200A4
:101B9000D84102007C410200443E002080B500AFE5
:101BA0004C210348FFF7E8FE0346184680BD00BFFE
:101BB0000080004080B500AF03210348FFF747FFD6
:101BC0000346184680BD00BF0080004080B489B045
:101BD00000AF0346FB710E4B3B613B69D3E84F3FBF
:101BE000FB60FB68DBB2FB72FB7AFB79FB77084B8F
:101BF000BB61FA7FB969C1E8432F7B617B69002B28
:101C0000E9D100BF00BF2437BD465DF8047B7047B3
:101C1000483E002080B487B000AF0E4BBB60BB686D
:101C2000D3E84F3F7B607B68DBB2FB75FF23BB755E
:101C3000084B3B61BA7D3969C1E8432FFB60FB6803
:101C4000002BEAD1FB7D18461C37BD465DF8047BAE
:101C5000704700BF483E002080B400AF064B1B78A1
:101C6000DBB2FF2B0CBF01230023DBB21846BD46BD
:101C70005DF8047B704700BF483E002080B582B00D
:101C800000AF0346FB71FB79FF2B03D0FB791846AD
:101C900004F08EFE00BF0837BD4680BD80B400AFA3
:101CA000034BFF221A7000BFBD465DF8047B7047EE
:101CB000483E002080B582B000AF0346FB71FB793F
:101CC000184600F08DFA00BF0837BD4680BD80B5CC
:101CD00084B000AF0346FB710023FB7306F0B4F839
:101CE0000346FB73FB7B002B09D0FFF7B5FF0346D0
:101CF000002B04D0FB79184604F05AFE03E0FB7970
:101D00001846FFF763FFFB7B002B01D006F0C6F8F7
:101D100000BF1037BD4680BD80B400AF00BFBD46D8
:101D20005DF8047B704780B500AFFFF773FF034693
:101D30001846FFF7A3FF00BF80BD80B500AFFFF7D7
:101D40008BFF0346002B14BF01230023DBB283F07B
:101D50000103DBB203F00103DBB2184680BD80B49F
:101D600089B000AF786039607B68BB61BB69D3E83C
:101D70004F3F7B617B69DBB2FB77FB7F002B0BD096
:101D8000BFF32F8F00BF3B681B78DBB20133DAB2A1
:101D90003B681A7000230FE00123FB747B68FB6033
:101DA000FA7CF968C1E8432FBB60BB68002BDBD12C
:101DB000BFF35F8F00BF012318462437BD465DF88F
:101DC000047B704780B483B000AF7860BFF35F8F4F
:101DD00000BF7B6800221A7000BF0C37BD465DF85B
:101DE000047B704790B587B000AF0023FB7500F00F
:101DF000DFFCF86000233B6126E03B695B01164A8B
:101E00001344BB60BB685B687B60BB689C6800F088
:101E1000D6FC0346E31AA3F5F0733B60BB681B785E
:101E2000FA7D9A420DD23A687968F86800F0CEFCE3
:101E3000034683F00103DBB2002B02D0BB681B78A2
:101E4000FB753B6901333B613B69012BD5D9FB7DB8
:101E500018461C37BD4690BD583E002080B582B064
:101E600000AFFFF7BFFF0346FB71064B1B78FA7903
:101E70009A4202D2034B1B78FB71FB791846083754
:101E8000BD4680BD543E002080B582B000AF034601
:101E90000A46FB711346BB71FB79032B05D9134B23
:101EA000134AB121134810F02DF8134B1B78002B67
:101EB00002D1BB79002B14D1FB79104AD35CDBB281
:101EC000BA799A4208D1BB79002B05D00C4B084A4D
:101ED000B921084810F016F8FB790849BA79CA54B4
:101EE00000E000BF0837BD4680BD00BFFC410200D6
:101EF0004443020014420200533E0020503E0020A2
:101F00005C42020080B582B000AF24492448FFF74C
:101F100026FF034683F00103DBB2002B39D11F4BB0
:101F20001B78FB711F4B1B78BB71FFF797FF0346B4
:101F30007B71BA797B799A4221D01A4A7B791370E6
:101F40007B79184606F0BCFA7B7919460220FFF728
:101F50009BFF7B79002B0CD100F0E9FD00210020D4
:101F6000FFF792FF00F0C0FE00210120FFF78CFF79
:101F700005E000F0E2FDFFF7D7FC00F097FE08480F
:101F8000FFF720FF054B1B78DBB2FA799A42BCD1F0
:101F900000E000BF0837BD4680BD00BF4C3E0020BA
:101FA0004B3E0020533E002080B483B000AF04239A
:101FB000FB7100233B600FE00C4A3B6813441B7825
:101FC000DBB2FA799A4204D9084A3B6813441B7879
:101FD000FB713B6801333B603B68022BECD9FB791A
:101FE00018460C37BD465DF8047B7047503E002014
:101FF00080B483B000AF0346FB71074B1B78FA79BE
:102000009A4294BF01230023DBB218460C37BD4629
:102010005DF8047B704700BF533E002080B582B05E
:1020200000AF16491648FFF79AFE034683F00103F6
:10203000DBB2002B1DD1114B1B78FB71FFF7B4FFF6
:102040000346BB710F4B1B78DBB2BA799A4206D0BC
:102050000C4ABB791370BB791846FFF738FE084865
:10206000FFF7B0FE054B1B78DBB2FA799A42D8D164
:1020700000E000BF0837BD4680BD00BF4A3E0020DB
:10208000493E00204D3E002080B584B000AF78600E
:102090007B68FB73FB7B5B01084A1344BB60FB7BE3
:1020A000184601F069FEBB6800221A70FFF72AFF8C
:1020B000FFF7B4FF00BF1037BD4680BD583E00207B
:1020C00080B584B000AF78607B68FB73FB7B5B01FD
:1020D0000E4A1344BB60FFF715FFBB685A68BB6824
:1020E000DA60BB689A68BB681A61BB68084A5A61C3
:1020F000BB687A689A61BB680C330121184600F00E
:102100007FFB00BF1037BD4680BD00BF583E00209A
:102110008920010080B582B000AF00F0B3FD06F069
:10212000C1F9184B00221A70174B00221A70174B76
:1021300000221A70164B00221A70164B00221A70D9
:1021400000237B6008E0144A7B685B011344002293
:102150001A707B6801337B607B68012BF3D9002305
:102160003B6007E00D4A3B68134400221A703B684D
:1021700001333B603B68022BF4D900BF00BF083736
:10218000BD4680BD493E00204B3E00204D3E002014
:10219000543E0020533E0020583E0020503E002078
:1021A00080B582B000AF00237B600CE07B685B01F0
:1021B00008330A4A134404330021184600F0C2FBD6
:1021C0007B6801337B607B68012BEFD906F071F9E6
:1021D00000F064FD00BF0837BD4680BD583E0020BA
:1021E00080B582B000AF0346FB71FB79002B084A33
:1021F000FB791370BFF35F8F00BFFFF783FEFFF71C
:102200000DFFFB79002B00BF0837BD4680BD00BF26
:10221000543E002080B500AF00F080FD00BF80BDBF
:1022200080B582B000AF7860786800F07FFD03462B
:1022300018460837BD4680BD80B588B000AFF8604D
:10224000B9607A60FB7097F82830012B06D94C4BA7
:102250004C4A4FF4D9714C480FF054FE97F828308F
:102260005B014A4A1344BB6100F0A2FA7861BB6883
:10227000A3F5F0733B61BB690C33184600F074FBA7
:10228000034683F00103DBB2002B06D1404B3D4AED
:1022900040F2B9113C480FF035FEBB691B78002BAA
:1022A00006D03C4B374A4FF4DD7137480FF02AFE19
:1022B000FB78002B06D1384B324A40F2BB11324832
:1022C0000FF020FE3A69F968786900F07FFA03465A
:1022D000002B1FD0BB69FA781A70BB69FA685A6084
:1022E000BB69BA689A60BB69FA68DA60BB693A6927
:1022F0001A61BB69294A5A6197F828301A46BB69A6
:102300009A61BB690C330021184600F079FA012369
:10231000FB772FE00420FFF76BFE0346002B27D04E
:10232000BA68F968786900F051FA0346002B1FD0AB
:10233000BB69FA781A70BB69FA685A60BB69BA68F7
:102340009A60BB69FA68DA60BB69BA681A61BB69EE
:10235000134A5A6197F828301A46BB699A61BB69DB
:102360000C330121184600F04BFA0123FB7701E002
:102370000023FB77FB7F18462037BD4680BD00BF9A
:102380009C4202005C43020014420200583E0020BE
:10239000B8420200F042020014430200C1200100D2
:1023A0008920010080B483B000AF0023FB710023BB
:1023B0003B600CE00B4A3B6813441B78DBB2002BFC
:1023C00002D00123FB7105E03B6801333B603B68B1
:1023D000022BEFD9FB7918460C37BD465DF8047B1C
:1023E000704700BF503E002080B582B000AF03466A
:1023F0000A46FB711346BB71FB79022B06D90A4BC7
:102400000A4A40F20E210A480FF07CFDFB79094A86
:10241000D35CDBB2BA799A4294BF01230023DBB2CA
:1024200018460837BD4680BD2C4302008843020091
:1024300014420200503E002080B500AF00F092FC34
:102440000346184680BD80B500AF04210120FFF788
:102450001BFDFFF7E3FD00BF80BD80B500AF042189
:102460000020FFF711FDFFF7D9FD00BF80BD80B44C
:1024700089B000AF78607B68FB61FB69D3E84F3FB0
:10248000BB61BB69DBB2FB72FB7ADBB2002B04D011
:10249000BFF32F8F00BF00230FE00123FB757B6884
:1024A0003B61FA7D3969C1E8432FFB60FB68002B73
:1024B000E1D1BFF35F8F00BF012318462437BD462B
:1024C0005DF8047B704780B483B000AF7860BFF3E1
:1024D0005F8F00BF7B6800221A7000BF0C37BD46BB
:1024E0005DF8047B7047000080B487B000AF104BEC
:1024F000BB60BB68D3E84F3F7B607B68DBB2FB709F
:10250000FB78DBB20133DBB2FB75094B3B61FA7D33
:102510003969C1E8432FFB60FB68002BE7D1BFF3AB
:102520005F8F00BF00BF1C37BD465DF8047B70475E
:102530009A3E002080B485B000AF786039607A6838
:102540003B68D31AFB60FB68DB0FDBB2184614371D
:10255000BD465DF8047B704780B582B000AF7860FF
:1025600039607B681A687B685B68D0183B681A68BA
:102570003B685B6813441946FFF7DCFF03461846C7
:102580000837BD4680BD000080B584B000AF174B52
:102590001B78FB73164B1B68BB601648FFF767FF81
:1025A0000346002B17D0BB68002B02D1F3F74FFF77
:1025B0000EE0BB681B687B60BB685B683B600C4BD4
:1025C0001B68BA689A4203D139687868F3F731FF1B
:1025D0000848FFF778FF054B1B78DBB2FA7B9A427D
:1025E000D5D100BF00BF1037BD4680BD9A3E002048
:1025F0009C3E0020983E002080B592B000AF7860ED
:1026000039607B68002B05D14F4B504ABD215048A3
:102610000FF078FC4F4B1B7887F840304E4B7B64B3
:102620000023FB600023FB63002387F84330002373
:1026300087F842307B6C7B637B6B53E8003F3B63E6
:102640003B6BFB63FB6B002B07D0FA6B7B689A42FA
:1026500003D0FB6B10337B64ECE73E4B1B78DBB2A3
:1026600097F840209A4229D1FA6B7B689A4212D19E
:10267000FB6B1B69FB60384B1B68FA6B9A420ED1EF
:10268000FB68002B03D0012387F8433007E00123C8
:1026900087F8423003E0BFF32F8F00BF10E0FB68E4
:1026A000FB627B6CBB62B96AFA6A41E800237B6219
:1026B0007B6A002BAED1FFF717FF01E000BFA9E74F
:1026C000002387F84130FB6B002B23D0012387F8D0
:1026D0004130FB6B10333B623B6A53E8003FFB61C8
:1026E000FB69BB63BB6BFA6B9A4206D11B4B174A63
:1026F0004FF4887116480FF005FCFB6B1033BA6B72
:10270000BA617B617969BA6941E800233B613B6941
:10271000002BDED13B68002B03D03B6897F84120AB
:102720001A7097F84330002B03D197F84230002BF2
:1027300001D0012300E0002303F00103DBB21846BF
:102740004837BD4680BD00BFAC4302007444020060
:10275000BC4302009A3E00209C3E00201844020028
:1027600080B400AF084B00221A60084B00221A7098
:10277000074B00221A70074B00221A7000BFBD469B
:102780005DF8047B704700BF9C3E0020983E00200F
:10279000993E00209A3E002080B500AFF3F757FE27
:1027A000024B00221A6000BF80BD00BF9C3E00208B
:1027B00080B500AFF3F72CFE0346184680BD80B508
:1027C00000AFF3F72EFE0346184680BD80B487B0F5
:1027D00000AFF860B9607A60BA687B6813447B61C7
:1027E0007A69FB68D31A3B613B69002BCCBF01239C
:1027F0000023DBB218461C37BD465DF8047B7047EA
:1028000080B58CB000AF78600B46FB707B68002B06
:1028100006D1444B444A4FF4AA7144480FF072FB6E
:102820007B689B68002B06D1414B3F4A40F2551113
:102830003E480FF067FBFB78002B08D0F3F7F1FD63
:1028400003465A1E7B685B681A447B685A60002105
:102850007868FFF7D1FE0346002B01D0FFF794FE06
:10286000344B1B7887F82730334BFB620023BB6265
:10287000FB6AFB61FB6953E8003FBB61BB693B62DC
:102880003A6A7B689A4206D12C4B274A4FF4B871BA
:1028900026480FF037FB3B6A002B02D10023BB62B6
:1028A0000DE0396A7868FFF757FE0346002B02D027
:1028B0003B6ABB6203E03B6A1033FB62D8E71D4B07
:1028C0001B78DBB297F827209A4222D1BA6A7B683C
:1028D0009A4206D11A4B144A40F2891113480FF05C
:1028E00011FB7B68BA6A1A617B687B61FB6A3B619A
:1028F00039697A6941E80023FB60FB68002BAFD19E
:10290000FFF7F2FD00BF0C4B1B687A689A4204D1B6
:1029100001E000BFA4E7FFF737FE00BF3037BD4638
:1029200080BD00BFAC43020084440200BC430200EF
:10293000304402009A3E00209C3E00204C4402009D
:102940006044020080B582B000AF786039603968B9
:102950007868FFF751FE0346002B01D0FFF714FE05
:1029600000BF0837BD4680BD80B487B000AF786037
:102970000023FB75104B1B78FB73104B1B683B61EE
:1029800009E03A697B689A4202D10123FB7505E0B0
:102990003B691B693B613B69002BF2D1064B1B78FD
:1029A000DBB2FA7B9A42E3D1FB7D18461C37BD4669
:1029B0005DF8047B704700BF9A3E00209C3E0020DB
:1029C00080B584B000AF1448FFF751FD0346002BDB
:1029D0001CD0124B1B68FB60FB68002B13D0FB68FC
:1029E0009B68BB60FB68DB687B60FB1C1946F86872
:1029F000FFF702FEFB78002B05D0BB68002B02D04E
:102A0000BB68786898470448FFF75DFDFFF7BCFD99
:102A100000BF1037BD4680BD993E00209C3E00207F
:102A200080B400AF00BFBD465DF8047B704780B541
:102A300082B000AF78600B46FB701346BB70BA786B
:102A400097F9033019467868FEF7F4FE00BF08379F
:102A5000BD4680BD80B582B000AF0346FB71FB79F7
:102A60001846F4F7BFFD00BF0837BD4680BD80B5EE
:102A700084B000AFF860B96011461A460B46FB718E
:102A80001346BB71BB7997F90720B968F868FEF760
:102A9000E6FE00BF1037BD4680BD80B582B000AFF6
:102AA00078600B46FB70FB7819467868F4F778FE7F
:102AB00000BF0837BD4680BD80B582B000AF034679
:102AC000FB71FB791846F4F7AFFE00BF0837BD462F
:102AD00080BD80B582B000AF0346FB71FB7918461C
:102AE000FEF7DFFE00BF0837BD4680BD80B582B06F
:102AF00000AF0346FB71FB791846FEF7DDFE00BF11
:102B00000837BD4680BD80B582B000AF0346FB717B
:102B1000FB791846FEF7DBFE00BF0837BD4680BDD7
:102B200080B400AF00BFBD465DF8047B704780B540
:102B300000AFFEF703FF00BF80BD80B400AF00BF51
:102B4000BD465DF8047B704780B400AF00BFBD4652
:102B50005DF8047B704780B584B000AF0346FB711D
:102B6000FB79184604F0B0FD0346FB73FB7B184667
:102B70001037BD4680BD80B584B000AF3A601A46BC
:102B80000346FB710B46BB7113467B717B79B979A8
:102B9000F8793A6804F0C8FD0346FB73FB7B1846DE
:102BA0001037BD4680BD80B586B002AF3A601A4688
:102BB0000346FB710B46BB7113467B717A79B97979
:102BC000F879FB6901933B7E009313463A6804F061
:102BD000F7FD0346FB73FB7B18461037BD4680BDEF
:102BE00080B584B000AF03463960FB71FB7939686A
:102BF000184604F03BFE0346FB73FB7B1846103778
:102C0000BD4680BD80B584B000AF7860786804F0C0
